:020000040800F2
:1080000008FA0020D9810008999B00089F9B00086E
:10801000A79B0008AF9B0008B79B0008000000006A
:108020000000000000000000000000004D8100087A
:10803000C59B00080000000081810008DD2F0108B9
:10804000F3810008F3810008F38100085BDD00087C
:10805000F3810008F3810008F3810008F381000830
:10806000F3810008F3810008F3810008F381000820
:10807000F3810008F3810008F3810008F381000810
:10808000F3810008F3810008F3810008F381000800
:10809000F3810008F3810008F3810008F3810008F0
:1080A000F3810008F3810008F3810008F3810008E0
:1080B000F3810008B5C60008F3810008F3810008C9
:1080C000F3810008F3810008F3810008F3810008C0
:1080D000F3810008815601086FEF0108E58B020863
:1080E000F3810008F3810008F3810008F3810008A0
:1080F000F3810008F3810008F3810008F381000890
:10810000F3810008F3810008F3810008F38100087F
:10811000F3810008F381000827C70008F3810008F5
:10812000F3810008F3810008F3810008F38100085F
:10813000DFF80CD02AF0A8F9004800472196000883
:1081400008FA002080F30888704700001A4B19686D
:108150000868B0E8F00F80F309884FF0000080F362
:1081600011884EF00D0E70470000000003480068B3
:10817000006880F3088862B600DF00BF08ED00E009
:10818000EFF309800C4B1A6820E9F00F106008B576
:108190004FF0000080F311880AF013FA4FF000004E
:1081A00080F31188BDE8084019680868B0E8F00F4E
:1081B00080F30988704700BFF401002001B44FF03C
:1081C000000080F3118801BC704701B44FF000003B
:1081D00080F3118801BC7047064880470648004775
:1081E000FEE7FEE7FEE7FEE7FEE7FEE7FEE7FEE767
:1081F000FEE7FEE7E59C00083181000829F0B9BCE4
:1082000054656D636F434F32414C4C000000004495
:108210000000000086B0002005904FF4FA700BF0CB
:10822000E5F8002004F06CFEFB4CDFF8F093DFF87B
:10823000F0B34FF0000847F619664FF6FF77DFF806
:10824000E4A39AF80100012806D0022819D0F648C4
:108250000078012815D025E0002004F051FE0A2006
:108260000BF0C4F8F1A300220621012004F05FFE08
:10827000F1A300220321022004F059FE10F064F85B
:1082800010E0002004F03CFEF0A3002206210120B3
:1082900004F04DFEE8A300220321022004F047FE73
:1082A00010F052F8ED48007838B101208AF8020049
:1082B0004FF47A700AF012F9C1E79AF8020020B17F
:1082C0008AF80280002004F01BFE9AF80400D528EA
:1082D00001D0D42809D1E2490978012905D1E14921
:1082E00008220A70E04901220A70E0490978082949
:1082F00045D2DFE801F004537FD2B9CDD2C3DC48C8
:10830000007820B3002505EB8500CDE90076C2009A
:1083100000212023084608F020F96D1CEDB2062D3F
:10832000F1D3CDE9017656200E2100901E23D14ACB
:10833000084608F09DF9D048007808B3B4F9141045
:108340000122002008F04DFBC94880F80080CDE9EB
:10835000017656200E2100901E23C64A084608F0DA
:1083600087F9C54D287890B1B4F914100122002086
:1083700008F037FB99F800001E2800D928788CE017
:108380000022B4F90C10104608F02BFBDCE70022A9
:10839000B4F90C10104608F024FBEBE7B448007861
:1083A000F8B1CDE90076202356221E21002008F0E6
:1083B000D4F8002505EB8500CDE90076C200002148
:1083C0002023084608F0C9F80022B4F9041010462A
:1083D00008F007FB6D1CEDB2072DEBD3A44880F825
:1083E00000800022B4F90410104608F0FAFA99F857
:1083F000000052E0D22805D0D32803D0342801D081
:10840000D9284AD19A48007810B3CDE900762023C4
:1084100056221E21002008F0A0F8002505EB85005B
:10842000CDE90076C20000212023084608F095F827
:108430006D1CEDB2072DF1D3DBF86C0029F040FD87
:1084400001B20022104608F0CCFA894880F800807A
:10845000DBF86C0029F034FD01B20022104608F070
:10846000C0FA99F8000018E0342816D18348002299
:10847000008801B2104608F0B4FA0EE034280CD19E
:108480007F480022B0F90A10104608F0AAFA04E06A
:1084900000221146104608F0A4FA7A48007807280E
:1084A00042D2DFE800F004507C41F5F3B800764892
:1084B000007820B3002505EB8500CDE90076C200E9
:1084C00020235021002008F048F86D1CEDB2072D44
:1084D000F1D3CDE9017656200E2100906E23654A36
:1084E000084608F0C5F864480078F0B10122B4F9F4
:1084F0001410104608F075FA634880F80080CDE942
:10850000017656200E2100906E235A4A084608F044
:10851000AFF85948007878B10122B4F91410104628
:1085200008F05FFA99F80000F4E0B4F90C100022AA
:10853000012008F056FADFE7B4F90C100022012000
:1085400008F04FFAEEE750480078F8B1CDE9007630
:10855000202356226E21002007F0FFFF002505EBA7
:108560008500CDE90076C20020235021002007F0CD
:10857000F4FF6D1CEDB2072DF1D3B4F90410002205
:10858000012008F02EFA404880F80080B4F9041069
:108590000022012008F025FA99F80000BAE09AF8C4
:1085A0000400D22805D0D32803D0342801D0D928FC
:1085B00030D13548007810B3CDE90076202356221B
:1085C0006E21002007F0C9FF002505EB8500CDE9ED
:1085D0000076C20020235021002007F0BEFF6D1C52
:1085E000EDB2072DF1D3DBF86C0029F069FC01B284
:1085F0000022012008F0F5F9234880F80080DBF81C
:108600006C0029F05DFC01B20022012008F0E9F9BC
:1086100099F800007EE047E0FC09002058030020A4
:108620009086002000000020B30200205570646195
:1086300074696E672E2E2E00446F6E277420706F43
:10864000776572206F6666210000000052657374C2
:10865000617274696E672E2E2E0000005C8D002002
:108660009F000020A6000020BD020020A4000020E2
:10867000BB0200201E50040854030020CE0400203A
:10868000AE8E0020A5000020BC02002018E0FFE70D
:108690009AF8040034283DD1FE480022008801B237
:1086A000012008F09EF935E09AF80400342831D111
:1086B000F9480022008801B2012008F092F929E06F
:1086C0009AF80400D62801D0D72823D1F349087995
:1086D00010B102280AD013E0C878F14A105C059066
:1086E0004869F04929F007FA049009E0EC48CA7893
:1086F0000930105C05904869EB4929F0FCF90490B9
:10870000DDE90410E94A19F0AFFF0022114601200B
:1087100008F067F9E6480078092830D2DFE800F071
:10872000053E63D7D7B2B8D7C000DFF888A39AF860
:108730000000C8B1002505EB8500CDE90076820078
:1087400020239E21012007F008FF6D1CEDB20C2DA7
:10875000F1D3D948007898B1B4F91410012202205D
:1087600008F03FF98AF80080D348007878B1B4F96E
:1087700014100122022008F034F999F80000A6E054
:10878000B4F90C100022022008F02BF9EAE7B4F942
:108790000C100022022008F024F9EEE7DFF814A301
:1087A0009AF80000B0B1002505EB8500CDE9007610
:1087B000820020239E21012007F0CFFE6D1CEDB228
:1087C0000C2DF1D3B4F904100022022008F009F9AD
:1087D0008AF80080B4F904100022022008F001F9A0
:1087E00099F8000073E09AF80400D22803D0D32847
:1087F00001D0D9286BD1DFF8BCA29AF8000038B3B9
:10880000002505EB8500CDE90076820020239E211E
:10881000012007F0A2FE6D1CEDB20C2DF1D3A7488C
:10882000007850B9CDE901764FF48470372100907B
:10883000AA23A34A084607F01BFFDBF86C0029F0C7
:108840003FFB01B20022022008F0CBF88AF800803A
:108850009A48007850B9CDE901764FF484703721F9
:108860000090AA23964A084607F002FFDBF86C0046
:1088700029F026FB01B20022022008F0B2F899F894
:10888000000024E000221146022008F0AAF81EE0B1
:1088900081480022008801B2022008F0A2F816E008
:1088A000844D287898B1CDE901764FF48470372152
:1088B0000090AA23834A084607F0DAFE8248002285
:1088C000B0F90010022008F08CF885F800807B4891
:1088D000007800283FF4ECAC07F08DFFE8E47B4E15
:1088E000002786F83C707AA018F057FC64200AF044
:1088F0007DFD15F0A2FD05F043F896F83C00012837
:1089000038D11E36717C3170B07E7072B08B708140
:108910002E2003F03AFE717A3B2003F036FE708978
:10892000010A3C2003F031FEB07A1E3EC1B23D2068
:1089300003F02BFE002574191A34617C2170A07D90
:108940006071A07E607205F12F0003F01EFE617958
:1089500005F1330003F019FE617A05F1370003F0E9
:1089600014FE6D1CEDB2042DE5D35D4901200870A5
:1089700086F83C704FF47A7009F0B0FDB9E701F069
:1089800080BE70B5574814F0D4FF22F07BFC232042
:1089900003F0CAFD0446242003F0C6FD44EA002487
:1089A000252003F0C1FD44EA0044262003F0BCFD6D
:1089B00044EA006045494C4C421C2CD058B3E0605E
:1089C00008794A490870E06822F063FC21F084F9D4
:1089D0004FF0FF3015F007F9207902250021444AB5
:1089E000444B454C342822D0D42825D0D52823D038
:1089F000D22825D0D32823D0D92821D0D62824D0B6
:108A0000D72822D008201070042018702170BDE8EB
:108A1000704013F067BE0878CA784B7840EA02606D
:108A20008A78120442EA03221043E060C8E7052076
:108A300010701D702170EAE715701D702170E6E757
:108A40000320107018702170E1E701201070187079
:108A50002170DCE70CF018FF2848294900780870DD
:108A600028A018F09AFB64200AF0C0FC284F294C7B
:108A70001D4D0026387830B1401EC0B23870012834
:108A800001D113F0CDFD0CF0CEFE207800B143E013
:108A900049E00000CE040020D2040020888D002090
:108AA000869104080000C84200002041288D002063
:108AB000A6000020BD02002054030020A7000020D3
:108AC0001EAB030856710408CE8C0020087B0020E2
:108AD000466C617368205461736B0D0A00000000DE
:108AE000B3020020747C002000000020B9020020A6
:108AF000EE040020EF040020F1040020C302002057
:108B0000C4020020434F4D4D205461736B0D0A0089
:108B1000C1020020BF0200202078401E2070207873
:108B200008B90CF0A5FD2878012802D0022804D04D
:108B300009E02E700CF09CFD05E02E70FFF721FF80
:108B4000002023F081FEFFF71AFF0A2009F0C6FC7F
:108B500090E786B0FE4C002084F83D00FFF711FF3F
:108B6000002023F001F8002023F06EFEF9A018F099
:108B700014FB64200AF03AFC4FF41675A07C68B927
:108B8000009000232A46F64901A822F052FB024633
:108B900022B10023F24901A823F027FE052009F0A5
:108BA0009DFCEBE72DE9F041EE48C17800290CD19E
:108BB0000121C1704FF4FA7110300AF031FCE9481C
:108BC00042F2107118300AF02BFC0BF0DEFEE64F7B
:108BD000388018B34FF400600AF08DFCE34CA18993
:108BE00088420BD101200AF0DBFD3888002855D0DF
:108BF0000BF079FDBDE8F0410BF0CFBE40F606006A
:108C00000AF079FCA189884248D10BF020FD388810
:108C1000002843D0BDE8F0410BF0BFBED148103072
:108C20000AF010FC002839D0CE4810300AF0FFFBC3
:108C30000024CF4DCF4E04EB840005EBC000306024
:108C400002200AF0ADFD388818B10BF04CFD0BF096
:108C5000A4FE641CE4B2142CEDD30024C64DC74E10
:108C600005EB8410306005200AF09AFD388818B1B1
:108C70000BF039FD0BF091FE641CE4B20A2CEFD32B
:108C8000B84818300AF0DEFB002807D0B548183085
:108C90000AF0CDFBBDE8F0410BF05DBCBDE8F08112
:108CA00064200AF0A3FBFFF76AFEFFF77BFF0520B5
:108CB00009F014FCF7E72DE9FC5F03F033FC4520D5
:108CC00006F033FF16F088FE002003F02DFCDFF8DD
:108CD000808288F80000012003F026FC88F801005B
:108CE000022003F021FC88F80200032003F01CFCA2
:108CF00088F803000C2003F017FC9A4C20724421E2
:108D0000042003F042FC0021052003F03EFC062075
:108D100003F00AFC88F804000227FF2800D060B99D
:108D2000607910B188F8047002E0FE2088F8040031
:108D300098F80410062003F028FC072003F0F4FB49
:108D400088F80E002071082003F0EEFB88F80F0071
:108D5000FF2800D028B9082188F80F10082003F058
:108D600014FC102003F0E0FB88F80D00112003F044
:108D7000DBFB88F810007B48814C00260079D52861
:108D80001ED0D4281CD034281AD02670152003F009
:108D9000CBFB88F80C000125052805D9294688F861
:108DA0000C50152003F0F1FB98F80C00754C4FF0B7
:108DB000030A062842D2DFE800F01019222A323ACC
:108DC0004FF4F56003F0B0FB20700028DED00128DE
:108DD000DCD00228DAD02670D8E74FF41650C8F855
:108DE00008000AF097F90620207027E04FF496401B
:108DF000C8F808000AF08EF984F800A01EE04FF4CD
:108E00001640C8F808000AF085F9277016E04FF4FC
:108E10006140C8F808000AF07DF925700EE04FF4B3
:108E2000E130C8F808000AF075F9257006E04FF443
:108E30009630C8F808000AF06DF92570142003F088
:108E400073FB88F81200032806D028B1514688F831
:108E500012A0142003F099FB0024E94604F1280035
:108E600003F062FB09F80400641CE4B2062CF5D39D
:108E70009DF800004FF0040BFF283ED19DF8010043
:108E8000FF283AD19DF80200FF2836D19DF8030053
:108E9000FF2832D19DF80400FF282ED19DF805004F
:108EA000FF282AD159468DF800B08DF80170352081
:108EB0008DF80200AF208DF803008DF804608DF866
:108EC0000550282003F061FB9DF80110292003F0D4
:108ED0005CFB9DF802102A2003F057FB9DF803105D
:108EE0002B2003F052FB9DF804102C2003F04DFBC7
:108EF0009DF805102D2003F048FB002008EB000230
:108F000019F800101175401CC0B20628F6D30024D1
:108F100004F12F0003F008FB09F80400641CE4B21C
:108F2000042CF5D39DF80000FF2845D19DF80100E1
:108F3000FF2841D19DF80200FF283DD19DF8030094
:108F4000FF2839D1C0218DF80010A8201CE00000B6
:108F5000087B00204D535450205461736B0D0A0060
:108F6000DC060020000000205C020020C06300201E
:108F7000C46B00207C0200200C6F002080020020C7
:108F8000C5020020C00200208DF801008DF80260AB
:108F90008DF803A02F2003F0F8FA9DF8011030207F
:108FA00003F0F3FA9DF80210312003F0EEFA9DF879
:108FB0000310322003F0E9FA002008EB000219F850
:108FC0000010917682F82B10401CC0B20428F4D314
:108FD0002E2003F0A9FA8DF80000012805D93146AA
:108FE0008DF800602E2003F0D0FA9DF8000088F87C
:108FF0001E0088F82F00002404F1330003F094FAD7
:1090000009F80400641CE4B2042CF5D39DF80000B8
:10901000FF2820D19DF80100FF281CD19DF80200F7
:10902000FF2818D19DF80300FF2814D1FF218DF8E7
:109030000360332003F0A9FA9DF80110342003F0F7
:10904000A4FA9DF80210352003F09FFA9DF8031052
:10905000362003F09AFA002008EB000219F80010FD
:10906000D17782F83010401CC0B20428F4D3002419
:1090700004F1370003F058FA09F80400641CE4B264
:10908000042CF5D39DF80000FF2827D19DF801009E
:10909000FF2823D19DF80200FF281FD19DF803006F
:1090A000FF281BD1C0218DF80010A8208DF80100E9
:1090B0008DF802608DF803B0372003F066FA9DF852
:1090C0000110382003F061FA9DF80210392003F0F6
:1090D0005CFA9DF803103A2003F057FA002008EBE1
:1090E000000219F8001002F8231F5174401CC0B28E
:1090F0000428F4D33B2003F017FA8DF80000FF2872
:1091000005D131468DF800603B2003F03EFA9DF812
:10911000000088F8270088F838003C2003F004FAA3
:109120008DF800003D2003F0FFF98DF801009DF857
:109130000010FF290AD1FF2808D14FF4FB70A8F8CE
:1091400028008DF80050F6208DF801009DF80100F0
:109150009DF8001040EA0120A8F82800A8F83A007D
:1091600088F83C6088F81360FC480670452003F0DE
:109170009EFAFB490870142400287DD0FF287BD07C
:10918000142800D90C70462003F091FAF5490870B4
:10919000002872D0FF2870D0142800D90C705120FC
:1091A00003F085FA0446522003F081FA44EA0020D5
:1091B000ED4C2081532003F07AFA8046542003F0CE
:1091C00076FA48EA002000B26081B4F908108142C2
:1091D00000DD20815F2003F06AFA8046602003F002
:1091E00066FA48EA0020A080612003F060FA804619
:1091F000622003F05CFA48EA002000B2E080B4F993
:109200000410814200DDA080632003F050FA804604
:10921000642003F04CFA48EA00202080652003F027
:1092200046FA8046662003F042FA48EA002000B27F
:109230006080B4F90010814200DD2080562003F0E8
:1092400036FACA49F0B3FF284ED00D70572003F00C
:109250002EFAC74C2070582003F029FA607059206C
:1092600003F025FAA0705A2003F021FAE07021786B
:1092700030390A2910D201E032E033E0617839292F
:109280000AD8302908D3A178392905D8302903D341
:10929000392801D8302818D231212170322060704D
:1092A0003320A0703420E070572003F0FEF961787D
:1092B000582003F0FAF9A178592003F0F6F9E17883
:1092C0005A2000E010E003F0F0F940F2D27420469A
:1092D00003F0EDF9A749C871FF2807D030B10DE0C0
:1092E0000F7050E70F705AE70E70AFE7012120466C
:1092F00003F0DBF9FF215E2003F0D7F95E2003F0D5
:10930000D6F99D49087040F20479484603F0CFF938
:109310009A4CA0764FF00508FF2805D184F81A80F2
:109320000521484603F0C1F940F20379484603F0AD
:10933000BEF96076FF2805D184F8198005214846DA
:1093400003F0B3F940F20279484603F0B0F98C49D2
:109350000870FF2805D181F800800521484603F0F8
:10936000A4F92661A6601522864940F2617003F0D7
:109370007AF940F2767003F09AF9044640F2777079
:1093800003F095F944EA00207F4C20804FF4EF6011
:1093900003F08DF9814640F2797003F088F949EACB
:1093A0000020608040F27A7003F081F9814640F23B
:1093B0007B7003F07CF949EA0020A08040F27C70C9
:1093C00003F075F9814640F27D7003F070F949EAC7
:1093D0000020E08040F27E7003F069F9814640F29F
:1093E0007F7003F064F949EA002020814FF4F060B7
:1093F00003F05DF9814640F2817003F058F949EAC3
:109400000020608140F2BB7003F051F95F490870A1
:109410004FF4FA64204603F04AF95D490870FF28CA
:1094200004D10E703146204603F03FF940F2D1746A
:10943000204603F03CF957490870012804D90E7002
:109440003146204603F031F95348007800287DD09A
:10945000DFF8209199F8040034280AD089F80560D3
:1094600040F2BC7003F023F94C4C2070FF2810D060
:1094700015E040F2CF74204603F019F989F8050091
:109480000128EDD9314689F80560204603F00DF931
:10949000E6E73146267040F2BC7003F006F999F811
:1094A0000400342808D0D6280FD0D7280DD0D528CE
:1094B0000ED0D4280CD00CE099F8050010B184F837
:1094C00000B006E00720207003E084F8008000E090
:1094D000267040F2BD7003F0EAF8314C2070FF288E
:1094E00005D12946257040F2BD7003F0DEF899F8E9
:1094F0000400342808D0D6280FD0D7280DD0D5287E
:109500000ED0D4280CD00CE099F8050010B106203C
:10951000207006E084F800B003E084F8008000E0EA
:10952000257040F2BE7B584603F0C1F81D4C2070F8
:10953000FF2804D139462770584603F0B6F899F849
:109540000400342830D0D62837D000E054E0D728A3
:1095500033D0D52834D0D42832D033E0F6020020DE
:10956000F8020020F90200203E03002077040020CA
:1095700078040020000000207C040020FC0900206A
:1095800059030020747C0020988C0020C004002027
:10959000C6020020C702002063000020A4000020B3
:1095A000A5000020A600002099F8050010B184F85D
:1095B00000A007E00620207004E084F8008001E0AD
:1095C00084F800A040F2C17003F071F800B10120EE
:1095D000FD49087099F80400342805D199F8050070
:1095E00008B10D7000E00E7040F2C27003F05FF839
:1095F00000B10120F5490870BDE8FC9F10B545F2A7
:10960000555001F035F8052001F035F84FF47A6037
:1096100001F034F801F03AF8BDE8104001F031B83B
:109620002DE9FF4701254FF00008E949080300F044
:10963000F4FB4FF4A06000F0BBFB482009F0A2FE51
:10964000FFF7DCFF0121142009F020FAE14F386018
:1096500009F021FBE04C206009F01DFBDF4E30607B
:109660000221052009F012FADD490860FFF787F9A9
:10967000386850B1206840B1306830B140F2B970FC
:1096800003F015F8632801D011E0FEE7422440F210
:10969000FF76FF21204603F008F8FFF770F9641CFD
:1096A000A4B2B442F5D30021102002F0FEFF40F234
:1096B000CE74204602F0FBFFCA4EB071FF2801D0E5
:1096C000012804D8FE21B171204602F0EEFF4FF4CC
:1096D000F86002F0ECFF00B10120C34F387050B1C8
:1096E000C349C248086006F023FFFFF7E4FA307967
:1096F000342809D02CE004F0FFF80022BDA3114665
:10970000104603F014FCF0E7387808BB40F27F798C
:10971000484602F0CCFF40EA080000020FFA80F849
:1097200040F27E7A504602F0C2FF40EA080404F597
:109730009670C9280CD3E1B2504602F0B6FFC4F3CC
:109740000721484602F0B1FFAF496FF0C70008811A
:10975000AE48007804F085F814F0D1FE02F03CFD2C
:109760000022ABA31146012003F0E1FB3079D2289F
:1097700003D0D32801D0D92805D140F2B77002F028
:1097800096FFA64908704FF001080024FFF7F7F88C
:10979000387860B90EE0FFF7F2F8142C1FD204F00D
:1097A000A9FAD0B1641CE4B2142009F01FFEB8F18C
:1097B000000FF0D1ADB1002299A31146022003F0B1
:1097C000B6FBFFF7DCF83079D22814D0D42812D0B9
:1097D000D62810D034280ED011E00025EAE7012564
:1097E000E8E7002292A31146022003F0A0FBE8E77D
:1097F000642009F0FBFD0BF02BF80028F8D10022C3
:109800008EA31146032003F092FB8FA017F0C5FC36
:10981000002290A31146042003F089FB642009F084
:10982000E5FDFFF7ACF840F2BA74204602F03FFFC6
:109830008A4A10800125FF280FD0401CC1B2204663
:1098400002F0A3FE30790024D2280CD0D4280AD00C
:10985000D62808D0342806D010E0294615802046A6
:1098600002F093FEEEE7CDE90054029400234FF49A
:10987000C0727BA17B48039408F0B8FC4FF0060946
:10988000CDE900944FF4207802940023424676A15B
:109890007748039408F0AAFC0720CDE9000402945D
:1098A0000023424673A17548039408F09FFC307969
:1098B0000325D22803D0D32801D0D92814D1CDE94B
:1098C0000094029400234FF480726DA16E480394BB
:1098D00008F08CFCCDE900540294002380226BA197
:1098E0006D48039408F082FC307934280AD1CDE920
:1098F0000094029400234FF4BD7268A16A48039457
:1099000008F074FC30794FF00409D6285AD0D728D3
:1099100058D0CDE9005402940023424663A169481F
:10992000039408F063FCCDE90054029400238022E4
:1099300065A16948039408F059FC4FF0050ACDE988
:1099400000A402940023802264A16648039408F0D6
:109950004DFCCDE9009402940023802262A164486A
:10996000039408F043FCCDE9009402940023802284
:1099700060A16148039408F039FC387848B1CDE91A
:1099800000A40294002380225CA15D48039408F0A7
:109990002DFCCDE900A4029400234FF4906259A15C
:1099A0005B48039408F022FC032017F09AFC3079FE
:1099B000D62808D0D72806D0CDE900540294002339
:1099C0004246A7E0B1E0AAE0A7000020A1040020E1
:1099D0000080000824030020D0030020840400201D
:1099E000940000200000002063000020C60000203A
:1099F000AC000020496E697469616C697A617469B0
:109A00006F6E2E2E2E000000988C00207C0400200B
:109A100045455020697320446F6E650004030020A3
:109A2000525443206973204661696C6564000000EC
:109A300052544320697320446F6E65004E65742054
:109A4000697320446F6E6500434F325F4E45540A80
:109A50000D000000446F6E6500000000A281002030
:109A60004E455400A18C00084D5354500000000096
:109A7000538B0008434F4D4D00000000558A0008ED
:109A8000436F325461736B001DEE0108416C6172CB
:109A90006D5461736B000000F3EE0108504D3235D8
:109AA0005461736B00000000BF7002085570646160
:109AB00074655F54656D70657261747572655F542D
:109AC00061736B00690A02087653746172745049BD
:109AD000445461736B0000004B670208464C4153CD
:109AE00048000000DF8800084F757450757400004E
:109AF000B5F501084B455900BDDE00084C43440054
:109B000015820008576966697461736B0000000074
:109B10000374020813A11848039408F067FB08F0C7
:109B200045FE04B00020BDE8F087CDE90094029422
:109B30000023802211A11748039408F057FBF2E696
:109B4000C1B2000A40EA01207047C0F30723C0F306
:109B50000741020E000640EA034040EA012010439C
:109B600070470000764765745F48756D5F5061729D
:109B7000615F5461736B0000010A020855706461F3
:109B800074655F50726573737572655F5461736B52
:109B900000000000156402080FA017F0FEBA11A023
:109BA00017F0FBFAFBE712A017F0F7FAFBE713A098
:109BB00017F0F3FAFBE714A017F0EFFAFBE716A093
:109BC00017F0EBBA16A017F0E8BA17A017F0E5BA2D
:109BD00017A017F0E2BA00004E4D49206661756C7F
:109BE0007400000068617264206661756C74000026
:109BF0004D656D204661756C7420000042757320C0
:109C00004661756C7420000055736167652046617C
:109C1000756C7420000000005356432000000000C3
:109C2000446562756720000050656E2000000000EA
:109C30005379735469636B20000000000CB5002257
:109C4000019200925148016841F4803101604FF463
:109C5000A063016801F4003100910199491C019150
:109C6000009911B901999942F3D10168890302D58C
:109C70000121009100E000920099012930D144496E
:109C80000A6842F010020A600A6822F003020A60C1
:109C90000A6842F002020A6041684160416841601E
:109CA000416841F480614160416821F47C11416068
:109CB000416841F4E8114160016841F08071016040
:109CC00001688901FCD5416821F0030141604168C8
:109CD00041F0020141604168C1F381010229FAD1DA
:109CE0000CBDABE710B52948016841F001010160E6
:109CF0004168284A114041600168274A11400160CB
:109D0000016821F480210160416821F4FE01416075
:109D10004FF41F018160FFF7E4FF21491F480860ED
:109D200010BD10B5194A506800F00C011D4B1E48BB
:109D300000290ED004290ED008290ED003605168E6
:109D4000194AC1F30311121D515C0268CA40026036
:109D500010BD0360F3E70360F1E7516801F470118F
:109D6000536803F48033022404EB914133B1536808
:109D70009B0307D50D4B59430160E0E70B4B59435B
:109D80000160DCE7074B59430160D8E7001002404F
:109D9000002002400000FFF8FFFFF6FE00800008F0
:109DA00008ED00E000127A002000002000093D00CC
:109DB0002A4908432A490860704770B50F23C278C2
:109DC00001260178002A1ED0254A126802F4E062BA
:109DD000C2F5E062120AC2F10404D3404578A540FE
:109DE00082781A402A43120101F1E02181F800240F
:109DF000007800F01F018E404009800000F1E02053
:109E0000C0F8006170BD01F01F0086404809800065
:109E100000F1E020C0F8806170BD124A114001439A
:109E20000F48001F016070470D4A121D002903D022
:109E300011680143116070471168814311607047D8
:109E40004FF0E021042804D0086920F004000861E4
:109E50007047086940F00400086170470000FA0587
:109E60000CED00E080FFFF1F10B5DB4988420AD1EE
:109E700044150121204600F052FD2046BDE8104067
:109E8000002100F04CBDD54988420AD104150121BA
:109E9000204600F044FD2046BDE81040002100F0BF
:109EA0003EBDCF4988420AD10121CC03204600F0B3
:109EB00036FD2046BDE81040002100F030BD10BD49
:109EC00010B54268C74B1A400C790B6842EA04226D
:109ED000134343608268C44B1A40D1E902432343D1
:109EE0004C7942EA440213438360C26A22F470024E
:109EF000097C491EC9B242EA0151C16210BD00216C
:109F00000160017141718160C1600121017470477C
:109F1000002904D0816841F00101816070478168A7
:109F200021F0010181607047002904D0816841F46B
:109F3000807181607047816821F480718160704711
:109F4000C9B2002A03D042680A434260704742689F
:109F50008A4342607047816841F008018160704720
:109F6000014600208968090700D5012070478168F3
:109F700041F004018160704701460020896849076B
:109F800000D501207047002904D0816841F4A00168
:109F900081607047816821F4A001816070470146AB
:109FA00000208968490200D501207047426822F4E8
:109FB0006042491E42EA413141607047002904D0A5
:109FC000416841F4006141607047416821F40061DB
:109FD0004160704770B5072609290AD9C568A1F103
:109FE0000A0404EB4404A640B543A3401D43C560E6
:109FF00007E0056901EB4104A640B543A3401D43BA
:10A0000005611F23072A09D2446B521E02EB82020C
:10A0100093409C4391400C43446370BD0D2A09D288
:10A02000046BD21F02EB820293409C4391400C438D
:10A03000046370BDC46A0D3A02EB820293409C43F4
:10A0400091400C43C46270BD002904D0816841F482
:10A05000801181607047816821F4801181607047B0
:10A06000C06C80B270475C484C3000687047002973
:10A0700004D0416841F4806141607047416821F437
:10A08000806141607047002904D0416841F48051EB
:10A0900041607047416821F4805141607047826897
:10A0A00022F4E0420A4382607047002904D08168AC
:10A0B00041F4004181607047816821F40041816072
:10A0C0007047002904D0816841F402118160704713
:10A0D000816821F40211816070470146002089687F
:10A0E000890200D50120704770B5072609290AD9D1
:10A0F000C568A1F10A0404EB4404A640B543A3409B
:10A100001D43C56007E0056901EB4104A640B54366
:10A11000A3401D430561836BC3F30154121B921CC2
:10A1200002EB82021F249440A34391400B438363BC
:10A1300070BD826B22F44012491E42EA01518163D4
:10A14000704708B50090009808440090009802609D
:10A1500008BD08B500900098084428300090009889
:10A16000006880B208BD4268204B1A400A43426032
:10A170007047416282627047426822F01F020A43C0
:10A180004260704714490831002804D0086840F440
:10A19000000008607047086820F4000008607047FD
:10A1A0000246002012680A4200D001207047C943CD
:10A1B0000160704710B5024600200B0A5468C9B20E
:10A1C0000C401168194202D0002C00D0012010BDB3
:10A1D000090AC9430160704700240140002801407A
:10A1E000003C0140FFFEF0FFFDF7F1FFFFFD3FFFE8
:10A1F00001684FF6FE72114001600021016041606C
:10A200008160C1607249724A0839904204D148683D
:10A2100040F00F00486070476D4A1432904204D1FC
:10A22000486840F0F00048607047694A2832904220
:10A2300004D1486840F4706048607047644A3C321A
:10A24000904204D1486840F4704048607047604ACA
:10A250005032904204D1486840F470204860704702
:10A260005B4A6432904204D1486840F47000486010
:10A270007047574A7832904204D1486840F0706085
:10A2800048607047534A111F904204D1086840F05B
:10A290000F00086070474F4A1432904204D108689A
:10A2A00040F0F000086070474A4A2832904204D1DA
:10A2B000086840F4706008607047464A3C3290423B
:10A2C00004D1086840F4704008607047414A503239
:10A2D0009042FAD1086840F470200860704730B5A9
:10A2E000026847F6F0739A430C6A8B682343D1E9FE
:10A2F00004452C4323438C692343CC6923434C6A94
:10A3000023438C6A234313430360CA6842600A688C
:10A3100082604968C16030BD002101604160816098
:10A32000C160016141618161C1610162416281621B
:10A330007047002904D0016841F0010101607047B5
:10A3400001684FF6FE72114001607047002A03D089
:10A3500002680A430260704702688A4302607047DD
:10A3600041607047406880B2704702460020D100CB
:10A3700003D518490839096802E015490839096800
:10A38000114200D001207047C10003D51149091FB7
:10A39000086070470E49083948607047024600203F
:10A3A000D10003D50B490839096802E0084908398A
:10A3B0000968114200D001207047C10003D505494A
:10A3C000091F08607047024908394860704700005B
:10A3D000080002400804024010B59C49884209D197
:10A3E0000121042000F09BFA0021BDE81040042068
:10A3F00000F095BA9649884209D10121082000F061
:10A400008EFA0021BDE81040082000F088BA91497A
:10A41000884209D10121102000F081FA0021BDE815
:10A420001040102000F07BBA8B49884209D10121ED
:10A43000202000F074FA0021BDE81040202000F038
:10A440006EBA8649884209D10121402000F067FA9E
:10A450000021BDE81040402000F061BA80498842E8
:10A4600009D10121802000F05AFA0021BDE81040F6
:10A47000802000F054BA7B4988420AD1841501211A
:10A48000204600F04CFA2046BDE81040002100F0C4
:10A4900046BA10BD10B50121084600F040FA00216F
:10A4A000BDE81040012000F03ABA2DE9F041002249
:10A4B000CC7804F00F03E40601D58C7823430C78A4
:10A4C0004FF00F0714F0FF0F4FF0010C1CD0056880
:10A4D0000CFA02F40E882640A64211D1960007FA23
:10A4E00006F825EA080503FA06F848EA0505CE78D5
:10A4F000282E02D0482E02D002E0446100E0046120
:10A50000521C082AE4D305600A88FF2A1ED9456830
:10A51000002202F108060CFA06F40E882640A64234
:10A5200010D1960007FA06F825EA080503FA06F89E
:10A5300048EA0505CE78282E00D14461CE78482E11
:10A5400000D10461521C082AE3D34560BDE8F081C4
:10A550004FF6FF710180022181700421C1707047A4
:10A560000246002092680A4200D0012070478068AD
:10A5700080B2704702460020D2680A4200D0012013
:10A580007047C06880B27047016170474161704791
:10A59000002A01D00161704741617047C160704776
:10A5A00041F4803282618161826181698069704792
:10A5B00010B52D4B1A684FF68074224042EA001005
:10A5C0000843186010BD2949C8617047F0B5264C92
:10A5D000002801DAE36900E06368C0F30346420D36
:10A5E000120185B2C0F301579540032F07D0C20274
:10A5F0000CD50322B240934343F0706209E023F08C
:10A600007062636823F07063636002E0AB4343F001
:10A61000706201B12A43002801DAE261F0BD626094
:10A62000F0BD10B58A07120F0F23934021F00304E9
:10A630000D4921448C689C438C608B689040034397
:10A640008B6010BD0949DC3108607047000801408B
:10A65000000C0140001001400014014000180140AE
:10A66000001C014000200140000001400000204289
:10A670000D49086070470C49486070470A49886076
:10A68000704709494AF6AA200860704706494CF607
:10A69000CC400860704701460020034AD2680A4255
:10A6A00000D001207047000000300040B44801682D
:10A6B00041F0010101604168B24A11404160016806
:10A6C000B14A11400160016821F4802101604168B4
:10A6D00021F4FE0141604FF41F0181607047A849D9
:10A6E0000A6822F480320A600A6822F480220A6032
:10A6F000B0F5803F07D0B0F5802F03D1086840F453
:10A70000A02008607047086840F4803008607047F7
:10A710000346002059099A4A01290AD002290AD081
:10A72000516A03F01F02012393400B4200D0012025
:10A7300070471168F5E7116AF3E718B5002000903B
:10A740004FF4A0643120FFF7E3FF0099491C00910A
:10A750000099A14201D00028F4D03120FFF7D8FFA2
:10A7600008B1012018BD002018BD854A116821F0EC
:10A77000F80141EAC00010607047844908607047E2
:10A780007F4B5A6822F47C1208431043586070478C
:10A790007E49086670477A4A516821F003010143F7
:10A7A000516070477648406800F00C007047744A6A
:10A7B000516821F0F001014351607047704A5168BF
:10A7C00021F4E0610143516070476D4A516821F402
:10A7D000605141EAC00050607047694A002903D0C7
:10A7E000517A014351727047517A814351727047D7
:10A7F0006649D83108607047614A516821F4404188
:10A800000143516070475E49002220310A7001F80F
:10A810002029012805D0042802D1052081F8200034
:10A820007047012081F8200070475949086070473F
:10A8300053490A6A02430A6270475549443908601D
:10A84000704710B54E4A516801F00C01514B002978
:10A8500027D0042927D0082927D00360516801F0A8
:10A86000F00109094C4B5C5C0168E14041605468AF
:10A8700004F4E064240A1C5D21FA04F48460546842
:10A8800004F46054E40A1B5DD940C160526802F4CC
:10A890004042920B404B1B1F9A5CB1FBF2F10161ED
:10A8A00010BD0360DAE70360D8E7516801F4701166
:10A8B000536803F48033022404EB914133B15368AD
:10A8C0009B0307D5354B59430160C7E7334B5943C9
:10A8D0000160C3E72F4B59430160BFE7284A0029B5
:10A8E00003D05169014351617047516981435161FE
:10A8F0007047234A002903D0916901439161704751
:10A9000091698143916170471D4A002903D0D16943
:10A910000143D1617047D1698143D1617047184AC1
:10A92000002903D0D1680143D1607047D1688143C9
:10A93000D1607047124A002903D0116901431161A7
:10A9400070471169814311617047114940390860AE
:10A9500070470E49C86470470949C8717047084874
:10A96000416A41F080714162704701460020044A0B
:10A9700092680A4200D001207047014988727047EE
:10A98000001002400000FFF8FFFFF6FE0000424208
:10A990008004424200127A003800002000093D0085
:10A9A0004F4A002903D01188014311807047118854
:10A9B0008143118070474A48001D018841F0100111
:10A9C000018070474648001D018821F01001018078
:10A9D000704743481C30008841491831098840EAD3
:10A9E0000140704700B50246FFF7E5FF3C49100CF7
:10A9F00018310880081D02805DF804EBE2E700B51D
:10AA00000246FFF7D8FF3649C2F3034008310880F9
:10AA1000081D02805DF804EBD4E700B50246FFF79D
:10AA2000CAFF2F49100C20310880081D02805DF8F4
:10AA300004EBC7E72A48103000880007010B2848BC
:10AA40001430008808437047002025494FF496735E
:10AA5000091D05E0401C80B2984201D301207047D7
:10AA60000A889206F6D51F49401D4881002070478C
:10AA700000201B49091D0A8822F008020A804FF4B1
:10AA8000967305E0401C80B2984201D301207047C4
:10AA90000A881207F6D50020704701460020104AA8
:10AAA000121D12880A4200D0012070470C49091D6E
:10AAB0000A8882430A8070470949091D0988C2B281
:10AAC0001140074A1288024202D009B101207047A2
:10AAD000002070470249091D0A8882430A80704796
:10AAE00000280040A281002010B5A94988420AD15F
:10AAF000841401212046FFF712FF2046BDE81040D4
:10AB00000021FFF70CBFA34988420AD10414012198
:10AB10002046FFF70FFF2046BDE810400021FFF759
:10AB200009BF9D4988420AD1C41301212046FFF77D
:10AB300001FF2046BDE810400021FFF7FBBE10BD1D
:10AB400030B5028802F441530A884C88CD882243EC
:10AB50008C882C4322430C8922434C8922438C89C4
:10AB60002243CC8922431A430280828B22F4006262
:10AB70008283098A018230BDF0B585B005460C4656
:10AB8000022000210126AA8B4FF240031A40AA831B
:10AB900002222A84AF8BA268022A21D0A08800B1A9
:10ABA00002266846FFF74DFE0098E188B1F5007F68
:10ABB0002CD07101B0FBF1F000EB8000A1684000E7
:10ABC000B0FBF1F0401D80B20A21B0FBF1F000F0C3
:10ABD0000101401AC0F34F004FF6FF7202EA012153
:10ABE000821EFE2A01D302200021E288084302438C
:10ABF0002A8420886188A2890843A18811430843D8
:10AC0000384340F40060A88305B0F0BD000A00EBB3
:10AC10008000A1684000B0FBF1F0401D80B2D3E796
:10AC20000021018041808180C18001814181818139
:10AC3000C18107210182704700210180418081800C
:10AC4000C1800222826081817047002904D001887E
:10AC500041F0400101807047018821F040010180EE
:10AC60007047002904D0818B41F480618183704753
:10AC7000818B21F4806181837047090901238B4016
:10AC800099B2002A03D082880A4382807047828862
:10AC90008A4382807047002A03D082880A438280D8
:10ACA000704782888A43828070478181704780899B
:10ACB0007047A1F57E42FF3A04D0018841F48071CB
:10ACC00001807047018821F480710180704700295C
:10ACD00004D0818841F0040181807047818821F08F
:10ACE000040181807047028822F400620280028899
:10ACF0000A4302807047018841F480510180704707
:10AD0000002904D0018841F4005101807047018876
:10AD100021F4005101807047012901D0008B704758
:10AD2000808A7047008A7047B1F5804F04D001884F
:10AD300021F4804101807047018841F48041018005
:10AD400070470246002012890A4200D00120704755
:10AD5000C9430181704730B50246002001F00F035E
:10AD6000012505FA03F4A3B2090905FA01F4A4B216
:10AD70009188214012891A4202D0002900D0012076
:10AD800030BD01F00F0201219140C943018170479C
:10AD90000030014000380040003C004010B5FE4942
:10ADA00088420AD1C41401212046FFF7B8FD20468D
:10ADB000BDE810400021FFF7B2BDB0F1804F0CD0CC
:10ADC000F649884213D101210220FFF7B3FD00218B
:10ADD000BDE810400220FFF7ADBD01210846FFF796
:10ADE000A9FD0021BDE810400120FFF7A3BDEC49FB
:10ADF000884209D101210420FFF79CFD0021BDE814
:10AE000010400420FFF796BDE649884209D1012190
:10AE10000820FFF78FFD0021BDE810400820FFF754
:10AE200089BDE149884209D101211020FFF782FD47
:10AE30000021BDE810401020FFF77CBDDB498842AF
:10AE400009D101212020FFF775FD0021BDE8104048
:10AE50002020FFF76FBDD64988420AD14414012152
:10AE60002046FFF75CFD2046BDE810400021FFF7BB
:10AE700056BDD04988420AD10121CC042046FFF7B3
:10AE80004EFD2046BDE810400021FFF748BDCA49ED
:10AE900088420AD101210C052046FFF740FD2046DB
:10AEA000BDE810400021FFF73ABDC44988420AD1ED
:10AEB00001214C052046FFF732FD2046BDE8104039
:10AEC0000021FFF72CBDBE49884209D10121402055
:10AED000FFF730FD0021BDE810404020FFF72ABDFC
:10AEE000B849884209D101218020FFF723FD0021C4
:10AEF000BDE810408020FFF71DBDB34988420AD14C
:10AF0000841501212046FFF715FD2046BDE81040BD
:10AF10000021FFF70FBDAD4988420AD101210C0481
:10AF20002046FFF7FCFC2046BDE810400021FFF75B
:10AF3000F6BCA74988420AD101214C042046FFF7FC
:10AF4000EEFC2046BDE810400021FFF7E8BCA14917
:10AF500088420AD101218C042046FFF7E0FC2046FC
:10AF6000BDE810400021FFF7DABC10BD30B5028803
:10AF7000894C8F4DA0420DD0A8420BD0B0F1804F2C
:10AF800008D0864B984205D0854B984202D0854B1D
:10AF9000984203D122F070034A881A43824B9842A8
:10AFA00006D0824B984203D022F44073CA881A43D9
:10AFB00002808A8882850A880285A0420AD0A84237
:10AFC00008D0824A904205D0814A904202D0814AFC
:10AFD000904201D1097A01860121818230BD30B5CC
:10AFE000028C22F001020284028C8388048B24F0FC
:10AFF000700424F003050C882C4322F002020D8912
:10B0000015434A882A43644DA8420BD0684DA84294
:10B0100008D06E4DA84205D06D4DA84202D06D4DAE
:10B02000A8420FD122F008054A892A4322F00405DC
:10B030008A882A4323F4807323F400738D891D4387
:10B04000CB892B4383800483C9888186028430BDE9
:10B0500070B5028C22F010020284028C8388048B6B
:10B0600024F4E04424F440760D884FF6FF7404EA9B
:10B070000525354322F020020E8904EA0616164300
:10B080004A8804EA02123243434EB04202D0484E8C
:10B09000B04217D122F080024E8904EA0616164308
:10B0A00026F040068A8804EA0212324323F48063C1
:10B0B00023F400638E8904EA86061E43CB8904EAE2
:10B0C0008303334383800583C9880187028470BD6D
:10B0D00070B5028C22F480720284028C8388848B87
:10B0E00024F0700424F003040D88254322F4007238
:10B0F0000E894FF6FF7404EA062616434A8804EACE
:10B1000002223243244EB04202D0294EB04217D11F
:10B1100022F400664A8904EA0222324322F480665D
:10B120008A8804EA0222324323F4805323F4005332
:10B130008E8904EA06161E43CB8904EA03133343BF
:10B1400083808583C9888187028470BD70B5028C35
:10B1500022F480520284058C8288838B23F4E0439E
:10B1600023F440760C884FF6FF7303EA042434433B
:10B1700025F400550E8903EA06362E434D8803EA6E
:10B1800005353543044EB04202D0094EB04226D1B7
:10B1900022F480468A891FE0002C01400004004010
:10B1A00000080040000C0040001000400014004067
:10B1B00000340140004C0140005001400054014067
:10B1C00000180040001C00400020004000400140EA
:10B1D000004401400048014003EA82123243828069
:10B1E0008483C988A0F84010058470BD828B22F446
:10B1F00040628283828B4FF6FF7303EA01210A4388
:10B2000082837047F0B5048C24F480540484868BC8
:10B21000048C4FF6FF7505EA013726F4734605EAFC
:10B220000222324305EA03331343F74A90420ED019
:10B23000F64A90420BD0B0F1804F08D0F44A9042C9
:10B2400005D0F44A904202D0F34A904205D124F44A
:10B250000051394341F4805104E024F402420A438E
:10B2600042F4805183830184F0BD828B22F00C0272
:10B270008283828B0A4382837047F0B5048C24F466
:10B2800080740484858B048C4FF6FF7707EA0126CF
:10B2900025F0F30507EA031313432B43DA4A9042E0
:10B2A0000ED0DA4A90420BD0B0F1804F08D0D84A85
:10B2B000904205D0D74A904202D0D74A904205D159
:10B2C00024F40071314341F4807104E024F42062DD
:10B2D0000A4342F4807183830184F0BD028B22F41F
:10B2E00040620283028B4FF6FF7303EA01210A4397
:10B2F00002837047F0B5048C24F010040484068B9C
:10B30000048C4FF6FF7505EA011726F4734605EA2B
:10B310000333334305EA02221A43BB4B98420ED053
:10B32000BA4B98420BD0B0F1804F08D0B84B98423E
:10B3300005D0B84B984202D0B74B984205D124F0C3
:10B340002001394341F0100104E024F0A0030B4335
:10B3500043F0100102830184F0BD028B22F00C0245
:10B360000283028B0A430283704770B5048C24F079
:10B3700001040484058B048C25F0F3054FF6FF7659
:10B3800006EA031313432B439F4A90420ED09F4A71
:10B3900090420BD0B0F1804F08D09D4A904205D02A
:10B3A0009C4A904202D09C4A904205D124F002026D
:10B3B0000A4342F0010104E024F00A020A4342F089
:10B3C00001010383018470BD70B505460C468E48AB
:10B3D000854209D08D48854206D0B5F1804F03D013
:10B3E0008B48854200D08B4820886188A2882389B9
:10B3F00058B1042811D0082817D02846FFF702FFBB
:10B40000E1882846BDE87040F0E62846FFF7ADFF2A
:10B41000E1882846BDE870409FE72846FFF76AFFAD
:10B42000E1882846BDE8704058E72846FFF725FF29
:10B43000E1882846BDE8704017E72DE9F04107464E
:10B440000C46002501266188002900D10225A2882A
:10B45000012A00D102262088238988B13846FFF7C7
:10B4600049FFE1883846FFF739FF238932462946EC
:10B470003846FFF77AFFE1883846BDE8F0416CE7CF
:10B480003846FFF772FFE1883846FFF766FF2389E9
:10B49000324629463846FFF72DFFE1883846BDE899
:10B4A000F0411BE710B50A884B88CC881A438B887B
:10B4B00023431A430B891A434B8989891A430A4348
:10B4C000A0F8442010BD4FF6FF718180002101805B
:10B4D000C1804180017270470021018041808180DC
:10B4E000C180018141818181C1817047002101803A
:10B4F000418001228280C18001817047002101804A
:10B5000041808180C1800181418181817047002912
:10B5100004D0018841F0010101807047018821F0C9
:10B52000010101807047002905D030F8441F41F423
:10B5300000410180704730F8441FC1F30E010180C3
:10B540007047002A03D082890A438281704782892A
:10B550008A4382817047818270471143A0F8481066
:10B560007047002A03D082890A438281704782890A
:10B570008A4382817047018921F007010181704768
:10B58000028922F070020A430281704700B5034627
:10B590001846FFF7F5FF188940F00700188100BD35
:10B5A00070B50D4604461146602D0CD00122204690
:10B5B000FFF7DBFE29462046FFF7E2FF208940F037
:10B5C0000700208170BD01222046FFF793FEF1E7BE
:10B5D00030B50489E4B24FF6FF7505EA032313433F
:10B5E0000B432343038130BD10B504462046FFF7CB
:10B5F000EFFF208920F0070040F0070020F07000E6
:10B6000040F07000208110BD002C0140003401404A
:10B610000004004000080040000C004010B5044643
:10B620002046FFF7D5FF208940F480402081EAE7DB
:10B63000018582827047028822F070020A430280EC
:10B64000704770B50589048B068C25F007050D43FE
:10B650004FF6FC410C4040F201110C4326F022064B
:10B660004FF6FF7101EA0311114331430581048351
:10B67000018470BD028B22F070020A43028370477E
:10B68000028B22F4E0424FF6FF7303EA01211143DB
:10B6900001837047828B22F070020A4382837047D5
:10B6A000828B22F4E0424FF6FF7303EA012111433B
:10B6B00081837047002904D0018841F08001018016
:10B6C0007047018821F0800101807047002904D073
:10B6D000818841F0040181807047818821F0040154
:10B6E00081807047002904D0818841F00801818061
:10B6F0007047818821F0080181807047002904D0BB
:10B70000818841F0010181807047818821F0010129
:10B7100081807047028B22F008020A43028370473F
:10B72000028B22F400624FF6FF7303EA01211143FA
:10B7300001837047828B22F008020A43828370479C
:10B74000828B22F400624FF6FF7303EA012111435A
:10B7500081837047028B22F004020A430283704700
:10B76000028B22F480624FF6FF7303EA012111433A
:10B7700001837047828B22F004020A438283704760
:10B78000828B22F480624FF6FF7303EA012111439A
:10B7900081837047028B22F080020A430283704744
:10B7A000028BC2F30E024FF6FF7303EA012111432D
:10B7B00001837047828B22F080020A4382837047A4
:10B7C000828BC2F30E024FF6FF7303EA012111438D
:10B7D00081837047028C22F002020A430284704780
:10B7E000028C22F008020A4302847047028C22F085
:10B7F00020024FF6FF7303EA0111114301847047E1
:10B80000028C22F080024FF6FF7303EA011111430C
:10B8100001847047028C22F400724FF6FF7303EA32
:10B820000121114301847047028C22F400624FF61B
:10B83000FF7303EA0121114301847047028C22F453
:10B8400000524FF6FF7303EA013111430184704740
:10B8500010B501238B40048C9C430484038C8A40E4
:10B8600013430384CFE610B504238B40048C9C4320
:10B870000484038C8A4013430384C4E630B500F18A
:10B88000180301248C40058CA5430584002911D0A0
:10B8900008290FD0091FC1F34E001844016821F494
:10B8A000E041016001684FF6FF7303EA0222114391
:10B8B000016030BD03EB5100016821F070010160AF
:10B8C00001681143016030BD002904D0018841F0B6
:10B8D000020101807047018821F002010180704758
:10B8E000002904D0018841F00401018070470188DB
:10B8F00021F0040101807047002904D0818841F0C3
:10B90000800181807047818821F0800181807047AB
:10B91000028822F00802028002880A4302807047EF
:10B92000828822F07002828082880A438280704777
:10B93000028922F00702028102890A4302817047CC
:10B94000028922F08002028102890A430281704743
:10B950008184704781857047818670470187704771
:10B9600081877047A0F840107047028822F4407227
:10B97000028002880A4302807047808E7047008FE1
:10B980007047808F7047B0F840007047808C7047D8
:10B99000008D704702460020128A0A4200D0012022
:10B9A0007047C9430182704702460020138A0B404A
:10B9B00092890A40002B02D0002A00D00120704753
:10B9C000C94301827047000010B5E14988420AD19D
:10B9D00001218C032046FEF7A2FF2046BDE810405F
:10B9E0000021FEF79CBFDB4988420AD101214C04AB
:10B9F0002046FEF79FFF2046BDE810400021FEF7DD
:10BA000099BFD54988420AD101218C042046FEF70E
:10BA100091FF2046BDE810400021FEF78BBFCF49C3
:10BA200088420AD10121CC042046FEF783FF20463C
:10BA3000BDE810400021FEF77DBFC94988420AD108
:10BA400001210C052046FEF775FF2046BDE8104099
:10BA50000021FEF76FBF10BD30B585B004460D461E
:10BA6000208A4CF6FF710840E98801432182A089B1
:10BA70004EF6F3110840A9882A8911436A890243C6
:10BA80001143A181A08A4FF6FF410840A9890143D3
:10BA9000A1826846FEF7D5FEAD48844201D10398E5
:10BAA00000E00298A189090408D500EBC00101EB70
:10BAB000001029684900B0FBF1F007E000EBC0017D
:10BAC00001EB001029688900B0FBF1F06422B0FBA3
:10BAD000F2F109010B096FF018056B4300EB8300CD
:10BAE000A3891D044FF0320307D503EBC000B0FB60
:10BAF000F2F000F00700084306E003EB0010B0FB93
:10BB0000F2F000F00F000843208105B030BD4FF483
:10BB10001651016000218180C18001810C22428187
:10BB20008181704710B5038A4FF2FF0213400A88E3
:10BB30004C8822438C88C9880C4322431A430282D2
:10BB400010BD0021018041808180C18070470029A3
:10BB500004D0818941F4005181817047818921F4A9
:10BB600000518181704710B540F66A13C1F342134A
:10BB700001F01F040121A140012B07D0022B07D0A7
:10BB800014303AB102680A43026010BD0C30F8E785
:10BB90001030F6E702688A43026010BD002A03D025
:10BBA000828A0A4382827047828A8A4382827047ED
:10BBB000028A22F00F020282028A0A43028270473E
:10BBC000828922F40062828182890A4382817047DD
:10BBD000002904D0818941F0020181817047818967
:10BBE00021F0020181817047028A22F02002028244
:10BBF000028A0A4302827047002904D0018A41F474
:10BC0000804101827047018A21F48041018270479E
:10BC1000C1F30801818070478088C0F30800704735
:10BC2000818941F0010181817047028BD2B2028388
:10BC3000028B42EA012101837047028B02F47F42AA
:10BC40000283028B0A4302837047002904D0818A51
:10BC500041F0200181827047818A21F02001818298
:10BC60007047002904D0818A41F010018182704719
:10BC7000818A21F0100181827047002904D0818AD5
:10BC800041F0080181827047818A21F00801818298
:10BC90007047002904D0818941F4004181817047B7
:10BCA0008189C1F30E0181817047002904D0818A06
:10BCB00041F4006181827047818A21F400618182B0
:10BCC0007047828A22F004028282828A0A43828238
:10BCD0007047002904D0818A41F0020181827047B7
:10BCE000818A21F002018182704702460020128879
:10BCF0000A4200D0012070478A05C943018070477D
:10BD000070B5002440F66A12C1F3421301F01F051A
:10BD1000012606FA05F2012B0CD0022B0DD0838AE6
:10BD20001340090A8E40008830400BB100B1012455
:10BD3000204670BD83891340F3E7038A1340F0E780
:10BD400040F66A120A0A01219140C94301807047F6
:10BD5000003801400044004000480040004C0040D2
:10BD60000050004010B50120FEF7EFFDBDE8104087
:10BD70000020FEF7EABD2049086070471E49091FF0
:10BD8000086070471C498431086070471B4A11885D
:10BD900021F46071014311807047184A118821F025
:10BDA0007F0101431180704708B5144A2C3A1044B2
:10BDB00000900098016008BD08B510492C3908446E
:10BDC00000900098008808BD0B489C300068C0B205
:10BDD00070470A480830018841F00101018070472E
:10BDE0000548A0300068C0B2704704480830018898
:10BDF00041F002010180704704860D422C6C004026
:10BE000010B501210C072046FEF794FD2046BDE841
:10BE100010400021FEF78EBD21490862704720497D
:10BE2000086170471F4A116821F0E0010143116069
:10BE300070471B49A031086070471A4B1A6822F0FE
:10BE4000030202431A601848026842F004020260CA
:10BE5000012905D020BF016821F00401016070476D
:10BE600030BFF8E70F48016841F004010160016844
:10BE700041F0020101600C48016841F004010160D9
:10BE800030BF704701460020064A52680A4200D07F
:10BE90000120704703490A6842EA80000860704741
:10BEA00000000E420070004010ED00E038B50121A6
:10BEB0004020FEF71EFD0F20ADF8000010208DF889
:10BEC000030003208DF802001A4C69462046FEF755
:10BED000ECFA0F212046FEF757FB38BD10B5164A85
:10BEE00084074FF000034FF0010105D502F5C2723F
:10BEF00013605160916010BD440705D502F5C27210
:10BF000011605360916010BD0007FCD502F5C2724C
:10BF100011605160936010BDC107074805D0D0F88B
:10BF20008011C943C0F8801170470121C0F8801109
:10BF300070470000001801400000234238B504207B
:10BF4000ADF8000048208DF803008D4C694620466E
:10BF5000FEF7ABFA04212046FEF716FB38BD08B504
:10BF60000420ADF8000010208DF8030003208DF8A8
:10BF7000020069468248FEF798FA08BD38B50820E5
:10BF8000ADF8000048208DF803007D4C694620463E
:10BF9000FEF78BFA08212046FEF7F6FA38BD08B501
:10BFA0000820ADF8000010208DF8030003208DF864
:10BFB000020069467248FEF778FA08BD38B50121DB
:10BFC0000420FEF796FC0C20ADF8000010208DF840
:10BFD000030003208DF80200694C69462046FEF7F5
:10BFE00064FA0C212046FEF7CFFA38BD70B5FFF792
:10BFF000B6FF644C012020606060634E3088800092
:10C0000007F0D4F9002525603088800007F0CEF9CC
:10C01000656070BD70B5FFF7A2FF5A4C00206060EC
:10C020002060594D2888800007F0C0F90120606029
:10C0300020602888BDE87040800007F0B7B92DE97E
:10C04000F0410024FFF77AFF504D0126C5F88861C2
:10C050004D4F388807F0AAF9C5F88C61388807F089
:10C06000A5F908E0641CE4B2FA2C04D9FFF7D2FF6A
:10C070000120BDE8F081D5F808010028F2D1C5F80B
:10C080008C01F6E770B53F4C00256560FFF767FF50
:10C0900025603D4E3088400007F088F9012060603F
:10C0A0003088400007F082F9656070BD2DE9F041ED
:10C0B000344C00276760FFF752FF01262660324D9F
:10C0C0002888400007F072F966602888400007F071
:10C0D0006DF96760CDE72DE9F0470546FFF73FFFB3
:10C0E0002A4E4FF00008C6F88C810024264F4FF0EE
:10C0F0000109E809C6F888016806050E388840007D
:10C1000007F054F9C6F88C913888400007F04EF9D2
:10C11000C6F88C813888400007F048F9641CE4B206
:10C12000082CE6D3BDE8F0872DE9F04782460024CD
:10C13000FFF704FF0025154E134FA0464FF00109ED
:10C14000C6F88C813888400007F030F9C6F88C9129
:10C150006006040ED6F8080108B1641CE4B2388801
:10C1600007F024F96D1CEDB2082DE9D3BAF1000FE8
:10C1700003D0FFF787FF2046D4E7FFF797FFFAE7E2
:10C1800000080140880121425C0300200000214298
:10C1900070B505466C4C02212046FEF7D2FD002802
:10C1A000F9D029462046FEF780FD01212046FEF702
:10C1B000C8FD0028F9D02046FEF779FDC0B270BD59
:10C1C00001466148028822F03802028002880A4350
:10C1D00002800121FEF739BD30B587B0012141F25F
:10C1E0000800FEF786FB01210846FEF7EFF9382428
:10C1F000ADF8184018208DF81B0003208DF81A00A8
:10C20000524D06A92846FEF750F9BDF818102846E9
:10C21000FEF7BAF90020ADF804004FF48271ADF8D2
:10C220000610ADF80800ADF80A00ADF80C0069156D
:10C23000ADF80E10ADF81040ADF812000720ADF8C3
:10C240001400414C01A92046FEF77AFC012120464A
:10C25000FEF7FBFCFF20FFF79BFF322007F0C6F83C
:10C260000820FFF7ADFFFF20FFF792FF07B030BDBA
:10C2700001463748028822F03802028002880A43C9
:10C2800002800121FEF7E1BC70B50546304C022169
:10C290002046FEF756FD0028F9D029462046FEF735
:10C2A00004FD01212046FEF74CFD0028F9D0204670
:10C2B000FEF7FDFCC0B270BD70B586B0012108204C
:10C2C000FEF717FB01218803FEF71EFB4FF46045C4
:10C2D000ADF8145018248DF8174003208DF816007F
:10C2E0001A4E05A93046FEF7E0F829463046FEF71B
:10C2F0004BF90020ADF800004FF48271ADF8021048
:10C30000ADF804000221ADF806100121ADF80810C7
:10C310004902ADF80A10ADF80C40ADF80E00072048
:10C32000ADF810000A4C69462046FEF709FC0121D1
:10C330002046FEF78AFCFF20FFF7A6FF3820FFF714
:10C3400097FF06B070BD000000300140000C0140B6
:10C350000038004070486F49416070494160704743
:10C360006D48016941F08001016170476A48C06809
:10C37000C10701D001207047410701D50220704755
:10C38000C00601D5032070470020704770B50446F1
:10C39000FFF7ECFF0546012D05D107F007F8641EF5
:10C3A000A4B2002CF4D104B9FF25284670BD70B5A5
:10C3B000054645F6FF763046FFF7E8FF002812D124
:10C3C000554C206940F0020020616561206940F011
:10C3D000400020613046FFF7D9FF012803D02169D2
:10C3E00021F00201216170BD70B506460D46FF20A7
:10C3F000FFF7CCFF00280ED1474C206940F0010028
:10C4000020613580FF20FFF7C1FF012803D021699B
:10C4100021F00101216170BD00887047C10703D080
:10C4200030F8010C000A70470088C0B270472DE94F
:10C43000F04105460E461746002407E036F8141072
:10C440002846FFF7D1FFAD1C641CA4B2BC42F5D353
:10C45000BDE8F08110B50446002307E02046FFF751
:10C46000DBFF21F81300A41C5B1C9BB29342F5D3A5
:10C4700010BD30B504460D46002306E02046FFF708
:10C48000CDFFE854641C5B1C9BB29342F6D330BDD5
:10C4900070472DE9F047ADF5006D0D46904600243C
:10C4A0000746A0F10060B0F5002F23D200264FF41C
:10C4B0008069EA4615E06878000215F8021B084416
:10C4C0002146641CA4B22AF811004A46944206D1BF
:10C4D000002469463846FFF7AAFF07F50067B61C37
:10C4E000B6B24645E7D3002C04D02246694638460A
:10C4F000FFF79DFF0DF5006DBDE8F08710B54168B1
:10C50000074C21600068FBF71DFE2068BDE8104065
:10C51000004700002301674500200240AB89EFCDB2
:10C5200048000020FFF74ABD70B504460025604E64
:10C53000691E306806F089FC012824D1FFF76AFDE6
:10C540000A2006F033FFFFF751FD200AA02101EB7E
:10C550004000C0B2FFF7BFFDFFF771FDE0B2FFF78B
:10C56000BAFDFFF76CFDFFF741FDA120FFF7B3FD1A
:10C57000FFF765FD0020FFF7D7FD0546FFF74AFDF1
:10C58000306806F0AAFB284670BD70B504460E461A
:10C59000474D4FF0FF31286806F057FC012823D1A2
:10C5A000FFF738FD012006F021FFFFF71FFD200AED
:10C5B000A02101EB4000C0B2FFF78DFDFFF73FFD6A
:10C5C000E0B2FFF788FDFFF73AFD3046FFF783FD45
:10C5D000FFF735FDFFF71EFD052006F007FF286871
:10C5E000BDE8704006F079BB70BD2DE9F04106460C
:10C5F0000D461746002409E0E00025FA00F0C1B21C
:10C60000301980B2FFF7C1FF641CE4B2BC42F3D31F
:10C61000BDE8F0812DE9F04102460E4600200024DD
:10C62000971908E00502381B401E80B2FFF77CFF17
:10C630002844641CE4B2B442F4D3E9E710B5FF2007
:10C64000FFF772FF55280AD05521FF20FFF79DFF05
:10C65000FF20FFF769FF552803D0012010BD0020FF
:10C6600010BD002010BD70B504460E46154608E00A
:10C670002046641CA4B2FFF757FF06F8010B6D1E9D
:10C68000ADB2002DF4D170BD70B506460D4614460E
:10C6900006E029783046FFF778FF761CB6B26D1CAD
:10C6A000641EA4B2F5D270BD6FE76EE73CE73BE7CE
:10C6B0008404002010B5784C01212046FFF76AF968
:10C6C0002046BDE810400121FFF76BB97FB5044655
:10C6D0000D4601210220FEF717F9ADF80840ADF82C
:10C6E00004500020ADF80A00ADF806006A4C01A91C
:10C6F0002046FEF73BFC1D218DF8001001218DF82E
:10C70000011002228DF802208DF803106846FDF713
:10C7100054FB012211462046FEF713FF012120465B
:10C72000FEF7F5FE7FBD70B5FBF748FD5B4C0121C0
:10C730002046FFF72FF95A4A012802D15068401CC1
:10C74000506058490B8841F288350020AB4203D233
:10C750000B885B1C0B8000E008801178491CC9B273
:10C7600011700A2900D1107001212046FFF719F934
:10C77000BDE87040FBF729BD7FB504460D46012199
:10C780001020FEF7C1F8ADF80840ADF804500020C5
:10C79000ADF80A00ADF80600404C01A92046FEF7AE
:10C7A000E5FB36218DF8001001218DF801100322E0
:10C7B0008DF802208DF803106846FDF7FEFA01227D
:10C7C00011462046FEF7BDFE01212046FEF79FFEE2
:10C7D0007FBD10B588B001210420FEF795F8012136
:10C7E0002120FEF786F801210C032046FDF7EEFE1E
:10C7F0004FF4E041ADF81C1018218DF81F100321F3
:10C800008DF81E1007A92848FDF74FFEADF814401B
:10C810000020ADF81000ADF81600ADF81200234C62
:10C8200004A92046FEF7A2FB7021ADF800100121FB
:10C83000ADF802100221ADF8081069462046FEF757
:10C84000CEFB69462046FEF703FC69462046FEF70C
:10C850003FFC08212046FEF75DFF08212046FEF739
:10C860005FFF08212046FEF765FF01212046FEF705
:10C870004EFE08B010BD0D4A002806D0012807D092
:10C88000022808D11046FFF76BB81046FFF764B8CE
:10C890001046FFF763B870470004004000100040E6
:10C8A0004C000020800600200014014000080040D9
:10C8B00038B501210820FEF71CF8C020ADF80000B3
:10C8C00010208DF8030003248DF80240FE4D6946C8
:10C8D0002846FDF7EAFDA915ADF8001048218DF8AE
:10C8E00003108DF8024069462846FDF7DEFD40F250
:10C8F000CF216420FFF740FF80212846FDF746FE48
:10C900000A2006F073FD80212846FDF73DFE0A202F
:10C9100006F06CFD80212846FDF738FE0A2006F05F
:10C9200065FD80212846FDF72FFE0A2006F05EFDFA
:10C9300080212846FDF72AFE0A2006F057FD8021B7
:10C940002846FDF721FE0A2006F050FD80212846EA
:10C95000FDF71CFE0A2006F049FD80212846FDF760
:10C9600013FE0A2006F042FD38BD70B504460D46A0
:10C97000D54E40213046FDF709FE05F01F0020434B
:10C98000FFF706FCFF20FFF703FC0446280603D54B
:10C99000FF20FFF7FDFB044640213046FDF7F4FD84
:10C9A000204670BD2DE9F04104460D461746C64E9F
:10C9B00040213046FDF7EAFD05F01F002043FFF758
:10C9C000E7FB3846FFF7E4FB3046BDE8F041402185
:10C9D000FDF7DABD70B505460C46BB4E402130462A
:10C9E000FDF7D4FD3A20FFF7D3FB05E06D1E0020D4
:10C9F000FFF7CEFB04F8010B002DF7D100202070CB
:10CA00003046BDE870404021FDF7BEBD70B504461C
:10CA10000D46AD4E40213046FDF7B8FD7A20FFF7B8
:10CA2000B7FB04E0641E2878FFF7B2FB6D1C002CF6
:10CA3000F8D13046BDE870404021FDF7A5BD70B586
:10CA40000546A24E05F06004307884420BD00322E4
:10CA50001F21A020FFF7A6FFC5F341121F21802050
:10CA6000FFF7A0FF347070BD10B504462046FFF7F5
:10CA7000E6FF2146BDE81040002076E770B5054688
:10CA80000C462846FFF7DBFF22462946BDE87040EA
:10CA9000402087E770B50D4600240146D420FFF7FB
:10CAA000EDFFE9B2D620FFF7E9FFC5F30721D72054
:10CAB000FFF7E4FF40F6FF7501E0641CA4B2EA2032
:10CAC000FFF7D2FFC00701D0AC42F6D370BD70B5FE
:10CAD00005460024FFF7ECFE4FF4FA7609E0FF224A
:10CAE00000211046FFF75EFF641CA4B20A2006F086
:10CAF0007DFC1D20FFF7B8FFC00701D1B442EED383
:10CB0000B44201D3012070BD70490020486000216B
:10CB10000820FFF7B3FF00210920FFF7AFFF002136
:10CB20000C20FFF7ABFF00210D20FFF7A7FF10211E
:10CB30000A20FFF7A3FF1A210B20FFF79FFF112107
:10CB40000420FFF79BFF1A210520FFF797FFFF2125
:10CB50000620FFF793FF1F210720FFF78FFFA1217A
:10CB60003820FFF78BFF3F212820FFF787FF302178
:10CB70002920FFF783FFF9213020FFF77FFFF721FE
:10CB80003120FFF77BFF0D21C020FFF777FF002149
:10CB9000C120FFF773FF3322C2218020FFF702FF7D
:10CBA0001221C620FFF76AFF0C21C720FFF766FF9E
:10CBB0001521C420FFF762FFEE21CA20FFF75EFFB8
:10CBC0000521CB20FFF75AFF2978E420FFF756FF15
:10CBD0006978E520FFF752FFA978E220FFF74EFFC2
:10CBE000E978E320FFF74AFF2979E020FFF746FFC5
:10CBF0006979E120FFF742FF4FF48074214600205D
:10CC0000FFF748FF21461020FFF744FF1F20FFF7E2
:10CC100016FFC0221B218020FFF7C4FE04221F2123
:10CC20008020FFF7BFFEE420FFF71EFF297888422F
:10CC300001D1002070BD012070BD722014E770B5D5
:10CC400005460E4611210220FFF718FF1A21032086
:10CC5000FFF714FF41F611202C18E1B20620FFF770
:10CC60000DFFC4F307210720FFF708FF002211463C
:10CC70007A20FFF797FE31462846FFF7C7FE0822C5
:10CC80001F218020FFF78EFE1C20FFF7EDFE80079E
:10CC900005D5BDE8704008221F21A02082E670BDA6
:10CCA0002DE9F04106460F463920FFF7DDFED8B3E7
:10CCB000064D00202979FFF7E1FEA888C0F307217F
:10CCC0000120FFF7DBFE03E0000C014054000020D0
:10CCD00000213A20FFF749FE686000213A20FFF763
:10CCE00044FE696841EA0020686000213A20FFF7AD
:10CCF0003CFE044600213A20FFF737FE44EA0024B8
:10CD0000241F00213A20FFF730FE804600213A2000
:10CD1000FFF72BFE48EA0020711E8C4200D9741EDA
:10CD2000000605D4002407E0FFE70020BDE8F081FD
:10CD300039462046FFF74EFE29790C20FFF79EFE6C
:10CD4000A888C0F307210D20FFF798FE40221E217E
:10CD50008020FFF727FE2046E8E7000030B5F749BE
:10CD6000C979002919D1F64A0024C2F8AC4101233F
:10CD7000C2F8B431050602D5C2F8BC3101E0C2F8F0
:10CD8000BC41C2F8B841C2F8B8314006000E491C97
:10CD9000C9B20829EED3C2F8AC3130BD30B5E7498D
:10CDA000C979002919D1E64A0023C2F8AC31C2F88A
:10CDB000B4310124050602D5C2F8BC4101E0C2F835
:10CDC000BC31C2F8B831C2F8B8414006000E491C67
:10CDD000C9B20829EED3C2F8AC4130BDD749C979F0
:10CDE000002902D13830C0B2D8E7704710B50446E8
:10CDF000D249C979002907D10020FFF7EFFF40345D
:10CE0000E0B2BDE81040C9E710BD10B50446CB48FC
:10CE1000C07900280DD1FFF7E1FF04F00F002409CD
:10CE2000E030C0B2FFF7BAFFF034E0B2BDE8104026
:10CE3000B4E710BD2DE9FC41074694461E46ACF10F
:10CE40002002D5B2BD48C079002817D0C7EB071023
:10CE50000A2202EB4004A1EB011000F5987082B2A7
:10CE6000F6B347F610604FF6FF71CDE90010634648
:10CE70002146022003F071FBBDE8FC8101EB41017A
:10CE8000032000EB410808F0FF00FFF7BEFF780623
:10CE9000000EFFF7ABFF0024AA4905EB450001EBAC
:10CEA00080050EB3285DC043C0B2FFF757FF641C76
:10CEB000E4B2062CF5D308F0FF00FFF7A6FF01202F
:10CEC00000EB4700C0B2FFF791FF002486B128199C
:10CED0008079C043C0B2FFF741FF641CE4B200E0B8
:10CEE0000BE0062CF2D3C7E7285DFFF737FFDEE73C
:10CEF00028198079FFF732FFEFE747F61960B2E7AC
:10CF000070B506468D48C079002805D0BDE8704050
:10CF100047F6196003F0BCB9002442F6A00530467C
:10CF2000FFF71CFF641CA4B2AC42F8D370BD2DE91E
:10CF3000FC4781460E4690461F460024384624F0A2
:10CF4000DDFBC5B27D48C6F11501C079C0B1C9EBA2
:10CF500009100A2101EB4001A6EB061000F59870BC
:10CF600082B2B8F1000F1BD047F610604FF6FF7386
:10CF7000CDE900303B46022003F05CFBBDE8FC87B6
:10CF8000A9420ADACDB208E03019C1B23A5D43468F
:10CF90004846FFF74FFF641CE4B2AC42F4D3EDE720
:10CFA00047F61960E2E7002267A31146BFE7F0B534
:10CFB000002442F2107564230A264FF47A77A842BF
:10CFC00021D3B0FBF5F430340C70B0FBF5F405FB65
:10CFD0001400B0FBF7F430344C70B0FBF7F407FBEF
:10CFE0001400B0FBF3F430348C70B0FBF3F403FBAB
:10CFF0001400B0FBF6F330330424CB70B0FBF6F32F
:10D0000006FB13003AE0B84219D3B0FBF7F4303412
:10D010000C70B0FBF7F407FB1400B0FBF3F43034F2
:10D020004C70B0FBF3F403FB1400B0FBF6F33033A9
:10D0300003248B70B0FBF6F306FB13001EE064289C
:10D0400011D3B0FBF3F430340C70B0FBF3F403FBFA
:10D050001400B0FBF6F3303302244B70B0FBF6F350
:10D0600006FB13000AE00A2808D3B0FBF6F33033BE
:10D0700001240B70B0FBF6F306FB13003030631C89
:10D08000DBB208550020C854002A1DD09A420DD3A7
:10D090005B1CDBB206E01C1A651815F8015C0D5527
:10D0A000401CC0B29842F6D3302008700020551CB6
:10D0B00005E01C1A0E5D0C446670401CC0B2A8420C
:10D0C000F7D32E209A1A8854F0BD2DE9FC47144658
:10D0D000DDE90AA980460E461A4620B21749C979E9
:10D0E000002902D1052A01D9002047E7B8F1050F30
:10D0F00001D8152E01D9002040E70025002802DACA
:10D100000125404284B269462046FFF750FF684639
:10D1100024F0F4FAC4B26F46BAF1000F03D0BAF1AA
:10D12000010F35D05DE03DB14B462D2231464046E2
:10D13000FFF780FE012528E000251AE05C000020B2
:10D1400000002342C8430308202020202020202064
:10D15000202020202020202020202020200000002F
:10D160007019C1B27A5D4B464046FFF763FE6D1CF5
:10D17000EDB2A542F4D334E07019C1B27A5D4B46EA
:10D180004046FFF757FE6D1CEDB2A542F4D328E0F0
:10D190000DB100251CE000250BE0601B38444B4618
:10D1A00010F8012C701BC1B24046FFF743FE6D1C06
:10D1B000EDB2A542F1D314E0601B38444B4610F8A1
:10D1C000012C701BC1B24046FFF734FE6D1CEDB25E
:10D1D000A542F1D3701BC1B24B462D224046FFF74A
:10D1E00029FE2046CAE610B5FB4A107901280CD169
:10D1F0001146A2F1100408782379497833B1D27826
:10D200000123FFF717FE0020207110BD9278012343
:10D21000FFF710FE0120207110BD10B5EE4C2070FC
:10D220006170A270E3700120207110BDEA490020F6
:10D2300008717047E8481038C179002901D10121EF
:10D2400081707047E4481038C179002900D181709D
:10D2500070473EB5E048E14C1038C07900280FD047
:10D2600063782278DEA1E24825F0DAFCA07900900C
:10D270006379B4F80320DFA1E24825F0D1FC3EBD7C
:10D2800060782178A279CDE9002102906379B4F821
:10D290000320D148DCA1401D25F0C2FC3EBD2DE994
:10D2A000F047CD4C103CE07900287DD16070DFF86C
:10D2B0007483DD4FDD4D98F80000DD4ED22814D088
:10D2C000D32812D0D92810D034286DD1307DC00792
:10D2D0006BD0D8A1DB4824F047FAF07B00287DD042
:10D2E000D9A1D84824F0E0F9D3E0BB48401D24F090
:10D2F00005FA00F0FF096078B74928444A46491DFD
:10D3000024F0AEF9607848446070C748553824F07E
:10D31000F5F900F0FF096078C34928444A465539B9
:10D3200024F09EF9607848446070BF484A3824F081
:10D33000E5F900F0FF096078BB4928444A464A39BC
:10D3400024F08EF9607848446070207870B1BF484E
:10D3500024F0D4F900F0FF0960784A462844BB491C
:10D3600024F07EF96078484460700FE0B7480830D8
:10D3700024F0C4F900F0FF096078B44928444A4613
:10D38000083124F06DF9607848446070A6483F3851
:10D3900024F0B4F900F0FF096078A34928444A4614
:10D3A0003F3924F05DF901E06DE085E060784844A4
:10D3B000C0B2607098F80010342914D008229A493D
:10D3C0002844363924F04CF9607808306070A04861
:10D3D000007830F080001FD09E4800E055E00078D3
:10D3E000012829D041E008228F4928442D3924F012
:10D3F00037F96078083060707089C0EB00103844ED
:10D4000024F07CF9C2B27089C0EB0010C1196078B9
:10D41000284424F025F92DE08348243824F06EF9BF
:10D42000C6B26078804928443246243924F018F97D
:10D430006078304460701DE087487B49874A807B74
:10D44000243900EBC000431885A17E4825F0E8FB95
:10D450007C4824F053F9C6B26078324628447949B2
:10D4600024F0FEF860783044607060782021284411
:10D4700000F8011C032260787BA1284424F0F0F816
:10D480006078C01C6070BDE8F08778A16D4824F01A
:10D490000BF9AFF238316B4824F006F9694824F0F3
:10D4A0002DF900F0FF08607842462844654924F0D1
:10D4B000D7F8607840446070307D4008C00730D0B5
:10D4C0006CA1604824F050F9DFF8AC8100226B4970
:10D4D00098F80000FFF76BFD68495A4824F0E4F81B
:10D4E00067A1584824F0E0F898F801000022634949
:10D4F000FFF75DFD6149534824F0D6F8AFF2A4313F
:10D50000504824F0D1F84F4824F0F8F800F0FF0814
:10D510006078424628444B4924F0A2F860784044A1
:10D520006070307D8008C0071FD057A1454824F0A7
:10D530001BF958485849007BC0EBC00001444148E2
:10D5400024F0B2F8AFF2EC313E4824F0ADF83D489B
:10D5500024F0D4F800F0FF086078424628443949A6
:10D5600024F07EF8607840446070307DC008C007C9
:10D570001CD04AA1334824F0F7F8307BC0EB0010F0
:10D58000C119304824F090F8AFF230412D4824F012
:10D590008BF82C4824F0B2F8C7B260783A46284499
:10D5A000284924F05DF8607838446070307D0028A8
:10D5B0007FF469AF3CA1234824F0D6F8214824F039
:10D5C0009DF8C6B26078324628441E4924F048F8D7
:10D5D00060783044607056E76C00002086000020C0
:10D5E00054696D6520253032643A2530326400007C
:10D5F000B0000020253034642D253032642D2530D4
:10D6000032640000BB000020253034642D25303208
:10D61000642D2530326420253032643A253032645E
:10D6200000000000040000208D4E03083409002093
:10D63000AE8E002053656E736F7253746174757390
:10D640003A000000288D00204F4B0000B84303082B
:10D65000F6020020F5020020348C0020408E0408E1
:10D6600025733A25732C0000202020004F66666C3D
:10D67000696E650052583A00D4020020708D002077
:10D680002054583A0000000042617564726174656C
:10D690003A000000087B0020D9900408204151493D
:10D6A000204C4556454C3A002020202020202000C8
:10D6B0002DE9F0478146DDE908088A4615461F46F0
:10D6C0002038C6B2B248C079002836D1BAF1820FEC
:10D6D00033D25046FFF799FB4FEA4960000EFFF73F
:10D6E00085FB2C46AB4800EB061609E0B8F1000FAD
:10D6F00012D0305DC043C0B2FFF730FB641CE4B20F
:10D70000BC42F3D35046FFF780FB012000EB4900F9
:10D71000C0B2FFF76BFB0EE0305DFFF71FFBEDE7DC
:10D72000B8F1000F0AD07019007AC043C0B2FFF7F9
:10D7300015FB6D1CEDB2BD42F2D3A4E67019007A60
:10D74000FFF70CFBF5E72DE9FC41914EF07900283D
:10D750007ED1B07800287BD0B079DFF83C82411CC4
:10D76000C9B218F800207078B1FBF0F300FB131475
:10D770000027CDE900270823727939460420FFF7F6
:10D7800097FF707907282CD20125601C18F8042017
:10D79000C0B27178B0FBF1F301FB1304CDE90027AF
:10D7A00070790823C0EBC500C1B200220420FFF746
:10D7B0007FFF6D1CEDB2102DE7D3601C18F804102C
:10D7C000C0B27278B0FBF2F0CDE900177079002298
:10D7D000011DCBB2C0EBC500C1B20420FFF768FF4A
:10D7E0002BE00125601C18F80420C0B27178B0FB52
:10D7F000F1F301FB1304CDE9002770790823C0EB96
:10D80000C500C1B200220420FFF752FF6D1CEDB22B
:10D81000112DE7D3601C18F80410C0B27278B0FB69
:10D82000F2F0CDE9001770790022811ECBB2C0EB77
:10D83000C500C1B20420FFF73BFF7079401CC0B2A5
:10D84000707108280BD37771B079401CC0B200E02A
:10D8500005E07178B0FBF1F201FB1200B071BDE898
:10D86000FC8110B54D49002808D00122C1F8A8213B
:10D87000474CE07004F0BDFFA06010BD0022C1F86D
:10D88000A821F5E770B5424C0025E07800280FD0BC
:10D89000FF280DD004F0ADFFE060A168411AE078E8
:10D8A00000EB4002C2EBC010B1EBC00F00D3E5703B
:10D8B000E0783A4908B9C1F8A851FF2802D10120FF
:10D8C000C1F8A80170BD38B501214020FDF711F85D
:10D8D0004FF47C44ADF8004010208DF80300032085
:10D8E0008DF802002E4D69462846FCF7DEFD2146E4
:10D8F0002846FCF749FE38BD10B5FFF7E4FF294C78
:10D9000000202060322005F071FD012020600A20F7
:10D9100005F06CFD0120FFF761FA0A2005F046FDD5
:10D920001120FFF73BFA0A2005F040FDAE20FFF77B
:10D9300035FA0A2005F03AFD0820FFF72FFA0A20F1
:10D9400005F034FD0020FFF749FA0A2005F02EFD0E
:10D950000520FFF723FA0C20FFF720FA0020FFF73D
:10D9600054FA0020FFF742FA0A2005F01FFDBDE837
:10D9700010400020FFF7C4BA05490A20087070471C
:10D9800003490878002801D0401E08707047000045
:10D990005C000020484803083409002000002342AE
:10D9A00000180140B001234208B503208DF80000A3
:10D9B00004208DF801008DF8020001208DF803008D
:10D9C0006846FCF7FAF908BD810701D000207047CE
:10D9D0006421B0FBF1F201FB120109B10120704793
:10D9E0004FF4C871B0FBF1F201FB120008B1002046
:10D9F00070470120704730B56423B0FBF3F4E4B204
:10DA0000B0FBF3F503FB1500132C01D96430C0B251
:10DA100000EB90030724B3FBF4F504FB1533DE4D54
:10DA20001A440D4415F8015C2A4492B2800703D1D0
:10DA3000032901D2521E92B2B2FBF4F004FB102073
:10DA400030BD2DE9F05F0746DDE90A9A0D4616461E
:10DA500098460024A7F2B270822802D30120BDE8C4
:10DA6000F09FA5F1010BBBF10C0F01D30120F6E7EC
:10DA7000C9480C30284410F8010CB04200D20646C8
:10DA80000846FFF7A1FF20B1012D02D01D2E00D9BD
:10DA90001D2626B1B8F1180F03D30120DFE70120BE
:10DAA000DDE7B9F13C0F01D30120D8E7BAF13C0F13
:10DAB00001D30120D3E740F2B2750AE02846FFF710
:10DAC00083FF10B1B548044401E0B54804446D1C1F
:10DAD000ADB2BD42F2D30BF0FF0B002511E0AE4812
:10DAE00040F2A3210C30405D484304EBC01438469B
:10DAF000FFF76AFF18B1012D01D1AA4804446D1C3B
:10DB0000ADB25D45EBD3761E40F2A320464304EB55
:10DB1000C610C8EB4811C1EB082100EB0110C9EB9E
:10DB2000091100EB810000EB0A0401214FF0C05005
:10DB3000FCF7EAFE0120FEF76FF9FCF785FF2046AF
:10DB4000FCF750FFFCF780FF002088E72DE9F04745
:10DB5000FCF73FFF0746DFF84C82B7FBF8F492482A
:10DB6000061D4188A14235D0448040F2B2754FF481
:10DB7000B7794FF4B67A0FE02846FFF725FF38B1A2
:10DB80004C4502D3A4F5B77404E06D1CADB205E0BA
:10DB9000A4F26D146D1CADB25445EDD8A6F8035037
:10DBA0000025DFF8F49109F10C090DE0B6F8030047
:10DBB000FFF70AFF08B1012D30D019F80500A04287
:10DBC00004D8241A6D1CADB21C2CEFD26D1C7571DB
:10DBD000641CB471B7FBF8F008FB10704FF461617E
:10DBE000B0FBF1F23270B0FBF1F201FB12033C2208
:10DBF000B3FBF2F37370B0FBF1F301FB1300B0FB66
:10DC0000F2F102FB1100B070B2797179B6F803003D
:10DC1000FFF7F1FEF0710020BDE8F0871D2CD5D391
:10DC20001D3CCFE770B5002401214FF0C050FCF738
:10DC30006BFE0120FEF7F0F8FEF794F80120FCF7E8
:10DC4000E2FD5AA013F0A9FA4FF4967508E0641C9F
:10DC5000A4B20A2005F0CAFBAC4201D3012070BD7A
:10DC60004120FCF755FD0028F1D057A013F095FA9C
:10DC70004FF48070FCF7DCFD0120FCF7DEFDFCF7C3
:10DC8000F7FEFCF7E1FE01210846FCF789FEFCF7F0
:10DC9000DBFE47F6FF70FCF7B2FEFCF7D5FE002076
:10DCA00070BD1CB54C4801783F48001D00290BD0C1
:10DCB00081784278CDE90021037882794179B0F802
:10DCC0000300FFF7BEFE1CBD44490978D22905D0E8
:10DCD000D32903D0D92901D001201CBD81784278F5
:10DCE000CDE90021037882794179B0F80300FFF78C
:10DCF000A8FE1CBD10B5FFF757FE0420FEF75CF828
:10DD00004AF2A554A04212D035A013F046FAFFF70C
:10DD100089FF012809D03AA013F03FFAFFF7C1FFAD
:10DD200021460420FEF740F813E0012010BD3AA080
:10DD300013F033FAFCF79CFE012808D001210846B5
:10DD4000FCF72EFEFCF780FE18B1012010BD01206B
:10DD500010BDFCF704FE002010BD10B50120FCF73B
:10DD6000ABFE30B1FFF7F2FE0F48017889B1002118
:10DD700001700220FCF7A0FE10B10220FCF7AAFE01
:10DD80000520FCF7A7FEFCF75FFEBDE81040FFF79B
:10DD900060BA01210170ECE7E74E03080085E2015B
:10DDA0008033E10180510100820000200D0A2057DC
:10DDB0006169742074696C6C204C53452069732030
:10DDC00072656164790000000D0A204C534520699A
:10DDD00073207265616479006300002004000020F4
:10DDE0000D0A0A20525443206E6F74207965742006
:10DDF000636F6E666967757265642E2E2E2E000045
:10DE00000D0A2052544320636F6E66696775726510
:10DE1000642E2E2E2E0000000D0A204E6F206E65FF
:10DE2000656420746F20636F6E6669677572652024
:10DE30005254432E2E2E2E0038B501210420FCF71B
:10DE400058FD01214348FCF7C1FB4FF47044ADF885
:10DE5000004048208DF8030003208DF802003E4D5D
:10DE600069462846FCF721FB21462846FCF78CFB37
:10DE700038BD2DE9F0410024374F3846FCF777FBD9
:10DE80004FF4704626EA0005142005F0AFFA384634
:10DE9000FCF76DFB86433540E80400D5BC14A804AC
:10DEA00001D544F40054680401D544F480442804A6
:10DEB00001D544F40044200BBDE8F08108B5FFF71C
:10DEC000BBFF26A013F069F9642005F08FFA264DF8
:10DED000264C2878D22807D0D42805D0D62803D0BD
:10DEE000342801D0FAF74BFDFFF7C3FF009061889B
:10DEF00088420BD000231A466946606804F068FE29
:10DF0000BDF800006080002020701FE0F0B1217893
:10DF1000462903D340F4407000900AE0322903D32D
:10DF200040F40070009004E01E2902D340F4807099
:10DF300000900A2905D300231A466946606804F058
:10DF400047FE2078462801D2401C2070642004F04F
:10DF5000C5FABEE700043000000801404B65792097
:10DF60005461736B0D0A0000040000209000002033
:10DF700070B5FDF7F4FFFB4C002525601E2005F071
:10DF800015FA65601E2005F011FA0120206060601E
:10DF90001E2005F00BFA25601E2005F007FA6560CB
:10DFA00070BD10B5FDF7DBFF1E2005F0FFF9ED4C4D
:10DFB0000020606020601E2005F0F8F901206060FC
:10DFC000206010BD2DE9F04104460825FDF7C7FF8C
:10DFD000E54E4FF000080127200602D5C6F88871EB
:10DFE00001E0C6F888816006040E1E2005F0DEF907
:10DFF000C6F88C711E2005F0D9F9C6F88C816D1E0B
:10E0000015F0FF05E8D1BDE8F0812DE9F0470024C7
:10E01000FDF794FF0025D44E01274FF6FF78A14667
:10E020001E2005F0C3F9C6F88C711E2005F0BEF95C
:10E03000D6F8080118B107EB440084B201E008EA01
:10E040004404C6F88C916D1CEDB2102DE8D3204627
:10E05000BDE8F0872DE9F0410024FDF76FFF0025B2
:10E06000C14E0127A0461E2005F0A0F9C6F88C710C
:10E070001E2005F09BF9D6F8080118B107EB440003
:10E08000C4B201E06006040EC6F88C816D1CEDB2CE
:10E09000082DE8D32046B6E770B50024FDF74EFF03
:10E0A0000A2005F083F9B04D0026D5F80801C0B26A
:10E0B00050B1022005F07AF9641CE4B20A2CF4D3C2
:10E0C000C5F88C61012070BD0120C5F88C0132209B
:10E0D00005F06CF9C5F88C61002070BD70B50024A6
:10E0E000FDF72CFFA04D06E0641CE4B2642C19D0AF
:10E0F000012005F05BF9D5F808010028F4D0FDF700
:10E100002EFF1E2005F052F905F5C47500242C6081
:10E110001E2005F04BF901266E601E2005F046F921
:10E120006C602E6070BD70B5FDF719FFFDF737FF0D
:10E130008C4C00256560012626601E2005F036F90E
:10E1400066601E2005F032F9256070BD10B5FFF73E
:10E150000FFF5220FFF736FF1E2005F027F9FFF7CB
:10E160009BFF08B1FFF71DFF642005F01FF9802019
:10E17000FFF728FF1E2005F019F9FFF78DFF08B102
:10E18000FFF70FFF642005F011F90320FFF71AFFD6
:10E190001E2005F00BF9FFF77FFF08B1FFF701FF25
:10E1A000BDE81040FDE610B5FFF7E2FE5220FFF794
:10E1B00009FF1E2005F0FAF8FFF76EFF18B1FFF710
:10E1C000F0FE002010BD642005F0F0F88120FFF77C
:10E1D000F9FE1E2005F0EAF8FFF75EFF18B1FFF721
:10E1E000E0FE002010BDFFF7DCFE642005F0DEF845
:10E1F000FFF7BEFE5320FFF7E5FEFFF74DFF18B116
:10E20000FFF7CFFE002010BDFFF724FF0446FFF705
:10E210008AFF1E2005F0CAF8FFF7C3FE204610BD96
:10E2200010B5FFF7A5FE5220FFF7CCFE1E2005F02B
:10E23000BDF8FFF731FF18B1FFF7B3FE002010BDA6
:10E24000642005F0B3F88720FFF7BCFE1E2005F020
:10E25000ADF8FFF721FF18B1FFF7A3FE002010BDB6
:10E26000FFF79FFE642005F0A1F8FFF781FE532021
:10E27000FFF7A8FEFFF710FF18B1FFF792FE00208E
:10E2800010BDFFF7E7FE0446FFF74DFF1E2005F027
:10E290008DF8FFF786FE3CB1012C07D0022C07D089
:10E2A000032C07D0012010BD012010BD022010BD9D
:10E2B000402010BD802010BD70B5FFF759FE5220E0
:10E2C000FFF780FE1E2005F071F8FFF7E5FE18B19C
:10E2D000FFF767FE002070BD642005F067F894200A
:10E2E000FFF770FE1E2005F061F8FFF7D5FE18B1AC
:10E2F000FFF757FE002070BDFFF753FE642005F0C6
:10E3000055F8FFF735FE5320FFF75CFEFFF7C4FE1C
:10E3100018B1FFF746FE002070BDFFF79BFE0446D4
:10E32000FFF7DCFE1E2005F041F8FFF793FE0546DF
:10E33000FFF7F9FE1E2005F039F8FFF732FE44EA38
:10E34000052070BD70B5FFF713FE5220FFF73AFEAF
:10E350001E2005F02BF8FFF79FFE38B1FFF721FED6
:10E36000002070BD8801214200002142642005F098
:10E370001DF89620FFF726FE1E2005F017F8FFF780
:10E380008BFE18B1FFF70DFE0020EAE7FFF709FE4C
:10E39000642005F00BF8FFF7EBFD5320FFF712FEAA
:10E3A000FFF77AFE18B1FFF7FCFD0020D9E7FFF771
:10E3B00051FE0446FFF792FE1E2004F0F7FFFFF720
:10E3C00049FE0546FFF7AFFE1E2004F0EFFFFFF702
:10E3D000E8FD44EA0520C4E770B5F84D00206871F7
:10E3E000FFF7C6FD5220FFF7EDFD1E2004F0DEFF13
:10E3F000FFF752FE18B1FFF7D4FD0020B1E764200B
:10E4000004F0D4FF9220FFF7DDFD1E2004F0CEFFC4
:10E41000FFF742FE18B1FFF7C4FD0020A1E7FFF7A8
:10E42000C0FD642004F0C2FFFFF7A2FD5320FFF7F8
:10E43000C9FDFFF731FE18B1FFF7B3FD002090E7EB
:10E44000FFF708FE0446FFF76EFE1E2004F0AEFF45
:10E45000FFF7A7FDDA48048314F0700F02D0012003
:10E4600068717EE700207CE770B5D44C00202070F6
:10E47000FFF77EFDC220FFF7A5FD1E2004F096FFEA
:10E48000FFF70AFE40B1FFF78CFD2078012801D08C
:10E49000002066E7012064E71E2004F087FFFFF7F5
:10E4A000B4FD0646FFF71AFE1E2004F07FFFFFF7BB
:10E4B000ACFD0546FFF775FD692D01D1207808B147
:10E4C00000204EE7F0B22071642801D9002048E70F
:10E4D000012046E770472DE9FE430020009001909F
:10E4E0000290DFF8D88288F80000FFF741FDC120D4
:10E4F000FFF768FD1E2004F059FFFFF7CDFD20B1A6
:10E50000FFF74FFD0020BDE8FE831E2004F04EFF04
:10E51000FFF77BFD0646ADF80000FFF7DFFD1E208C
:10E5200004F044FFFFF771FDADF802000746FFF766
:10E53000D5FD1E2004F03AFFFFF767FDADF804009B
:10E540000546FFF7CBFD1E2004F030FFFFF75DFD11
:10E55000ADF806000446FFF7C1FD1E2004F026FFBB
:10E56000FFF753FDADF808008146FFF71AFDF019DB
:10E570002919084481B2894502D198F8000008B1F0
:10E580000020C0E78F48BDF800100180BDF80210E0
:10E590004180C58204760120B5E770B50446874EF8
:10E5A00000203070FFF7E4FCE520FFF70BFDE525C8
:10E5B0000A2004F0FBFEFFF76FFD18B1FFF7F1FC36
:10E5C0000020CEE6C4F30720FFF7FCFC05EB242077
:10E5D00085B21E2004F0EAFEFFF75EFD18B1FFF7DA
:10E5E000E0FC0020BDE6E0B2FFF7ECFCE0B228441E
:10E5F00084B21E2004F0DAFEFFF74EFD18B1FFF7DB
:10E60000D0FC0020ADE61E2004F0D0FEFFF7FDFC9C
:10E61000A04208D1FFF7C5FC3078012801D00120C5
:10E620009FE600209DE6FFF7BCFC002099E670B550
:10E630000446624E00203070FFF79AFCE620FFF798
:10E64000C1FCE6251E2004F0B1FEFFF725FD18B140
:10E65000FFF7A7FC002084E6200AFFF7B3FC05EBD8
:10E66000142085B21E2004F0A1FEFFF715FD18B19D
:10E67000FFF797FC002074E6E0B2FFF7A3FCE0B2DE
:10E68000284484B21E2004F091FEFFF705FD18B166
:10E69000FFF787FC002064E61E2004F087FEFFF7EA
:10E6A000B4FCA04208D1FFF77CFC3078012801D0EF
:10E6B000012056E6002054E6FFF773FC002050E6E8
:10E6C0002DE9F04104460D463C4F00203870FFF71D
:10E6D0004FFCD320FFF776FCD3261E2004F066FE05
:10E6E000FFF7DAFC18B1FFF75CFC00208BE4200A8E
:10E6F000FFF768FC06EB142086B21E2004F056FEDD
:10E70000FFF7CAFC18B1FFF74CFC00207BE4E0B235
:10E71000FFF758FCE0B2304484B21E2004F046FEFD
:10E72000FFF7BAFC18B1FFF73CFC00206BE4280AA5
:10E73000FFF748FC04EB152084B21E2004F036FEDF
:10E74000FFF7AAFC18B1FFF72CFC00205BE4E8B24D
:10E75000FFF738FCE8B2204484B21E2004F026FE05
:10E76000FFF79AFC18B1FFF71CFC00204BE41E20B9
:10E7700004F01CFEFFF749FCA04208D1FFF711FC92
:10E780003878012801D001203DE400203BE4FFF768
:10E7900008FC002037E410B5084C00202070FFF77B
:10E7A000E7FBE420FFF70EFC1E2004F0FFFDFFF75F
:10E7B00073FC48B1FFF7F5FB002010BD9A00002064
:10E7C000A2810020FC0900201E2004F0EFFDFFF7CD
:10E7D0001CFCE42803D0FFF7E4FB0020EDE7FFF783
:10E7E000E0FB2078012801D00120E6E70020E4E7E3
:10E7F0002DE9FC4704468846914600200090019090
:10E80000FD4F3870FFF7B4FBD420FFF7DBFB1E2071
:10E8100004F0CCFDFFF740FC20B1FFF7C2FB002065
:10E82000BDE8FC872046FFF7CDFB1E2004F0BEFDAF
:10E83000FFF732FC18B1FFF7B4FB0020F0E71E2011
:10E8400004F0B4FDFFF7E1FBADF800000446FFF76C
:10E8500045FC1E2004F0AAFDFFF7D7FBADF802002F
:10E860000546FFF73BFC1E2004F0A0FDFFF7CDFBA3
:10E87000ADF804000646FFF731FCFFF792FB601984
:10E8800081B28E4201D1387808B10020C8E7A8F8DB
:10E890000040A9F800500120C2E72DE9FC410646DE
:10E8A000FFF766FBEF20FFF78DFB1E2004F07EFDD7
:10E8B000FFF7F2FB20B1FFF774FB0020BDE8FC81FD
:10E8C0001E2004F073FDFFF7A0FBADF80000054625
:10E8D000FFF704FC1E2004F069FDFFF796FBADF87E
:10E8E00002000446FFF7FAFB1E2004F05FFDFFF76D
:10E8F0008CFBADF804000746FFF7F0FB1E2004F088
:10E9000055FDFFF74EFB281981B28F4204D104EB6D
:10E91000052030800120D1E70020CFE72DE9FE431C
:10E9200004460D460020009001900290DFF8C88256
:10E9300088F80000FFF71CFB2046FFF743FB1E2072
:10E9400004F034FDFFF7A8FB18B1FFF72AFB002005
:10E95000D9E52846FFF736FB1E2004F027FDFFF718
:10E960009BFB18B1FFF71DFB0020CCE51E2004F037
:10E970001DFDFFF74AFB0646ADF80000FFF7AEFBB2
:10E980001E2004F013FDFFF740FBADF80200074620
:10E99000FFF7A4FB1E2004F009FDFFF736FBADF8DE
:10E9A00004000546FFF79AFB1E2004F0FFFCFFF76A
:10E9B0002CFBADF806000446FFF790FB1E2004F088
:10E9C000F5FCFFF722FBADF808008146FFF7E9FAF6
:10E9D000F0192919084481B2894502D198F800003C
:10E9E00008B100208FE58548BDF800100180BDF812
:10E9F00002104180C5820476012084E52DE9FC47A0
:10EA00000446DDF828900D461646984600200090F2
:10EA10000190794F3870FFF7ABFA2046FFF7D2FA32
:10EA20001E2004F0C3FCFFF737FB18B1FFF7B9FA5B
:10EA30000020F5E62846FFF7C5FA1E2004F0B6FCD4
:10EA4000FFF72AFB18B1FFF7ACFA0020E8E63046E2
:10EA5000FFF7B8FA1E2004F0A9FCFFF71DFB18B160
:10EA6000FFF79FFA0020DBE61E2004F09FFCFFF773
:10EA7000CCFAADF800000446FFF730FB1E2004F08E
:10EA800095FCFFF7C2FAADF802000546FFF726FB3A
:10EA90001E2004F08BFCFFF7B8FAADF80400064620
:10EAA000FFF71CFBFFF77DFA601981B28E4201D19E
:10EAB000387808B10020B3E6A8F80040A9F8005063
:10EAC0000120ADE62DE9FC4107460D461446002025
:10EAD00000900190484E3070FFF74AFA3846FFF731
:10EAE00071FA1E2004F062FCFFF7D6FA28B1FFF796
:10EAF00058FA0A2020800020E0E62846FFF762FA54
:10EB00001E2004F053FCFFF7C7FA28B1FFF749FABB
:10EB10000B2020800020D1E6FFF777FAADF8000047
:10EB20000546FFF7DBFA1E2004F040FCFFF76DFA04
:10EB3000ADF802000746FFF7D1FA1E2004F036FCBC
:10EB4000FFF763FAADF804008046FFF7C7FA1E200E
:10EB500004F02CFCFFF725FAE81981B2884501D1B1
:10EB6000307818B10C2020800020A7E625800120F5
:10EB7000A4E62DE9F04106460D4614461E4F00203E
:10EB80003870FFF7F5F93046FFF71CFA1E2004F045
:10EB90000DFCFFF781FA18B1FFF703FA0020A5E595
:10EBA0002846FFF70FFA1E2004F000FCFFF774FA66
:10EBB00018B1FFF7F6F9002098E57019C0B2FFF719
:10EBC00001FA1E2004F0F2FBFFF766FA18B1FFF716
:10EBD000E8F900208AE5C4F30720FFF7F3F9C4F34E
:10EBE0000F251E2004F0E2FBFFF756FA40B1FFF7B5
:10EBF000D8F900207AE500009A000020FC090020E6
:10EC0000E0B2FFF7DFF9E0B2284484B21E2004F03E
:10EC1000CDFBFFF741FA18B1FFF7C3F9002065E516
:10EC20001E2004F0C3FBFFF7F0F9A04208D1FFF764
:10EC3000B8F93878012801D0012057E5002055E5C2
:10EC4000FFF7AFF9002051E52DE9F04180460E466F
:10EC500015461C46F74F00203870FFF789F94046EB
:10EC6000FFF7B0F91E2004F0A1FBFFF715FA18B169
:10EC7000FFF797F9002039E53046FFF7A3F91E208A
:10EC800004F094FBFFF708FA18B1FFF78AF90020A7
:10EC90002CE508EB0600C0B2FFF794F91E2004F043
:10ECA00085FBFFF7F9F918B1FFF77BF900201DE5A7
:10ECB0002E0A3046FFF786F91E2004F077FBFFF797
:10ECC000EBF918B1FFF76DF900200FE5E8B2FFF797
:10ECD00079F9E8B2304485B21E2004F067FBFFF7F3
:10ECE000DBF918B1FFF75DF90020FFE4200AFFF718
:10ECF00069F905EB142085B21E2004F057FBFFF7DD
:10ED0000CBF918B1FFF74DF90020EFE4E0B2FFF7BF
:10ED100059F9E0B2284484B21E2004F047FBFFF703
:10ED2000BBF918B1FFF73DF90020DFE41E2004F025
:10ED30003DFBFFF76AF9A04208D1FFF732F93878B6
:10ED4000012801D00120D1E40020CFE4FFF729F908
:10ED50000020CBE42DE9FE4F04460D460020009034
:10ED600001900290DFF8CCA28AF80000FFF700F9CA
:10ED70002046FFF727F91E2004F018FBFFF78CF957
:10ED800020B1FFF70EF90020BDE8FE8F2846FFF7FF
:10ED900019F91E2004F00AFBFFF77EF918B1FFF7FE
:10EDA00000F90020F0E7FFF730F90646ADF8000063
:10EDB000FFF794F91E2004F0F9FAFFF726F9ADF8F1
:10EDC00002000746FFF78AF91E2004F0EFFAFFF76A
:10EDD0001CF90446ADF80400FFF780F91E2004F08A
:10EDE000E5FAFFF712F9ADF806000546FFF776F9E8
:10EDF0001E2004F0DBFAFFF708F9ADF808008046A2
:10EE0000FFF76CF91E2004F0D1FAFFF7FEF8ADF819
:10EE10000A008146FFF7C5F8F0196119084440441B
:10EE200081B2894502D19AF8000008B10020ABE711
:10EE30008148BDF800100180BDF802104180C482F5
:10EE400005760120A0E71CB504467C480078002820
:10EE50001ED1784801796F291AD00A2918D0DE29E5
:10EE600016D07548828804B93AB101210020CDE955
:10EE700000100B460C21FEF728F9002C08D002B038
:10EE800000232522BDE810400D211846FDF7D2BF12
:10EE90001CBD68480079182801D2FFF71CBB04D1BB
:10EEA0004FF0C1014FF05A0038E5C1215A2051E717
:10EEB00060490979182901D2FFF76FBB0246E521A5
:10EEC0005A2056E65B4A1279182A01D2FFF7F8BB9E
:10EED0000B460246D3215A20B6E608B5554B1B799E
:10EEE000182B02D2BDE8084082E400920B4602468D
:10EEF000D4215A20FFF782FD08BD4E48007918281A
:10EF000000D248E40122E4215A2032E64949097935
:10EF1000182901D2FFF78BBB02B2E6215A2028E65E
:10EF200044490979182900D2B7E40246EF215A2052
:10EF3000C8E540490979182903D90246D5215A2044
:10EF400017E6002070470246C4215A20BAE52DE991
:10EF5000F041384C00262046A278374DB0F9060023
:10EF6000012A10D03649022A097820D0042A09D172
:10EF700002296DD0C0B2FFF7DCFF002802D0A670D6
:10EF8000A079607006E4AA89E98B801A0844E883B6
:10EF9000A670C1B240F25A70FDF786FBE88BBDE85F
:10EFA000F041C0F3072140F25B70FDF77DBB40F2FA
:10EFB0005C7740F25D78012902D0022924D036E046
:10EFC00020481C4A01782048D2880088101A00B2D4
:10EFD00001290DD06884C1B240F25E70FDF764FB78
:10EFE000688CC0F3072140F25F70FDF75DFB1EE007
:10EFF0002884C1B23846FDF757FB288CC0F307219F
:10F000004046FDF751FB12E022F03BFF0F49096833
:10F0100022F039FD22F054FF2884C1B23846FDF7B2
:10F0200043FB288CC0F307214046FDF73DFBA6704B
:10F03000B5E50DE09A000020FC09002063000020E7
:10F0400050030020560300206603002070030020B8
:10F05000012801D018B104E000F0A7FF01E000F0A2
:10F06000B2FFA670A079607099E570B521480024C0
:10F07000214D0078002801D0EC7070BD1E481F495A
:10F080006B7890F903200978501C40B21BB1182A04
:10F090001FDAE87070BD1A4B40F2B6369B88B34257
:10F0A00015D9782A01DAE87070BD0126022907D047
:10F0B0000120FFF73EFF0028F6D0EC706E7070BDA7
:10F0C00000F073FF0028FAD1EC706E7070BDEC7028
:10F0D00070BD022907D00020FFF72BFF0028F7D0D2
:10F0E000EC706C7070BD00F06EFF0028FAD1EC700F
:10F0F0006C7070BD520300209A0000205003002065
:10F10000FC09002070B592B00020A14D002425F824
:10F110001040401CC0B25028F9D3F020ADF80400D4
:10F120008DF8074001A99B48FBF7BFF90320ADF814
:10F1300004008DF8074001A99748FBF7B6F9302085
:10F14000ADF804008DF8074001A99448FBF7ADF92C
:10F1500001210846FBF7C2FB914E3046FBF748F809
:10F1600090490291039504945020059006948020C4
:10F170000790400008908000099020200A9000022B
:10F180000B900C9402A93046FBF7A9F801213046F8
:10F19000FBF7CFF801214802FBF7ABFB4FF400402F
:10F1A000FBF72AFB0D9401208DF838008DF839000B
:10F1B0004FF460200F90109408208DF84400794C93
:10F1C0000DA94C3C2046FAF77BFE052301220421C1
:10F1D0002046FAF7FFFE0523022219462046FAF7D9
:10F1E000F9FE0523032206212046FAF7F3FE052344
:10F1F000042207212046FAF7EDFE05231A460821CE
:10F200002046FAF7E7FE0523062209212046FAF7F1
:10F21000E1FE052307220E212046FAF7DBFE052337
:10F2200008220F212046FAF7D5FE01212046FAF7E1
:10F230007BFE01212046FAF76BFE2046FAF78BFE93
:10F240002046FAF78DFE0028FAD12046FAF78FFE05
:10F250002046FAF791FE0028FAD101212046FAF75C
:10F2600092FE12B070BD4DE72DE9F04186B0002549
:10F27000474F01AE08286ED2DFE800F01E110445AA
:10F28000382B50610020052101EBC00237F8122015
:10F2900026F81020401CC0B20A28F5D35BE00020FD
:10F2A000042101EBC00237F8122026F81020401C80
:10F2B000C0B20A28F5D34EE00020032101EBC002C2
:10F2C00037F8122026F81020401CC0B20A28F5D3C7
:10F2D00041E00020022101EBC00237F8122026F89D
:10F2E0001020401CC0B20A28F5D334E000200121D0
:10F2F00001EBC00237F8122026F81020401CC0B2E3
:10F300000A28F5D327E0002007EB0011098826F82A
:10F310001010401CC0B20A28F6D31CE000244FF0A5
:10F32000060808EBC40037F8100026F814000A207D
:10F3300004F05CF8641CE4B20A2CF2D30BE0002069
:10F34000072101EBC00237F8122026F81020401CDC
:10F35000C0B20A28F5D3BDF804201346002036F8C1
:10F3600010104C19A5B2914200D80A46994200D318
:10F370000B46401CC0B20A28F1D3A81AC01AC11704
:10F3800000EB517006B0C0F3CF00BDE8F081000083
:10F39000300A002000080140000C0140001001402C
:10F3A000080002404C24014070B506460420FDF7D9
:10F3B0001DFD6C20FDF729FDF74D012E18D000240E
:10F3C0000020FDF7CBFC641CE4B2182CF8D3052018
:10F3D000FDF70CFD6C20FDF718FD012E11D0002467
:10F3E0000020FDF7BBFC641CE4B2182CF8D370BD00
:10F3F0000024285DFDF7B2FC641CE4B2182CF8D39D
:10F40000E5E700242819007EFDF7A8FC641CE4B29F
:10F41000182CF7D370BD2DE9F041DFF8808320F080
:10F42000800098F80010884234D088F80000062048
:10F43000FDF7DCFC6C20FDF7E8FCD74D98F80000E8
:10F44000303505F1300605F16007022824D0032885
:10F4500022D0012829D00024385DFDF77FFC641CF0
:10F46000E4B2182CF8D30720FDF7C0FC6C20FDF7A0
:10F47000CCFC98F80000022820D003281ED00128D8
:10F4800026D000243819007EFDF768FC641CE4B225
:10F49000182CF7D3BDE8F0810024285DFDF75EFC51
:10F4A000641CE4B2182CF8D3DDE70024305DFDF7CE
:10F4B00055FC641CE4B2182CF8D3D4E700242819B6
:10F4C000007EFDF74BFC641CE4B2182CF7D3E1E797
:10F4D00000243019007EFDF741FC641CE4B2182CB6
:10F4E000F7D3D7E72DE9F04707468846202A29D0E9
:10F4F0002A2A29D02E2A29D0303A092A20D8D0B257
:10F500000025A74900EB401001EB80064046FDF7BF
:10F510007CFC7819C0B2FDF769FC002405EB4500BE
:10F5200000EBC50006EB400919F80400FDF716FCD6
:10F53000641CE4B2162CF7D36D1CEDB2062DE5D396
:10F54000BDE8F0870A20DBE70B20D9E70C20D7E7DE
:10F550002DE9FC4104460E4692A003C8CDE9000106
:10F560006F46002E0BD0002516206843C1B27A5D8D
:10F570000220FFF7B7FF6D1CEDB2052DF4D306B1E5
:10F580000126202164B364220A2042F210754FF450
:10F590007A7396B3AC427CD22E259C427AD3B4FBCC
:10F5A000F3F130318DF80010B4FBF3F103FB11419E
:10F5B000B1FBF2F330338DF80130B1FBF2F302FB13
:10F5C0001311B1FBF0F230328DF802208DF80350A8
:10F5D000B1FBF0F200FB121030308DF80400C8E0EF
:10F5E0008DF800108DF801102A208DF802008DF89A
:10F5F00003008DF804000026BBE0FFE7AC4227D3F0
:10F60000B4FBF5F130318DF80010B4FBF5F105FBDA
:10F610001141B1FBF3F430348DF80140B1FBF3F448
:10F6200003FB1411B1FBF2F330338DF80230B1FB60
:10F63000F2F302FB1311B1FBF0F230328DF803202C
:10F64000B1FBF0F200FB121030308DF8040090E0B6
:10F650009C4223D38DF80010B4FBF3F130318DF8C8
:10F660000110B4FBF3F103FB1141B1FBF2F33033B2
:10F670008DF80230B1FBF2F302FB1311B1FBF0F293
:10F6800030328DF80320B1FBF0F200FB1210303065
:10F6900001E097E03FE08DF804006AE0642C19D3A4
:10F6A0008DF800108DF80110B4FBF2F130318DF8B7
:10F6B0000210B4FBF2F102FB1141B1FBF0F2303267
:10F6C0008DF80320B1FBF0F200FB121030308DF802
:10F6D00004004EE00A2C12D38DF800108DF80110B2
:10F6E0008DF80210B4FBF0F130318DF80310B4FB4B
:10F6F000F0F100FB114030308DF8040039E08DF856
:10F7000000108DF801108DF802108DF803103034C0
:10F710008DF804402DE0642C19D38DF80010B4FB53
:10F72000F2F130318DF80110B4FBF2F102FB11411E
:10F73000B1FBF0F230328DF802208DF80350B1FBAE
:10F74000F0F200FB121030308DF8040011E08DF85B
:10F7500000108DF80110B4FBF0F130318DF802107B
:10F760008DF80350B4FBF0F100FB114030308DF800
:10F770000400DEB10024B44226D9C4F1040000EB39
:10F7800040013A5C01EBC0000C2101EB4000C1B22A
:10F790000220FFF7A7FE20E0B3550308180300205E
:10F7A000FF4E030820202020200000000024162007
:10F7B0006043C1B23A5D0220FFF794FE641CE4B2DC
:10F7C000052CF4D3BDE8FC81C4F1040016213A5C99
:10F7D0004843C1B20220FFF785FE641CE4B2052C49
:10F7E000C9D3EFE72DE9F0470746202A09D02D2A93
:10F7F00009D02E2A09D0A2F13000092807D8C0B2BA
:10F8000016E00C2014E00B2012E00A2010E04F2A32
:10F8100034D0552A34D0542A34D0522A34D0412AF4
:10F8200034D04E2A34D0472A34D0452A25D114204A
:10F830000025C1EBC101022202EB4108C0EBC00070
:10F84000414900EB400001EB800908F0FF00FDF7A3
:10F85000DCFA7819C0B2FDF7C9FA0024C5EBC5007F
:10F8600009EB4006305DFDF779FA641CE4B20E2C1A
:10F87000F8D36D1CEDB2062DE7D361E60D20D7E776
:10F880000E20D5E70F20D3E71020D1E71120CFE7D6
:10F890001220CDE71320CBE72DE9F04780460E4636
:10F8A00017460024384621F029FFC5B227480178C1
:10F8B000D4290DD0D5290BD0342909D0D62901D08F
:10F8C000D72935D1C6F10900A8423ADAC5B238E0E5
:10F8D000082E00D9082606F101094D450DD909F079
:10F8E000FF050AE0281B384410F8012C301BC1B278
:10F8F0004046FFF777FF641CE4B2AC42F2D3002429
:10F90000751B6D1C06E0202221464046FFF76AFF6A
:10F91000641CE4B2A542F6DC09F0FF0406E02022F4
:10F9200021464046FFF75EFF641CE4B2092CF6D383
:10F9300006E63019C1B23A5D4046FFF753FF641C3A
:10F94000E4B2AC42F5D3FBE5735603080400002093
:10F9500070B5FCF704FB6E4C012626606D4D2888BF
:10F9600003F024FD6660288803F020FD0026266051
:10F97000288800EB8000400003F018FD66602888AE
:10F98000BDE8704000EB8000400003F00FBD70B593
:10F99000FCF7E5FA5E4C002666605E4D288803F0B1
:10F9A00005FD2660288803F001FD01266660288891
:10F9B00000EB8000400003F0F9FC26602888BDE8D9
:10F9C000704000EB8000400003F0F0BC2DE9F047F0
:10F9D0008146FCF7C4FA80244F4E4E4D00274FF06D
:10F9E000010814EA090F02D1C6F8887101E0C6F8CF
:10F9F0008881298801EB810003F0D8FCC6F88C814E
:10FA0000298801EB810003F0D1FCC6F88C712888AD
:10FA100003F0CCFC6408002CE3D1BDE8F047FCF710
:10FA20000EBB2DE9F04104460026FCF7A7FA4FF47F
:10FA30007A77394D08E0641EE4B202D20420BDE8B2
:10FA4000F081384603F0B2FCD5F80C010028F2D062
:10FA50003046F4E72DE9F84F05468A4693464FF0C5
:10FA6000000985F800902C4E4FF00108C6F88881F7
:10FA7000FCF764FA8024274FC6F88C81388803F09D
:10FA800095FC5846FFF7CDFF0090388800EB40000A
:10FA900003F08CFCFCF783FAD6F8080110B1287843
:10FAA00020432870C6F88C91388803F07FFC6408E6
:10FAB000002CE1D1FCF753FABAF1000F18D0C6F8C8
:10FAC0008881388803F072FCC6F88C81388800EB96
:10FAD000800003F06BFCC6F88C91C6F888813888EA
:10FAE00000EB8000800003F061FC0098BDE8F88F17
:10FAF000C6F88891E5E710B5FFF72AFF0020FFF769
:10FB000065FF002803D1BDE8104006205EE710BD68
:10FB1000880121425C03002000002142F949400095
:10FB2000087040F0010048707047F7E7FFF72FBFFB
:10FB300070B50546FF20002340F2311410E0EA5C66
:10FB400050400822060603D584EA4000C0B201E016
:10FB50004006000E521ED2B2002AF3D15B1CDBB26B
:10FB60008B42ECD370BD10B51446FFF7E1FFA04205
:10FB700001D0022010BD002010BD7CB504460D460A
:10FB8000002101A8FFF766FF28B9002211460DF1F8
:10FB90000500FFF75FFF20B9002229466846FFF7FE
:10FBA00059FF28B99DF80020022101A8FFF7DBFFCB
:10FBB0009DF805109DF8042041EA022121807CBDBA
:10FBC00010B5FFF7C5FECF484078BDE81040FFF7FD
:10FBD000FDBE70B50446200AFFF7F8FE0546E0B208
:10FBE000FFF7F4FE284370BD10B5FFF7B1FEC5481E
:10FBF0000078BDE81040FFF7E9BEF8B50646FFF70C
:10FC0000F3FF05464FF45E50FFF7E3FF40EA0504BB
:10FC100014B9FFF7D5FF04462CB9642200216846C9
:10FC2000FFF7ABFF044634B9002201210DF10200B9
:10FC3000FFF7A3FF0446FFF779FF34B9BDF80200D0
:10FC4000BDF8001040EA014030602046F8BD70B5B4
:10FC50000546FFF7C9FF044624B94FF22D30FFF7E0
:10FC6000B8FF044614B9FFF7ABFF04462CB90022D5
:10FC700001212846FFF781FF0446FFF757FF204682
:10FC800070BD10B5FFF7B0FF044624B943F2410040
:10FC9000FFF79FFF0446FFF749FF204610BD10B550
:10FCA00022F0F8F8984921F0F4FE984921F0F1FE8D
:10FCB000BDE81040964921F01EBF10B522F0EAF8C9
:10FCC000944921F0E6FE914921F0E3FE904921F0AC
:10FCD00012FFBDE81040904921F0D5BE2DE9FC414E
:10FCE0000746884616461D46FFF77EFF044620005D
:10FCF00005D196B1012E0AD0022E02D0802494B1F3
:10FD000020E042F21640FFF764FF0446F7E742F2B4
:10FD10000B40FFF75EFF0446F1E74FF41050FFF78A
:10FD200058FF0446EBE74FF47A7606E0FFF748FF0A
:10FD300004462CB1304603F039FB6D1EEDB2F5D20E
:10FD400005B9042464B90022114601A8FFF715FF84
:10FD50000546002201216846FFF70FFF40EA05042F
:10FD6000FFF7E4FE54B9BDF80400FFF7A6FF3860C2
:10FD7000BDF80000FFF793FFC8F800002046BDE87B
:10FD8000FC812DE9FC4106460F4615469846FFF7D3
:10FD90002BFF04462CB995B1012D0AD0022D02D0BB
:10FDA000802494B114E042F61040FFF712FF04469D
:10FDB000F7E742F60D40FFF70CFF0446F1E742F685
:10FDC0000640FFF706FF0446EBE7FFF7F9FE04469F
:10FDD0002CB94246002101A8FFF7CFFE04462CB9FA
:10FDE000002201216846FFF7C8FE0446FFF79EFE89
:10FDF0004CB9BDF80400FFF760FF3060BDF80000AB
:10FE0000FFF74DFF38602046B9E730B4029C002B65
:10FE100004D0012B05D0802030BC7047234630BC75
:10FE2000AFE7234630BC59E770B505460E46FFF7ED
:10FE3000DBFE04462CB97DB3012D2ED0022D04D05B
:10FE40008024FFF773FE204670BD052E22D2DFE826
:10FE500006F003090F151B0042F22F00FFF7B9FE51
:10FE60000446EEE742F22D10FFF7B3FE0446E8E742
:10FE700042F22B20FFF7ADFE0446E2E742F22930C2
:10FE8000FFF7A7FE0446DCE742F22A70FFF7A1FE67
:10FE90000446D6E78024D4E726E0052E22D2DFE808
:10FEA00006F003090F151B0042F22400FFF791FE34
:10FEB0000446C6E742F22610FFF78BFE0446C0E771
:10FEC00042F22020FFF785FE0446BAE742F22230D4
:10FED000FFF77FFE0446B4E742F22170FFF779FE98
:10FEE0000446AEE78024ACE7052E2FD2DFE806F00B
:10FEF00003161C22280042F23200FFF76AFE044675
:10FF00009FE70000A20000200000C842000020413E
:10FF100000FF7F4700002F430000E14342F2301012
:10FF2000FFF757FE04468CE742F23620FFF751FEFA
:10FF3000044686E742F23430FFF74BFE044680E782
:10FF400042F23770FFF745FE04467AE7802478E7EF
:10FF50007CB505460E46FFF747FE044624B94FF42C
:10FF60006040FFF736FE044614B9FFF729FE044649
:10FF70002CB90022114601A8FFF7FFFD04462CB959
:10FF8000002201216846FFF7F8FD04464CB9BDF890
:10FF90000400FFF792FE2860BDF80000FFF77FFE27
:10FFA0003060FFF7C3FD20467CBD10B5FFF71CFE97
:10FFB000044624B943F26D00FFF70BFE0446FFF739
:10FFC000B5FD204610BD10B5FFF70EFE044624B95E
:10FFD00043F26600FFF7FDFD0446FFF7A7FD20464C
:10FFE00010BD70B5FFF700FE054643F2A200FFF713
:10FFF000F0FD40EA0504FFF799FD1CB94CF25030C2
:020000040801F1
:1000000003F0D4F9204670BD10B5244C4FF0805059
:100010002060234803F0CAF9A0142060BDE8104016
:100020004CF2503003F0C2B938B5010A8DF8001017
:100030008DF8010002216846FFF77AFD04469DF81D
:100040000000FFF7C3FC18B99DF80100FFF7BEFCE4
:10005000002802D12046FFF7B9FC38BD10B5114980
:1000600021F0BFFC104921F046FD104921F011FD9F
:1000700021F03FFF80B210BD10B50D4921F03BFDCE
:100080000A4921F006FD21F034FF80B210BD03487B
:1000900008380068C0F3802070470000100C014051
:1000A000A08601000000344200002F4300FF7F477C
:1000B0000000C84270B586B001214020FAF719FC53
:1000C0004FF40050ADF8140010258DF8175002249D
:1000D0008DF81640FE4E05A93046FAF7E6F9E00223
:1000E000ADF810008DF813508DF8124004A9304679
:1000F000FAF7DBF96003ADF80C008DF80F508DF8BE
:100100000E4003A93046FAF7D0F9A003ADF8080075
:100110008DF80B508DF80A4002A93046FAF7C5F960
:10012000A002ADF804008DF807508DF8064001A933
:10013000E848FAF7BAF96002ADF800008DF803500C
:100140008DF8024069463046FAF7AFF906B070BD47
:100150007047704770B572B60024DF4BC3F8AC41EE
:100160000125C3F8B4510022C3F8B841060602D5F0
:10017000C3F8BC5101E0C3F8BC41C3F8B851400614
:10018000000E521CD2B2082AEED30020C3F8B841A8
:100190000A0602D5C3F8BC5101E0C3F8BC41C3F85C
:1001A000B8514906090E401CC0B20828EED3C3F866
:1001B000AC5162B670BDC0F30722C1B21046C9E7A8
:1001C00030B572B60023C44AC2F8AC31C2F8B431BB
:1001D00000210124C2F8B831050602D5C2F8BC419D
:1001E00001E0C2F8BC31C2F8B8414006000E491C1B
:1001F000C9B20829EED3C2F8AC4162B630BD30B501
:10020000B54A0023C2F8AC310124C2F8B441002140
:10021000C2F8B831050602D5C2F8BC4101E0C2F807
:10022000BC31C2F8B8414006000E491CC9B20829C9
:10023000EED3C2F8AC4130BD2DE9F043814688468B
:10024000C2F30724D5B2C3F30726DFB22A20FFF793
:10025000B7FF0020FFF7D3FF4846FFF7D0FF00208D
:10026000FFF7CDFF4046FFF7CAFF2B20FFF7A8FF9F
:100270002046FFF7C4FF2846FFF7C1FF3046FFF7CF
:10028000BEFF3846FFF7BBFFBDE8F0432C2097E7E1
:100290002DE9F0410746002240F23F13EF211046BE
:1002A000FFF7CAFF00254FF4A07600243846FFF779
:1002B00082FF641CF02CF9D36D1CB542F5D3BDE868
:1002C000F08100B52820FFF77BFF10205DF804EBDC
:1002D00076E710B51120FFF773FF782003F086F85A
:1002E000BDE8104029206BE770B57C4C01252560E6
:1002F000052003F07BF8002060600A2003F076F808
:100300006560782003F072F81120FFF759FF78201C
:1003100003F06CF8CF20FFF753FF0020FFF76FFFCB
:10032000C320FFF76CFF3020FFF769FFED20FFF7D8
:1003300047FF6420FFF763FF0320FFF760FF1220F1
:10034000FFF75DFF8120FFF75AFFE820FFF738FF36
:100350008520FFF754FF1020FFF751FF7920FFF7AA
:100360004EFFCB20FFF72CFF3920FFF748FF2C2052
:10037000FFF745FF0020FFF742FF3420FFF73FFF64
:100380000220FFF73CFFF720FFF71AFF2020FFF7BE
:1003900036FFEA20FFF714FF0020FFF730FF0020B0
:1003A000FFF72DFFC020FFF70BFF2220FFF727FFED
:1003B000C120FFF705FF1120FFF721FFC520FFF740
:1003C000FFFE3D20FFF71BFF2020FFF718FFC7208F
:1003D000FFF7F6FEAA20FFF712FF3620FFF7F0FE28
:1003E000C820FFF70CFF3A20FFF7EAFE5520FFF781
:1003F00006FFB120FFF7E4FE0020FFF700FF132007
:10040000FFF7FDFEB620FFF7DBFE0A20FFF7F7FE41
:10041000A220FFF7F4FEF620FFF7D2FE0120FFF73F
:10042000EEFE3020FFF7EBFEF220FFF7C9FE0020C2
:10043000FFF7E5FE2620FFF7C3FE0120FFF7DFFEF2
:10044000E020FFF7BDFE0F20FFF7D9FE3F20FFF7AA
:10045000D6FE2F20FFF7D3FE0C20FFF7D0FE102092
:10046000FFF7CDFE0A20FFF7CAFE5320FFF7C7FEB5
:10047000D520FFF7C4FE4020FFF7C1FE0A20FFF79A
:10048000BEFE1320FFF7BBFE0320FFF7B8FE0820D7
:10049000FFF7B5FE0320FFF7B2FE0020FFF7AFFE27
:1004A000E120FFF78DFE0020FFF7A9FE0020FFF7F7
:1004B000A6FE1020FFF7A3FE0320FFF7A0FE0F20EB
:1004C000FFF79DFE0520FFF79AFE2C2008E00000B4
:1004D000001801400014014000002342AC012342F7
:1004E000FFF78DFEA220FFF78AFE3F20FFF787FE71
:1004F0000520FFF784FE0E20FFF781FE0C20FFF79A
:100500007EFE3720FFF77BFE3C20FFF778FE0F20B2
:10051000FFF775FE1120FFF753FE782002F066FF0B
:100520002920FFF74DFEBDE87040322002F05EBF8B
:1005300010B5FFF7BFFDFE4800210160C1600161F9
:1005400041608160FFF7D0FEFA480078FDF789F935
:10055000BDE8104047F619609AE62DE9F05FDDE945
:100560000A7800281DD0203B012839D0F24D2026E2
:1005700010245802C31700EB537005EBE0058819EF
:10058000401E00F0FF0C1319C8B25B1E6146FFF756
:1005900053FE7443E01704EB5070C0F3CF090026FC
:1005A00044E0E64D482628242D2B10D0202B11D0D6
:1005B0002E2B12D0303B03EB8300C00000EBC000B9
:1005C000C000C31700EB537005EBE005D7E705F556
:1005D0006165D4E705F67875D1E705F58755CEE76F
:1005E000D74D2026182403EB43000002C31700EB6D
:1005F000537005EBE005C2E700244FEA182A4FEAE2
:10060000172B2878E040C00704D0F9B25846FFF70E
:10061000A1FD04E008F0FF015046FFF79BFD641CBC
:10062000A4B2082CEDD36D1C761CB6B24E45E3D3B4
:10063000BDE8F09F2DE9FC470646DDE90A890F4633
:1006400014461D460BE0A2B2B9B23046CDE900898E
:10065000FFF783FF46B1012E08D00F3C6D1C2B78AD
:10066000002BF0D1BDE8FC87283CF7E7173CF5E705
:1006700070B51646049A01FB00F4A5B2541818444C
:10068000401EC1B2641ED8B22346FFF7D5FD002438
:1006900007E036F81400C1B2000AFFF75BFD641CE6
:1006A000A4B2AC42F5D370BD2DE9F041089E069A84
:1006B00001FB00F4A5B254181844401EC1B2641ED8
:1006C000D8B22346FFF7B8FD0024370A05E0F1B29F
:1006D0003846FFF73FFD641CA4B2AC42F7D3EEE509
:1006E0002DE9F0438DB0DFF85C9299F804000928F9
:1006F00002D9092089F8040099F80400002877D06D
:100700000024904EDFF84082223606F11E052D3679
:100710006AE034B1012C10D0022C1AD0032C61D124
:1007200035E088480C3020F0E9FF02468548223049
:10073000A0F1160120F094FF54E08248173020F019
:10074000DDFF02467F483130A0F11A0120F088FF1A
:1007500048E07E4820F0D2FFC7B228463A467B499F
:1007600020F07EFF7A48007840B17A4820F0C6FF3A
:100770000246E819774920F073FF33E0764820F00D
:10078000BDFF0246E819744920F06AFF2AE0734869
:1007900020F0B4FFC7B230463A46704920F060FFFF
:1007A0006F48007830F0800004D06E48007801284F
:1007B00005D017E0F019D8F80010016012E06A487F
:1007C0006A4A6BA1807B00EBC00000EB080368461F
:1007D00022F026FA684620F091FF0246F019694699
:1007E00020F03EFF641CE4B299F80400844290D3E8
:1007F0000DB0BDE8F0832DE9FC5FFFF771FFDFF876
:1008000044815D4F4FF0000998F8041047F6106AD4
:100810004FF6FF7E4FF48C7208F1220C012911D0A3
:1008200024D9A1F10101C1EB011000EB0C03D8F8B0
:10083000081003F1010088422FD800205C1A04F14F
:100840000F0519E00020491EC1EB011161440B5C4A
:100850003B54401CC0B20D28F9D387F80D90CDE968
:1008600000EA454BCD210120FFF7E4FEBDE8FC9FE7
:100870000E5C3E54401CC0B28542F9DC0020CE1A0A
:1008800008E004EB000BBB441CF800508BF80F5041
:10089000401CC0B28642F4DC06E000200C5C3C54F4
:1008A000401CC0B20D28F9D30E338B4202D1C8F8D8
:1008B00008C002E0491CC8F8081087F80D90CDE97F
:1008C00000EA2D4BCD210120FFF7B4FECEE7F0B5B5
:1008D00087B047F610664FF6FF770025CDE9017621
:1008E0002B462A462D21EF200095FFF7DDFE002044
:1008F000144C114A04AB61791E3A00EB010C12F85A
:100900000CC003F800C0401CC0B20A28F5D38DF813
:100910001A50CDE9007604AB002208210120FFF730
:1009200089FE6079192829D2401C607107B0F0BD9A
:10093000AC0123427C040020765D0308D6980308AE
:1009400036750308A4000020694E0308384E0308DA
:100950005C000020B8430308C0430308574E030857
:10096000F6020020F5020020348C0020408E04089E
:1009700025733A25732C0000D00A00206571D5E755
:10098000FEB5FE4E98254FF6FF743078002801D052
:10099000012808D1CDE9005408213C230022084653
:1009A0000294FFF781FE707808B1012808D1CDE9E3
:1009B000005408218C23002208460294FFF774FE9D
:1009C000B07808B101280BD1F078002808D1CDE922
:1009D00000540821DC23002208460294FFF764FE3D
:1009E000FEBD2DE9F04F85B00C4662420FFA82FB46
:1009F000E24A64250A264FF4847140F2E7374FF447
:100A00007A7A47F619694FF6FF78002807D0DFF8A1
:100A100070C301287ED0022841F02383FEE31078C2
:100A200058B1012877D0022876D0072875D004283D
:100A300074D0052873D001F014BB8DE80203372170
:100A40000A23D04A0846FFF713FE002C7FDB274617
:100A5000F520CDE90009202300220F210520CDF843
:100A60000890FFF721FE544534DB97FBF6F007B200
:100A7000642F0BDB97FBF5F03030C3B20021C822A6
:100A80000846CDE90089FFF768FD07E00021202333
:100A9000C8220846CDE90089FFF75FFD97FBF5F016
:100AA00005FB107090FBF6F03030C3B20021A0229D
:100AB0000846CDE90089FFF750FD97FBF6F006FBED
:100AC00010703030C3B2002168220846CDE9008999
:100AD000FFF743FD544539DA642C0BDB97FBF5F047
:100AE0003030C3B20021C8220846CDE90089FFF7A3
:100AF00034FD07E000212023C8220846CDE9008903
:100B0000FFF72BFD97FBF5F005FB107090FBF6F05F
:100B1000303006E09AE289E007E1A6E130E282E2C5
:100B200015E0C3B20021A0220846CDE90089FFF7F5
:100B300014FD97FBF6F006FB10703030C3B20021B5
:100B400068220846CDE90089FFF707FD59E0F52046
:100B5000CDE90008202300220A210320CDF80880D7
:100B6000FFF7A2FDBBF1640F27DB9BFBF5F03030F4
:100B7000C3B20021C8220846CDE90089FFF7EDFC89
:100B80009BFBF5F005FB10B090FBF6F03030C3B2E4
:100B90000021A0220846CDE90089FFF7DEFC9BFB7F
:100BA000F6F006FB10B03030C3B2002168220846D0
:100BB000CDE90089FFF7D1FC23E000212023C822E2
:100BC0000846CDE90089FFF7C8FC9BFBF5F005FB63
:100BD00010B090FBF6F03030C3B20021A0220846DE
:100BE000CDE90089FFF7B9FC9BFBF6F006FB10B0DE
:100BF0003030C3B2002168220846CDE90089FFF7F2
:100C0000ACFC6148007840B160A341222121012061
:100C1000CDE90089FFF70EFD0DE75DA342222121FA
:100C20000120CDE90089FFF705FD04E78DE8020307
:100C300037210A23574A0846FFF71AFD002CEBDB41
:100C40002746544534DB97FBF6F007B2642F0BDBE5
:100C500097FBF5F03030C3B20021C8220846CDE939
:100C60000089FFF77AFC07E000212023C82208460C
:100C7000CDE90089FFF771FC97FBF5F005FB1070DB
:100C800090FBF6F03030C3B20021A0220846CDE937
:100C90000089FFF762FC97FBF6F006FB107030301E
:100CA000C3B2002168220846CDE90089FFF755FC50
:100CB000544531DA642C0BDB97FBF5F03030C3B2CE
:100CC0000021C8220846CDE90089FFF746FC07E06D
:100CD00000212023C8220846CDE90089FFF73DFC0A
:100CE00097FBF5F005FB107090FBF6F03030C3B2C7
:100CF0000021A0220846CDE90089FFF72EFC97FBD2
:100D0000F6F006FB10703030C3B2002168220846AE
:100D1000CDE90089FFF721FC1FA3422221210120F8
:100D2000CDE90089FFF786FC85E68DE802033721CF
:100D30000A231A4A0846FFF79BFC42F210708442CD
:100D400000DB441E002CEFDB544549DB94FBFAF03A
:100D50003030C3B20021CD220846CDE90089FFF72B
:100D6000FCFB94FBFAF00AFB104090FBF5F03030EE
:100D7000A722C3B20021084612E00000A400002010
:100D8000888D0020DA20040854030020462000004B
:100D9000432000007C380408252020001EAB0308F7
:100DA000CDE90089FFF7D9FB94FBF5F005FB104076
:100DB00090FBF6F03030C3B2002181220846CDE925
:100DC0000089FFF7CAFB94FBF6F006FB10403030B9
:100DD000C3B200215B220846CDE90089FFF7BDFBC5
:100DE000544539DA00212023CD220846CDE9008977
:100DF000FFF7B3FB642C0BDB94FBF5F03030C3B290
:100E00000021A7220846CDE90089FFF7A6FB07E0ED
:100E100000212023A7220846CDE90089FFF79DFB8A
:100E200094FBF5F105FB114090FBF6F03030C3B2B6
:100E3000002181220846CDE90089FFF78EFB94FB53
:100E4000F6F106FB11403030C3B200215B220846A8
:100E5000CDE90089FFF781FBFBA33E222121012080
:100E6000CDE90089FFF7E6FBE5E58DE802033721D0
:100E70000A23F64A0846FFF7FBFB544500DB3C46D5
:100E8000002CF1DB54453CDA642C0BDB94FBF5F0D1
:100E90003030C3B20021D3220846CDE90089FFF7E4
:100EA0005CFB07E000212023D3220846CDE900891E
:100EB000FFF753FB0A2C0FDB94FBF5F105FB114008
:100EC00090FBF6F03030C3B20021AB220846CDE9EA
:100ED0000089FFF742FB07E000212023AB220846F0
:100EE000CDE90089FFF739FB94FBF6F106FB1140D1
:100EF0003030C3B2002183220846CDE90089FFF7D4
:100F00002CFBD348007B0628AED2DFE800F0030CB0
:100F1000151E2730CFA3662221210120CDE90089AB
:100F2000FFF788FB87E5CDA3662221210120CDE9CB
:100F30000089FFF77FFB7EE5CAA3662221210120FD
:100F4000CDE90089FFF776FB75E5C8A3662221216C
:100F50000120CDE90089FFF76DFB6CE5C5A3662292
:100F600021210120CDE90089FFF764FB63E5C3A3DC
:100F7000662221210120CDE90089FFF75BFB5AE5BC
:100F80008DE8020337210A23BE4A0846FFF770FBAB
:100F9000BDA3662221210120CDE90089FFF74AFB8C
:100FA000544500DB3C465445BCDA642C0BDB94FB17
:100FB000F5F03030C3B20021D3220846CDE90089D4
:100FC000FFF7CBFA07E000212023D3220846CDE922
:100FD0000089FFF7C2FA0A2C0FDB94FBF5F105FB41
:100FE000114090FBF6F03030C3B20021AB2208462E
:100FF000CDE90089FFF7B1FA07E000212023AB22F9
:101000000846CDE90089FFF7A8FA94FBF6F106FB44
:1010100011403030C3B2002183220846CDE9008957
:10102000FFF79BFA07E540F203108DE80103372133
:101030001423974A0846FFF71BFB96A3E2222121BF
:101040000120CDE90089FFF7F5FAF4E45078012892
:1010500009D088B302287CD004287BD006287AD017
:10106000052879D0E7E48DE8020337215A238C4A1A
:101070000846FFF7FDFA002CD4DB2746F020CDE927
:101080000009752300220F210520CDF80890FFF7F5
:101090000BFB544535DB97FBF6F007B2642F0CDBF6
:1010A00097FBF5F03030C3B2C82250210020CDE9C3
:1010B0000089FFF752FA08E066E02023C822502199
:1010C0000020CDE90089FFF748FA97FBF5F005FB12
:1010D000107090FBF6F03030C3B2A02250210020F7
:1010E000CDE90089FFF739FA97FBF6F006FB10709F
:1010F0003030C3B2682250210020CDE90089FFF7CB
:101100002CFA544536DA642C0BDB97FBF5F03030C3
:10111000C3B2C82250210020CDE90089FFF71DFA93
:1011200007E02023C82250210020CDE90089FFF7E5
:1011300014FA97FBF5F005FB107090FBF6F03030D9
:10114000C3B2A02250210020CDE90089FFF705FAA3
:1011500003E03DE1C9E11CE26FE297FBF6F006FB1C
:1011600010703030C3B2682250210020CDE90089D0
:10117000FFF7F3F9AFF2E033422271210120CDE90C
:101180000089FFF757FA56E48DE8020337215A2306
:10119000444A0846FFF76CFA002C54DB2746F5203A
:1011A000CDE90009752300220F210520CDF8089014
:1011B000FFF77AFA544536DB97FBF6F007B2642F57
:1011C0000BDB97FBF5F03030C3B2C8225021002072
:1011D000CDE90089FFF7C1F907E02023C82250219B
:1011E0000020CDE90089FFF7B8F997FBF5F005FB82
:1011F000107090FBF6F03030C3B2A02250210020D6
:10120000CDE90089FFF7A9F997FBF6F006FB10700E
:101210003030C3B268225021002000E02DE2CDE939
:101220000089FFF79AF9544562DA642C3CDB97FB9E
:10123000F5F03030C3B2C82250210020CDE900893A
:10124000FFF78BF938E054E070706D00380904083E
:10125000AE8E002020476F6F6400000020204D6F8D
:101260006400000020536F536F00000020506F6F28
:10127000720000002020426164000000416C617235
:101280006D00000052C2030875672F6D3300000027
:1012900096F1030850726573737572653A00000029
:1012A0007C380408DA2004082023C82250210020BA
:1012B000CDE90089FFF751F997FBF5F005FB1070B8
:1012C00090FBF6F03030C3B2A02250210020CDE9CF
:1012D0000089FFF742F997FBF6F006FB10703030FB
:1012E000C3B2682250210020CDE90089FFF735F90B
:1012F00059E0F520CDE90008702300220A210320DF
:10130000CDF80880FFF7D0F9BBF1640F27DB9BFB1A
:10131000F5F03030C3B2C82250210020CDE9008959
:10132000FFF71BF99BFBF5F005FB10B090FBF6F007
:101330003030C3B2A02250210020CDE90089FFF750
:101340000CF99BFBF6F006FB10B03030C3B26822FC
:1013500050210020CDE90089FFF7FFF823E020238A
:10136000C82250210020CDE90089FFF7F6F89BFB49
:10137000F5F005FB10B090FBF6F03030C3B2A022C0
:1013800050210020CDE90089FFF7E7F89BFBF6F03C
:1013900006FB10B03030C3B2682250210020CDE9E6
:1013A0000089FFF7DAF8FB48007840B1FAA3412240
:1013B00071210120CDE90089FFF73CF92CE4F7A366
:1013C000422271210120CDE90089FFF733F923E49E
:1013D00042F21070844200DB441E8DE80203372184
:1013E0005A23EF4A0846FFF743F9002CE6DB544541
:1013F00035DB94FBFAF03030C3B2CD22502100200F
:10140000CDE90089FFF7A9F894FBFAF00AFB104038
:1014100090FBF5F03030C3B2A72250210020CDE977
:101420000089FFF79AF894FBF5F005FB104090FB5C
:10143000F6F03030C3B2812250210020CDE900897E
:10144000FFF78BF894FBF6F006FB10403030C3B288
:101450005B2250210020CDE90089FFF77EF854453A
:1014600039DA2023CD2250210020CDE90089FFF771
:1014700074F8642C0BDB94FBF5F03030C3B2A72278
:1014800050210020CDE90089FFF767F807E020230D
:10149000A72250210020CDE90089FFF75EF894FBD8
:1014A000F5F105FB114090FBF6F03030C3B281221C
:1014B00050210020CDE90089FFF74FF894FBF6F1A9
:1014C00006FB11403030C3B25B2250210020CDE931
:1014D0000089FFF742F8AFF290233E2271210120EC
:1014E000CDE90089FFF7A6F81EE48DE80203372155
:1014F0005A23AC4A0846FFF7BBF8AFF274236622C2
:1015000071210120CDE90089FFF794F8544500DBF3
:101510003C465445E8DA642C0BDB94FBF5F03030A4
:10152000C3B2D32250210020CDE90089FFF715F87E
:1015300007E02023D32250210020CDE90089FFF7C6
:101540000CF80A2C0FDB94FBF5F105FB114090FB26
:10155000F6F03030C3B2AB2250210020CDE9008933
:10156000FEF7FBFF07E02023AB2250210020CDE94E
:101570000089FEF7F2FF94FBF6F106FB11403030D4
:10158000C3B2832250210020CDE90089FEF7E5FF98
:101590006AE48DE8020337215A23834A0846FFF79D
:1015A00067F8AFF21C33662271210120CDE9008972
:1015B000FFF740F8544500DB3C46544594DA642C70
:1015C0000BDB94FBF5F03030C3B2D3225021002066
:1015D000CDE90089FEF7C1FF07E02023D322502187
:1015E0000020CDE90089FEF7B8FF0A2C0FDB94FB41
:1015F000F5F105FB114090FBF6F03030C3B2AB22A1
:1016000050210020CDE90089FEF7A7FF07E0202345
:10161000AB2250210020CDE90089FEF79EFF94FB0C
:10162000F6F106FB11403030C3B283225021002076
:10163000CDE90089FEF791FF1AE29CF883004FF490
:101640008072012807D0594B50210020CDE9008934
:10165000FEF7F0FF0CE256A3154650210020CDE91D
:101660000089FEF7E7FF0020CDE9000953A32A46D1
:101670006E210120FEF7DEFFFAE1534893784FF424
:101680008E72C078022B09D0F3B3012B7DD0052BCD
:101690007CD0062B7BD0082B7AD0E9E142F2107384
:1016A0009C4200DB5C1E002CC6DB70B30120049062
:1016B0009E20039068274FF0140B44A39E21012025
:1016C000CDE90089FEF7B6FFAFF284433E229E21AA
:1016D0000120CDE90089FEF7ADFF54453CDB94FBCA
:1016E000FAF03030C3B20BEB4B00C219CDE90089E0
:1016F000DDE90310FEF731FF94FBFAF00AFB10401E
:1017000090FBF5F0303001E0A7E066E0C3B2CDE930
:101710000089DDE9031007EB4B02FEF71EFF94FB87
:10172000F5F005FB104090FBF6F03030C3B2CDE988
:101730000089DDE9031007EB0B02FEF70EFF94FBB7
:10174000F6F006FB10403030C3B2CDE90089DDE988
:1017500003103A46FEF701FF54458DDA0BEB4B00C0
:10176000C219CDE90089DDE903102023FEF7F5FE5B
:10177000642C4BDB94FBF5F03030C3B2CDE900892B
:10178000DDE9031007EB4B0224E05BE263E375E362
:10179000C8E300005403002046202000432020001E
:1017A0001EAB030852C20308F4D90308288D002099
:1017B0002020202020202020000000004F55542011
:1017C00052414E4745210000A4000020434F323AC9
:1017D00000000000FEF7C1FE21E08DE80203372182
:1017E000AA23FD4A0846FEF743FF00200490A020EC
:1017F00003905B274FF0260BAFF2B4533E22BF217C
:101800000120CDE90089FEF715FF66E7CDE90089E3
:10181000DDE9031007EB4B022023FEF79EFE94FB4D
:10182000F5F105FB114090FBF6F03030C3B2CDE985
:101830000089DDE9031007EB0B02FEF78EFE94FB37
:10184000F6F106FB11403030C3B2CDE90089DDE985
:1018500003103A46FEF781FE0AE12746E0B1012077
:101860000490DEA39E21CDE90089FEF7E3FE002C63
:101870007DDB54457CDB97FBF6F007B2642F78DB09
:1018800097FBF5F03030C3B2A4229E21CDE9008948
:101890000498FEF762FEFEE08DE802033721AA23DA
:1018A000D04A0846FEF7E4FEA0200390002C70DB2F
:1018B000544534DB97FBF6F007B2642F0BDB97FB44
:1018C000F5F03030C3B2C822CDE900890020039979
:1018D000FEF743FE07E02023C822CDE9008900205F
:1018E0000399FEF73AFE97FBF5F005FB107090FBAD
:1018F000F6F03030C3B2A022CDE900890020039970
:10190000FEF72BFE97FBF6F006FB10703030C3B2EB
:101910006822CDE9008900200399FEF71EFE544598
:1019200035DA642C0BDB97FBF5F03030C3B2C822FC
:10193000CDE9008900200399FEF70FFE07E0202380
:10194000C822CDE9008900200399FEF706FE97FB27
:10195000F5F005FB107090FBF6F03030C3B2A0221A
:10196000CDE9008900200399FEF7F7FD02E0E3E0EE
:10197000ADE088E097FBF6F006FB10703030C3B2A4
:101980006822CDE9008900200399FEF7E6FD5AE0C0
:10199000FFE7F020CDE90008202300220A210320E0
:1019A000CDF80880FEF780FEBBF1640F27DB9BFBC0
:1019B000F5F03030C3B2C822CDE900890020039988
:1019C000FEF7CBFD9BFBF5F005FB10B090FBF6F0AE
:1019D0003030C3B2A022CDE9008900200399FEF780
:1019E000BCFD9BFBF6F006FB10B03030C3B26822A2
:1019F000CDE9008900200399FEF7AFFD23E0202305
:101A0000C822CDE9008900200399FEF7A6FD9BFBC3
:101A1000F5F005FB10B090FBF6F03030C3B2A02219
:101A2000CDE9008900200399FEF797FD9BFBF6F0B6
:101A300006FB10B03030C3B26822CDE90089002027
:101A40000399FEF78AFD56208DE801030E21BE237F
:101A5000654A0846FEF70CFE6448007848B1AFF2CC
:101A6000C8234122C1210120CDE90089FEF7E2FD12
:101A7000F7E2AFF2D8234222C1210120CDE900894B
:101A8000FEF7D8FDEDE22023A4229E21CDE90089B6
:101A90000498FEF762FD97FBF5F005FB107090FBD4
:101AA000F6F03030C3B290229E21CDE9008904982F
:101AB000FEF753FD97FBF6F006FB10703030C3B213
:101AC00086229E21CDE900890498FEF746FD544503
:101AD00031DA642C0BDB97FBF5F03030C3B29A227D
:101AE0009E210120CDE90089FEF737FD07E0202384
:101AF0009A229E210120CDE90089FEF72EFD97FB59
:101B0000F5F005FB107090FBF6F03030C3B2862282
:101B10009E210120CDE90089FEF71FFD97FBF6F01D
:101B200006FB10703030C3B25E229E210120CDE949
:101B30000089FEF712FD66E0F020CDE900088D2354
:101B400000220A210320CDF80880FEF7ADFDBBF18D
:101B5000640F27DB9BFBF5F03030C3B29A229E2145
:101B60000120CDE90089FEF7F8FC9BFBF5F005FBB1
:101B700010B090FBF6F03030C3B286229E210120D7
:101B8000CDE90089FEF7E9FC9BFBF6F006FB10B0FF
:101B90003030C3B25E229E210120CDE90089FEF7DC
:101BA000DCFC30E020239A229E210120CDE900892F
:101BB000FEF7D3FC9BFBF5F005FB10B090FBF6F0B5
:101BC0003030C3B286229E210120CDE90089FEF784
:101BD000C4FC9BFBF6F00BE01EAB030854454D50D4
:101BE0003A000000DA2004081E50040854030020C4
:101BF00006FB10B03030C3B25E229E210120CDE939
:101C00000089FEF7AAFC2E2374229E210220CDE932
:101C10000089FEF7A2FCFB48007848B1AFF2884388
:101C20003E229E210120CDE90089FEF703FD18E246
:101C3000AFF298433E229E210120CDE90089FEF7B4
:101C4000F9FC0EE2002CF2DB2746C8B1EEA39E2180
:101C50000120CDE90089FEF7EDFC54457EDB97FBC2
:101C6000F6F007B2642F7ADB97FBF5F03030C3B2A1
:101C70009A229E210120CDE90089FEF76EFC89E0C1
:101C80008DE802033721AA23E14A0846FEF7F0FC5B
:101C90004FF0A00B544534DB97FBF6F007B2642FEE
:101CA0000BDB97FBF5F03030C3B2C8225946002059
:101CB000CDE90089FEF751FC07E02023C8225946F0
:101CC0000020CDE90089FEF748FC97FBF5F005FB05
:101CD000107090FBF6F03030C3B2A02259460020BD
:101CE000CDE90089FEF739FC97FBF6F006FB107092
:101CF0003030C3B2682259460020CDE90089FEF792
:101D00002CFC544534DA642C0BDB97FBF5F03030B7
:101D1000C3B2C82259460020CDE90089FEF71DFC58
:101D200007E02023C82259460020CDE90089FEF7AC
:101D300014FC97FBF5F005FB107090FBF6F03030CB
:101D4000C3B2A02259460020CDE90089FEF705FC68
:101D500097FBF6F006FB1070303001E036E011E042
:101D6000C3B2682259460020CDE90089FEF7F5FB91
:101D7000AFF6DC734222C1210120CDE90089FEF7D4
:101D800059FC6EE120239A229E210120CDE9008991
:101D9000FEF7E3FB97FBF5F005FB107090FBF6F008
:101DA0003030C3B286229E210120CDE90089FEF7A2
:101DB000D4FB97FBF6F006FB10703030C3B25E2206
:101DC0009E210120CDE90089FEF7C7FB544531DA99
:101DD000642C0BDB97FBF5F03030C3B29A229E21C6
:101DE0000120CDE90089FEF7B8FB07E020239A2205
:101DF0009E210120CDE90089FEF7AFFB97FBF5F0AE
:101E000005FB107090FBF6F03030C3B286229E21A5
:101E10000120CDE90089FEF7A0FB97FBF6F006FB59
:101E200010703030C3B25E229E210120CDE90089BE
:101E3000FEF793FB2E2374229E210220CDE9008918
:101E4000FEF78BFB734B3E229E210120CDE90089DA
:101E5000FEF7F0FB05E19CF803006F4900EB400042
:101E600001EB40016D481FF07FFC6C4B68229E2106
:101E70000120CDE90089FEF7DDFBF2E08DE80203E9
:101E80003721AA23664A0846FEF7F2FB544500DBD9
:101E90003C4654453CDA642C0BDB94FBF5F03030C7
:101EA000C3B2D322A0210020CDE90089FEF755FB63
:101EB00007E02023D322A0210020CDE90089FEF7EE
:101EC0004CFB0A2C0FDB94FBF5F105FB114090FB5A
:101ED000F6F03030C3B2AB22A0210020CDE900895A
:101EE000FEF73BFB07E02023AB22A0210020CDE939
:101EF0000089FEF732FB94FBF6F106FB114030300F
:101F0000C3B28322A0210020CDE90089FEF725FB82
:101F1000AFF68C436622C1210120CDE90089FEF78E
:101F200089FB9EE042F21070844200DB441E002CCC
:101F30003FDB002004904FF0A00B5B2739A33E222B
:101F4000BF210120CDE90089FEF774FB544530DA4A
:101F5000CD2220235946CDE900890498FEF7FDFAE9
:101F6000642C27DB94FBF5F03030C3B2A72259462E
:101F7000CDE900890498FEF7F0FA94FBF5F105FB32
:101F8000114090FBF6F03030C3B281225946CDE9C2
:101F900000890498FEF7E1FA94FBF6F106FB114084
:101FA0003030C3B23A465946CDE900890498FEF76D
:101FB000D4FA56E00A2C37DBA72220235946CDE974
:101FC00000890498FEF7C9FA94FBF5F105FB11406E
:101FD00090FBF6F03030C3B281225946CDE900893A
:101FE0000498FEF7BAFA94FBF6F106FB1140303084
:101FF000C3B23A465946CDE900890498FEF7ADFAD6
:102000002FE000005403002048554D3A0000000026
:102010007C380408980D010850910408288D002090
:10202000F4D903084C757800A72220235946CDE93E
:1020300000890498FEF791FA812220235946CDE9C0
:1020400000890498FEF789FA94FBF6F106FB11402B
:102050003030C3B23A465946CDE900890498FEF7BC
:102060007CFA544503DD0020FEF78AFC02E00120E3
:10207000FEF786FC2649887902280FD005283CD037
:1020800006283AD000208DE8010303461A21214A90
:102090000846FEF7EDFA05B0BDE8F08F087A46284D
:1020A00009D200208DE8010303461A211A4A084686
:1020B000FEF7DEFAEFE7502809D200208DE8010391
:1020C00003461A21154A0846FEF7D2FAE3E75A28D2
:1020D00009D200208DE8010303461A21104A084660
:1020E000FEF7C6FAD7E700208DE8010303461A2160
:1020F0000C4A0846FEF7BCFACDE700208DE8010344
:1021000003461A21084A0846FEF7B2FAC3E7000060
:10211000B89A0020EE560408A65104080E6C040874
:10212000C66604087E610408365C040870B50024A5
:10213000F74D04EB840005EB800000F061FC641CAB
:10214000062CF6D3F248783000F05AFCF0488C3078
:1021500000F056FCEE48A03000F052FCEC48B430E1
:1021600000F04EFCEA48C83000F04AFCE849E94873
:10217000783141631431816370BD70B504461546F2
:10218000102204F134001FF0ADFA002084F843005F
:10219000062D00D30525E5626564201D00F03BFC9B
:1021A00004F1180000F037FC2461C5F10600A061BD
:1021B000646270BD70B506460D46482000F02EFFE3
:1021C000044644B1B60045B12846206348B1A52273
:1021D00031461FF057FA204670BD304600F01EFF12
:1021E000F3E7204600F070FF0024F4E72DE9FF4FED
:1021F00081B08246DDE90E68109917469B46384645
:10220000FFF7D8FF0446C34DECB3216B781E01EBFA
:10221000800020F00709009732462046119B029962
:10222000FFF7ABFF5A465146484600F09BFE206040
:10223000B8F1000F01D0C8F8004000F0BEFEA86859
:10224000401CA860286810B1A86938B10BE02C6068
:10225000A868012807D1FFF769FF04E02868C06A71
:10226000B04200D82C60E06A2969884200D9286110
:10227000E96A491CE9626969884200D9686100EB32
:102280008001A34800E008E000EB8100211D00F080
:10229000C5FB012400F099FE01E04FF0FF34012C52
:1022A00007D1A86928B12868C06AB04201D200F0FD
:1022B0007EFE05B02046BDE8F08F70B5054600F003
:1022C0007CFE944E3068854200D10025FDB12C463D
:1022D000201D00F0C9FBA06A18B104F1180000F03D
:1022E000C3FB8B48211DB43000F098FB7068401C84
:1022F0007060F06A401CF06200F067FEB069002870
:1023000007D0002D05D1BDE8704000F050BE346804
:10231000DEE770BD70B57F4DE869002803D0286AFC
:10232000401C286270BDE868401CE860E8684FF017
:10233000FF3670B9686BA96B6963A863A86A401C13
:10234000A862686B0068A0B1686BC068C06840682C
:102350002863E868296B8842E4D3686B006850B151
:10236000686BC068C4686068E968814205D2286308
:1023700070BD2E63EDE72E6370BD201D00F074FB71
:10238000A06A18B104F1180000F06EFBE06A6969F8
:10239000884200D968615E4900EB800001EB800053
:1023A000211D00F03BFBD8E72DE9F041002700F0AC
:1023B00004FE584EF069401EF061F069E8BBB06859
:1023C000D8B30025DFF8488108F1A0081CE0D8F850
:1023D0000C00C46804F1180000F046FB201D00F05A
:1023E00043FBE06A7169884200D97061484900EB9B
:1023F000800001EB8000211D00F010FBE06A3168D5
:10240000C96A884200D30125D8F800000028DED12F
:10241000306A28B908E0FFF77DFF306A401E30625D
:10242000306A0028F7D10125012D02D0706A0128F9
:1024300006D101270020706200E001E000F0B7FD46
:1024400000F0C3FD3846BDE8F08170B50446314D5B
:1024500028684460E868844206D22968A86B091D90
:10246000BDE8704000F0E8BA2968686B091D00F00B
:10247000E3FA286B844200D22C6370BD2548C16901
:10248000491CC161704770B503460C460022FFF736
:10249000F5FF186804441F49CD68A84206D9A04238
:1024A0000AD9C868844207D9012205E0A04202D8AF
:1024B000C868844200D901221C6032B10868001D3E
:1024C00000F0D2FA2046FFF7C0FFFFF76DFF0028AB
:1024D00003D1BDE8704000F06ABD70BD10B5024682
:1024E0000020002A0DD0FFF7C9FF0A48C1688C18E8
:1024F0000068001D00F0B8FA2046FFF7A6FFFFF7BE
:1025000053FF002803D1BDE8104000F050BD10BDBE
:10251000E00A0020F401002010B5044600F04DFD53
:102520000CB9F7480468E46A00F04FFD2046EEE776
:102530002DE9F04106460D460027062D00D305255E
:1025400000F03BFDDFF8B883D8F80000864200D1E8
:10255000002646B13446606CA8422ED0854205D98B
:1025600036B1012704E0D8F80040F4E706B90127A6
:10257000E26A904200D1E5626564C5F10601A1619D
:10258000E04D00EB8000616905EB8000814210D1D5
:10259000201D00F069FAE06AD8F81410884201D9C9
:1025A000C8F8140000EB800005EB8000211D00F04E
:1025B00035FA012F01D100F0FAFCBDE8F04100F03E
:1025C00004BDCF49C869002802D001204862704785
:1025D000CC4A02E04869401E4861486900EB80002F
:1025E00052F820000028F5D0486900EB800002EB8B
:1025F000800042685268426000F108039A4201D1AB
:10260000526842604068C0680860704770B505460F
:1026100000F0D3FCBA4E3068854200D10025C5B128
:102620002C46201D00F020FAA06A18B104F1180011
:1026300000F01AFAB348211DC83000F0EFF900F09D
:10264000C4FC002D0FD1B06928B1BDE8704000F086
:10265000AEBC3468E5E7AB48C8300068B168884272
:1026600002D10020306070BDBDE87040A9E70021B4
:10267000A44B4269C8339A4206D1806AA3F128026A
:10268000904201D000B901210846704770B5044658
:10269000002C25D09A4D2868844221D000F08DFC72
:1026A0002046FFF7E4FF012816D1201D00F0DCF9D9
:1026B000E06A6969884200D96861924900EB80004C
:1026C00001EB8000211D00F0A9F9E06A2968C96AC0
:1026D000884201D300F06BFCBDE8704000F075BC8F
:1026E00070BD70B5044600252046FFF7C0FF0128E5
:1026F00008D1834EF06938B1824804F11801A03046
:1027000000F08CF9284670BDE06A3168C96A8842D9
:1027100001D3012500E00025201D00F0A5F9E06AA5
:102720007169884200D97061764900EB800001EB45
:102730008000211D00F072F9E4E710B50446206B1B
:1027400000F0C2FC2046BDE8104000F0BDBC70B5F2
:102750006B4D686800281FD0FFF790FE694EB436B5
:102760003068B8B10024FFF71FFE002C14D100F030
:1027700024FCF068C468201D00F076F9A868401EAB
:10278000A8606868401E686000F01FFC2046BDE835
:102790007040D2E70124E6E770BD5A4CFFF7D7FF3F
:1027A00020680128FAD900F002FCF7E71FB50024E1
:1027B0000094019402942346802253A15448039428
:1027C000FFF714FD012809D1F5F7F8FC4C48012169
:1027D0008161C460BDE81F4000F0D5BB1FBD10B5CE
:1027E000F5F7ECFC464900208861BDE8104000F098
:1027F000DDBB10B500F0E1FB4148C46800F0E5FB2B
:10280000204684E610B5F5F7D9FC3D48C468F5F7D5
:10281000DCFC20467BE63A488068704770B50D4680
:10282000374C2168183100F007F92068001D00F0CE
:102830001BF9681C04D0E0682844BDE8704004E639
:102840002168BDE870402F48091DC83000F0E6B887
:1028500070B5C068C46804F11800064600F004F9B9
:10286000274DEA695AB127483146A03000F0D6F822
:10287000E06A2968C96A884212D3012070BD201D10
:1028800000F0F2F8E06A6969884200D968611D4980
:1028900000EB800001EB8000211D00F0BFF8E7E7AE
:1028A000002070BD16498A6A0260C968416070479D
:1028B00070B504460D4600F080FB2868411C0AD024
:1028C0000F4B21689A6A914207D06168DA68914299
:1028D00003D8012410E000240EE06268D968891A48
:1028E000814208D2D968891A401A28602046FFF729
:1028F000D9FF002400E0012400F067FB204670BDF2
:10290000F4010020E00A002049444C45000000008A
:102910009B2701083849012048627047002102E0E6
:10292000401C491C89B20278A52AF9D08808704752
:10293000002801D130480068006BEFE72E4800689E
:1029400070472D488169002903D0C06918B1022061
:102950007047002070470120704770B50446264D2F
:10296000E06A2968C96A8842C9D22868C06AC0F189
:102970000600A061E06A214E00EB8000616906EB71
:102980008000814212D1201D00F06EF82868C06AD4
:10299000E0626969884200D9686100EB800006EB5B
:1029A0008000211DBDE8704000F038B82868C06A7A
:1029B000E062A4E710B5044600281BD0616CE06A11
:1029C000884217D0201D00F04FF8606CE062C0F123
:1029D0000600A0610849E06A4A69904200D948614E
:1029E000064900EB800001EB8000211DBDE810408E
:1029F00000F014B88BE50000F4010020E00A00208C
:102A000000F1080141604FF0FF328260C160016156
:102A100000210160704700210161704742685368DE
:102A20004B6043688B6053689960516041600861F6
:102A30000168491C0160704710B50B685A1C02D030
:102A400000F1080202E0026904E052685468246858
:102A50009C42FAD953684B6099608A605160086162
:102A60000168491C016010BDD0E901219160D0E9E5
:102A70000112516001694A68824201D182684A604C
:102A8000002202610868401E086070472DE9F0418D
:102A900005460E460027002D28D04C2000F0BEFA37
:102AA0000446200022D005FB06F0401C00F0B6FAD8
:102AB0002060C0B105FB060161600021A163A06038
:102AC000691E01FB0600E060E5632664781E606411
:102AD000A06404F11000FFF793FF04F12400FFF756
:102AE0008FFF274602E0204600F0EEFA3846BDE8A8
:102AF000F08170B5044600F060FA04F124050AE0A4
:102B0000606A58B12846FFF7A3FE08B1FFF702FF3D
:102B1000A06C401EA064A06C0028F1DC4FF0FF35D3
:102B2000A56400F052FA00F048FA04F110060AE039
:102B3000206958B13046FFF78BFE08B1FFF7EAFE77
:102B4000606C401E6064606C0028F1DC6564BDE868
:102B5000704000F03ABA10B5044600F02EFAA06BAF
:102B6000E16B884201D1012400E0002400F02DFA3D
:102B7000204610BD10B504461046226C002A11D024
:102B8000C8B1E0681EF06CFDE168206C091AE160D4
:102B90002268914202D26168081AE060A06B401C72
:102BA000A06310BD20680028F8D16068FFF702FF1D
:102BB00000206060F2E7A0681EF052FD216CA06862
:102BC0000844A06061688842E8D32068A060E5E717
:102BD0002DE9FF4182B0044688461F4600250026A5
:102BE00000F0EBF9A06BE16B884213D23A46414604
:102BF0002046FFF7BFFF606A38B104F12400FFF7F9
:102C000027FE012801D100F0D2F900F0DEF9012001
:102C100006B06CE7049808B125B107E000F0D5F9DB
:102C20000020F5E76846FFF73DFE012500F0CDF9ED
:102C3000FFF724FC00F0C1F9606C401C00D1666411
:102C4000A06C401C00D1A66400F0BFF904A968463E
:102C5000FFF72EFE30B12046FFF74BFFFFF7A4FB36
:102C60000020D5E72046FFF776FF70B104F1100091
:102C70000499FFF7D3FD2046FFF73BFFFFF794FBD6
:102C80000028ADD100F093F9AAE72046FFF731FF05
:102C9000FFF78AFBA4E710B54C2000F0BFF904460B
:102CA000CCB1002060602060A060E060A0630121E2
:102CB000E1632064401E6064A06404F11000FFF72B
:102CC0009FFE04F12400FFF79BFE00231A461946DD
:102CD0002046FFF77DFF204610BD10B50446FFF7E4
:102CE0002DFE616888420BD1E068401EE06028B983
:102CF00000231A4619462046FFF76AFF012010BD3F
:102D0000002010BD10B5044600F057F9A06B20B1AB
:102D1000002400F05AF9204610BD0124F9E730B430
:102D20000C460368002B0CD0026CC1681144C160D2
:102D30004568A94200D3C360C168204630BC1EF07C
:102D40008FBC30BC70472DE9FF4383B004468946F1
:102D500098460025002604F1240700F02EF9A06B08
:102D600050B3E56849462046FFF7D9FFB8F1000F98
:102D70000ED0E560606A28B13846FFF769FD08B1FA
:102D800000F015F900F021F9012007B0BDE8F0834B
:102D9000A06B401EA063206810B9FFF7CFFD6060F4
:102DA00020690028EED004F11000FFF751FD012842
:102DB000E8D100F0FCF8E5E7059808B125B107E097
:102DC00000F003F90020E0E701A8FFF76BFD012503
:102DD00000F0FBF8FFF752FB00F0EFF8606C401CCE
:102DE00000D16664A06C401C00D1A66400F0EDF830
:102DF00005A901A8FFF75CFD30B12046FFF779FE79
:102E0000FFF7D2FA0020C0E72046FFF77BFFB0B102
:102E1000206830B900F0D1F86068FFF79EFD00F03F
:102E2000D4F838460599FFF7F9FC2046FFF761FE14
:102E3000FFF7BAFA002890D100F0B9F88DE72046E4
:102E4000FFF757FEFFF7B0FA87E770B504460D4667
:102E5000FFF774FD6368984204D1E068401CE060AD
:102E6000012070BD00232A4619462046FFF76BFF5C
:102E70000128F6D1E168491CE16070BD2DE9F041FF
:102E800004460F4615461E46F5F798F9A06BE26B0F
:102E9000904217D2324639462046FFF76BFEA06CAF
:102EA000411C03D0401CA06401240CE0606A00288F
:102EB000FAD004F12400FFF7CBFC0028F4D0012065
:102EC0002860F1E70024F5F780F920460FE670B599
:102ED00004460E461546F5F771F9A06BC8B13146A8
:102EE0002046FFF71CFFA06B401EA063606C411CD6
:102EF00003D0401C606401240CE020690028FAD053
:102F000004F11000FFF7A4FC0028F4D00120286091
:102F1000F1E70024F5F759F9204670BD10B50446D5
:102F200000F04BF8A46B00F050F8204610BD806B09
:102F3000704710B50446206800F0C6F82046BDE88A
:102F4000104000F0C1B8806B002801D0002070470D
:102F500001207047816BC06B814201D10120704715
:102F60000020704720384FF08073C36181610021D9
:102F7000416140F8202970474FF0E020234941612A
:102F800007210161704710B52148016841F47F01B4
:102F90000160016841F07F410160FFF7EDFF1D49CD
:102FA00000200860F5F7E2F8002010BD70471849CE
:102FB0004FF080501C390860704710B5F5F7FEF8E7
:102FC00014480168491C016010BD12490868401E80
:102FD0000860002801D1F5F7F8B8704710B50C4922
:102FE0004FF080501C390860F5F7E8F8FFF792F9C8
:102FF0000949087828B1401EC0B2087008B902F02B
:1030000037FBBDE81040F5F7E0B800003F190100BC
:1030100020ED00E030020020C40200202DE9F04144
:1030200004460025FFF72AFA384E06F108017068B9
:1030300001F1080360B936480860002048604FF489
:10304000B0425A60186032484260036001207060EC
:103050003CB11034600704D004F00700C0F1080050
:103060000444601E45F2FF72904228D2274A08327B
:10307000096801E00A4601464868A04202D2086891
:103080000028F7D199421AD01568103508681060E9
:103090004868001B20280ED90B1958604C605C68EA
:1030A0001A48083000E0104602685768A742FAD371
:1030B00002681A60036048683168081A3060FFF7D8
:1030C00073F92846BDE8F08110B5002818D01038F3
:1030D0000446FFF7D3F960680C49083100E0114657
:1030E0000A6853688342FAD3086820600C60074876
:1030F0006168026811440160BDE81040FFF754B9EF
:1031000010BD02480068704770470000340200207C
:10311000C00B00202DE9F04387B00646012144F2A0
:103120000400F7F7E6FBDFF840824046F8F74CFC76
:103130004FF40070ADF8180003258DF81A501820D0
:103140008DF81B00DFF8249206A94846F7F7ADF981
:103150004FF48067ADF8187004208DF81B0006A9A5
:103160004846F7F7A2F9BC10ADF8184010208DF8CA
:103170001B0006A94846F7F798F921464846F7F795
:1031800003FA25208DF8040000248DF805408DF801
:10319000065001208DF8070001A8F6F70EFE0296F2
:1031A000ADF80C40ADF80E407148B9000078012828
:1031B00019D002281ED0ADF81040ADF814400C20F4
:1031C000ADF8120002A94046F8F746FC012240F291
:1031D00025514046F8F7C7FC01214046F8F7B7FCF7
:1031E00007B0BDE8F0834FF4C060ADF81000ADF853
:1031F0000C10E2E7ADF81070ADF80C10DDE770B51B
:1032000086B0054601210820F7F7E0F901214804BE
:10321000F7F77AFB01212020F7F76BFB554E30467C
:10322000F8F7D2FB2020ADF8140003208DF816002B
:1032300018208DF81700504C05A92046F7F735F9EE
:103240004020ADF8140028208DF8170005A920466D
:10325000F7F72BF926208DF8000000248DF80140A7
:1032600001208DF802008DF803006846F6F7A5FDF1
:103270000195ADF80840ADF80A40ADF80C40ADF846
:1032800010400C20ADF80E0001A93046F8F7E4FB21
:10329000012240F225513046F8F765FC0121304605
:1032A000F8F755FC06B070BDF0B587B005460121B2
:1032B0008804F7F729FB01210920F7F71AFB2F4EA5
:1032C0003046F8F781FB3015ADF8180003208DF873
:1032D0001A0018208DF81B00294F06A93846F7F769
:1032E000E4F8F014ADF8180004208DF81B0006A9CE
:1032F0003846F7F7DAF87415ADF8184010208DF855
:103300001B0006A93846F7F7D0F821463846F7F7EC
:103310003BF927208DF8040000248DF80540022099
:103320008DF8060001208DF8070001A8F6F745FD8D
:103330000295ADF80C40ADF80E40ADF81040ADF878
:1033400014400C20ADF8120002A93046F8F784FBB7
:10335000012240F225513046F8F705FC01213046A4
:10336000F8F7F5FB07B0F0BD003801400008014058
:10337000C502002000440040001401400048004005
:10338000000C01404FF0E0210A6922F004020A61BA
:10339000224A1070C0084FF47A73584301235380B7
:1033A0004861086940F00100086170472DE9F0416B
:1033B00000244FF0E0277E69054618480078454311
:1033C000FFF7FBFDBA69B9699142FCD003D2A2EBC9
:1033D0000100044403E0A6EB0100104404440A4643
:1033E000AC42F0D3BDE8F041FFF7EFBD70B5044645
:1033F000FFF7A7FA60B1094D6888844203D3B4FB94
:10340000F0F0FFF76BF86888B4FBF0F100FB1144B3
:103410004FF47A706043BDE87040C7E74C0200206B
:1034200010B50446616001F00DFA206010BDD0E9CE
:10343000001211440160704710B5044601F002FA11
:10344000206010BD10B5044601F0FCF92168401A57
:103450006168884201DB012010BD002010BD000022
:10346000FE490881704730B5C278FC4D0A443035BA
:10347000D4B2EC70827802EB1122D2B2AA704378F7
:103480006B7000782870B2EB112F05D25B1CDBB299
:103490006B700BB9401C2870C8B284420DD2521C0C
:1034A000D0B2A870002808D16878401CC0B26870FB
:1034B000002802D12878401C287030BD10B58B1828
:1034C0005B1E0BE04A780C7802EB042292B21044A7
:1034D00080B2904201D2401C80B2891C9942F1D343
:1034E000994207D109780902084480B2884201D282
:1034F000401C80B210BD010241EA102080B270472A
:1035000010B50A4601460020FFF7D8FFBDE810407D
:10351000F1E710B51422D2490020FFF7CFFF10B118
:10352000BDE81040E7E74FF6FF7010BD10B5CC497D
:103530006FF013030E394A7C097C03EB012111441F
:103540008CB2204480B2C64908220C31FFF7B6FF86
:10355000C34922461431FFF7B1FF10B1BDE8104056
:10356000C9E74FF6FF7010BD0620DFE71120DDE749
:1035700010B5BA4A00215170BA4B507823F8101098
:10358000401CC0B250701428F7D35170B64B50781D
:1035900000EB800403EBC4046176401CC0B25070A1
:1035A0001428F4D34FF4806050815170AD4B283310
:1035B000507803EB8014A180401CC0B250700A28E0
:1035C000F6D310BD2DE9F04106460F46A64BA34C9D
:1035D0004FF4FA4800256089401C80B26081404564
:1035E00002D34FF4805060816570607800EB8000FA
:1035F00003EBC002507E28B16089FFF77CFF918801
:103600008842E8D06078401CC0B260701428ECD3C7
:1036100000226570617801EB810003EBC00090F837
:1036200019C0BCF1000F03D0BCF1070F02D009E0B4
:1036300002460CE02AB190F81AC092F81A80C445EC
:1036400000D90246491CC8B260701428E2D322B3E4
:103650000220507681482C300178117341785173E3
:1036600081789173C078D07340F2CA705082908292
:1036700001201082D5769076032010769575102063
:10368000D0756089FFF737FF9080D7803088108031
:10369000708850801046BDE8F0810020FBE72DE9DE
:1036A000F04104460F466F4B00256C4A4FF4FA4830
:1036B0004FF4805628335089401C80B250814045D9
:1036C00000D3568155705089FFF715FF0146507899
:1036D00003EB801CBCF804C06145ECD0401CC0B2B8
:1036E00050700A28EFD300205570517803EB8116F3
:1036F000B6889EB1491CC9B251700A29F5D388B168
:1037000051890A0242EA11218180C78064B121886F
:1037100001806188418040210172BCE7507803EB51
:103720008010ECE70020B6E70560F4E730B54B4ABF
:10373000002555704B4B517833F81140844203D12A
:10374000507823F8105030BD491CC9B2517014296B
:10375000F1D330BD10B5414A00215170414B517831
:1037600033F811402CB1491CC9B251701429F6D359
:1037700010BD517823F8110010BD10B5374C01462B
:10378000606A0830FFF76FFE04F13001606A0A7862
:1037900002724A7842728A788272C978C17210BD08
:1037A0002DE9FF5FDFF8B490D9F824402C4D0026B6
:1037B0000E3D05F136014FF6FF780391042869D0DC
:1037C0000399C9F81C10C9F820104FF0100A0328FB
:1037D00019D0022825D005F12A04052870D004F656
:1037E000A2577888401C78803846A97B0088401C06
:1037F00080B245297ED03880F888401CF8801BA014
:1038000001F0EEF8C7E0607E00F00F000328F9D168
:10381000208A0028F6D1082089F8000001F0D2F8AB
:10382000FEE30E492C31C878401C10F0FF00C87030
:103830000ED18878401C10F0FF00887008D14878BD
:10384000401C10F0FF00487002D10878401C08703E
:10385000A9F80460A9F80660607E1CE05802002008
:10386000CE630020E46E0020C46B002069703A2013
:10387000696E76616C69642076657273696F6E201B
:103880006F7220686561646572206C656E6774682C
:103890002E000000B2E1072813D0052811D000281F
:1038A000B0D0218A39B3A07E411EA176AAD2E07E93
:1038B00008282CD0617E02290BD0012909D00AE00A
:1038C00042E0A07E401CC0B2A07678289AD16676ED
:1038D00061E005281BD0042800D904200321814081
:1038E000A176E07E401CE076F648C18C491CC1847C
:1038F000607E01E03DE01DE000F00F000928E7D206
:10390000DFE800F049FD0F12FC49FC49FC00667637
:10391000802089F8000001F055F8142085F82F0068
:10392000ECE385F82F602CE3042089F8000001F017
:1039300049F8F7E300F00F000328C9D1082089F8FF
:10394000000001F03FF86BE3D9F8280080880028D8
:10395000BED0C9F82460C9F81C40C9F82040A9F8B5
:103960000660A9F80460082089F8000001F0A4FDB1
:1039700044E1697C2A7C01EB0221B9F804209142E0
:1039800006D8CB46A9F80410297D890606D103E0A4
:10399000CDA001F025F86DE1697D39B13880B88995
:1039A000401CB881D4A001F01BF863E1D849B1F8FC
:1039B00000E049880291BEF1000F01D10299C9B11E
:1039C000D44AEB7DD18B128C112B0CD1414501D106
:1039D000424569D0CE4B0833B3F800C0614502D1EF
:1039E0005B889A4260D0714502D102998A4201D027
:1039F00038803FE1FFF78DFD404509D03888401CF5
:103A00003880F889401CF881C3A000F0E9FF31E15B
:103A1000E87D06280DD0112846D001281AD0388814
:103A2000401C3880388A401C3882C0A000F0D8FF83
:103A300020E1B88B401CB883FFF796FD40457DD050
:103A4000788B401C7883388C401C3884BEA000F0F2
:103A5000C7FF0FE1B88A401CB88295F822000828F9
:103A600009D0788A401C7882388B401C3883BBA0F0
:103A700000F0B6FFFEE085F82260A88C4FF6F771E3
:103A8000884202D30930A88401E00830A884688BFA
:103A9000E883A88B28849E48018869834088A8838E
:103AA000F88A401CF882FDE3BBF804001C38ABF830
:103AB0000400CBF81C40288D50B1FFF757FD40455E
:103AC00006D0B88D401CB885788E401C7886D1E031
:103AD000A848CBF828007B4FC4E082887AB3A98C31
:103AE00091422CD1018809B943884BB3414502D199
:103AF000438843452BD06B8B8B4201E0BEE33EE213
:103B000003D1A98B4388994221D0E98B414502D149
:103B10002B8C43451BD0DFF8F8C1BCF8003099422C
:103B200004D12B8CBCF802C0634510D0DFF8E0C193
:103B30000CF1080CBCF80030994202E09EE07FE0F6
:103B400005E07DD1298CBCF80230994278D1DBF8B0
:103B50002810C98811B1B2F5884F42D0698CC18054
:103B6000698BADF80410AA8BADF80620DBF81220A3
:103B700000929DF800309DF80420C3F1FF031A4322
:103B80008DF804209DF801309DF80520C3F1FF0356
:103B90001A438DF805209DF802309DF80620C3F1E8
:103BA000FF031A438DF806209DF803309DF8072087
:103BB000C3F1FF031A438DF80720554ABDF80430BE
:103BC00008321788BB4204D1BDF8063052889342B0
:103BD00004D0A0F80080A0F8028002E00180A98B48
:103BE0004180CBF8246002208BF80000CBF81C4009
:103BF000CBF82040ABF8066001F05EFCB9F8061087
:103C0000002937D001F11C00A9F80400020A2A7427
:103C10006874D9F82800027AAA751122EA75083169
:103C2000C1F3072242EA0121E9842E858188698453
:103C3000C188A98436490A886A834988A98300E033
:103C40000DE00188E983408828840398C9F81C00A6
:103C5000FFF78CFCC04380B2288560B1FEE34030A2
:103C6000CBF82800DBF82800B842FFF436AF42A0BA
:103C700000F0B6FE8FE2A5F82880EFE3474CB5F8D8
:103C800022C0B5F81A80A98B04F53E73A88C91E088
:103C9000627EAAB1A288904212D1E28894450FD1E7
:103CA000228890450CD16288914209D1CBF82440FA
:103CB0008BF8006095F82F00410702D566766FE01B
:103CC00077E085E18C71002069703A207061636B48
:103CD00065742073686F72746572207468616E20F9
:103CE0007265706F7274656420696E204950206837
:103CF00065616465722E000069703A2066726167C2
:103D00006D656E742064726F707065642E000000C3
:103D100066020020C063002069703A20626164205E
:103D2000636865636B73756D2E0D0A0069703A20C8
:103D30006E65697468657220746370206E6F72209E
:103D400069636D702E0D0A007463703A20626164BD
:103D500020636865636B73756D2E000069636D7019
:103D60003A206E6F742069636D70206563686F2EF2
:103D70000D0A00000C6F00207564703A206E6F20F1
:103D80006D61746368696E6720636F6E6E656374DE
:103D9000696F6E20666F756E64000000C46B002052
:103DA000FDA000F01DFE20208BF8000000F00AFEB0
:103DB00073E328349C427FF66BAF95F82F1001F027
:103DC0003F01022918D1ABF80C008BF80160FC4AC6
:103DD0009BF8011032F81130834204D100248BF893
:103DE0000160F84B4EE0491CC9B28BF80110142950
:103DF000EED3788D401C788595F82F004007D7D4F6
:103E0000B88C401CB8841420263568722820ABF882
:103E1000040050202872EB78E879E870A978A87936
:103E2000A870A9716A78687968706A7128788BF8C7
:103E300001002C792C7028715B1C13F0FF03EB71CF
:103E4000A5F126050ED1491C11F0FF0185F82C10B3
:103E500008D1521C12F0FF0185F82B1002D1401C32
:103E600085F82A00688CABF80C00A98C6984A884BA
:103E7000688BE883A88B2884D348018869834088AD
:103E8000A88316E39BF8011001EB810003EBC0004F
:103E9000427E12B1072A07D00DE09BF8010000EB2B
:103EA000800003EBC0040CE024B1827E94F81AC0B9
:103EB000624500D90446491CC8B28BF80100142899
:103EC000E0D3B4B3CBF824400320A0762076A675C7
:103ED0000420E075E6761A356889A0802889E0809C
:103EE000288820806888608001216176B6481E306D
:103EF00002782273427862738278A273C078E0738A
:103F00002182E87BE072A87BA072687B6072287BCC
:103F100020720120FFF731FC287D1A3D00F0F001EE
:103F200050292CD98BF801606FF0040101EB1013BC
:103F300020E0FFE7388D401C3885A4A000F050FD3C
:103F4000ABE22A1892F836108BF80210B9B10129A9
:103F500002D0022904D007E0401C8BF8010009E0E0
:103F600092F83710042920D092F8371039B108445C
:103F70008BF801009BF80100B0EB830FE1DB85F8C3
:103F80002FA02E35687840F0020068700220287259
:103F9000042068720720A872CA20E8722C20A9F8B1
:103FA0000400602005F82E0943E29BF8010092F816
:103FB0003810284490F8390040EA0120ABF80C0092
:103FC00040F2CA71884200D908466082A082D6E7D2
:103FD00095F82E10A846090989008BF80110BBF846
:103FE0000420511A143989B2ABF80410627E02F031
:103FF0000F02022A03D100F03F02122A19D009B998
:10400000810716D098F82610227A4346914274D13F
:1040100093F82710627A9142F9D193F8281000E0C2
:1040200070E1A27A9142F2D193F82910E27A91429A
:10403000EDD1C0063ED5218AE1B304F10C00FFF7B3
:1040400012FA614B98F82A102233C646187881423A
:1040500030D19EF82B2059788A422BD19EF82CC063
:104060009A78944526D19EF82DC0DB789C4521D1C5
:1040700020736173A273E373E07EA8B9207EA17EF2
:10408000401AA17DA0EBD10040B20144C9B2A17594
:10409000002801DA404240B2E27DA0EB92001044D9
:1040A000E07500EBD100207601208BF80000207E27
:1040B000A0762682627E02F00F0009286BD2DFE82C
:1040C00000F06A051EBBF5F4F31CF2009BF800003B
:1040D000C00760D00320607640208BF80000268265
:1040E000BBF8040020B142218BF80010FFF745FB1C
:1040F000ABF8066000F066FC04E192E193E19BF806
:104100000000C00705D098F82F0000F03F001228EB
:1041100009D020208BF8000000F054FCDBF82400CC
:10412000467669E611E198F82E0000F0F00150297A
:1041300025D98BF801606FF0040101EB101319E031
:1041400008EB000292F836108BF80210B9B1012981
:1041500002D0022904D007E0401C8BF8010009E0DE
:1041600092F83710042954D092F8371039B1084426
:104170008BF801009BF80100B0EB830FE0DB03201C
:10418000607698F82600207298F82700607298F8F8
:104190002800A0722CE08AE07463703A20676F7484
:1041A0002072657365742C2061626F7274696E672A
:1041B00020636F6E6E656374696F6E2E0000000081
:1041C000E46E0020C46B0020660200207463703A25
:1041D00020666F756E64206E6F20756E75736564F2
:1041E00020636F6E6E656374696F6E732E000000DE
:1041F00098F82900E0720120FFF7BFFA42208BF8FF
:1042000000002682ABF80460ABF8066000F0DAFB31
:1042100078E09BF8010092F83810404490F839009B
:1042200040EA0120ABF80C0040F2CA71884200D984
:1042300008466082A082A2E798F82F00C10721D02B
:10424000D1061FD4208A90BBBBF80400401C80B26A
:10425000FFF793FA9BF8000040F010008BF8000085
:10426000BBF8041019B140F002008BF8000000F018
:10427000A9FB0120208208206076E676112085F8CF
:104280002F00D0E0800616D598F8350098F8341045
:1042900040EA0120DBF81C100144CBF81C10BBF8ED
:1042A000041005E02DE173E0F0E0A3E07AE078E0AF
:1042B000081AABF80400BBF8040048B1D10607D4D3
:1042C0009BF8001041F002018BF80010FFF755FA3F
:1042D00098F8310098F8301000EB012080B2ABF86C
:1042E0000C00A18A814200D308B9ABF80C10BBF8CE
:1042F0000C0060829BF80000800752D0ABF806608B
:1043000000F060FB99F80000810606D5A9F8066068
:104310006676142085F82F0085E0C1060AD5A9F835
:1043200006600120208204206076E676112085F860
:104330002F0078E0B9F8061031B1C00700D026820E
:10434000208A90B1A9F80600E676D9F82000C9F8CD
:104350001C00B9F8060088B1208A78B12830A9F885
:104360000400182085F82F0060E0608A884201D29E
:10437000A9F80600B9F806002082E5E799F80000E0
:1043800080070ED52820A9F8040085F82FA04DE05D
:104390009BF80000C00704D066768BF800A000F000
:1043A00011FB7AE0BBF8040008B1FFF7E6F998F8D2
:1043B0002F00C00712D09BF80000C00704D00720D0
:1043C0006076A676268201E0062060760120FFF75F
:1043D000D4F98BF800A000F0F5FA22E09BF8000079
:1043E000C00703D005206076268256E0BBF80400A3
:1043F000B8B952E0BBF8040008B1FFF7BEF998F86D
:104400002F00C0070AD007206076A6760120FFF7AC
:10441000B4F98BF800A000F0D5FA02E0BBF8040074
:1044200098B388F82FA02820A9F80400502085F818
:104430002E001835207AA874607AE874A07A28755E
:10444000E07A6875207BA873607BE873A07B287492
:10445000E07B6874062005F8010C00E039E0A088D4
:104460006881E088A8813148018869804088A880F7
:104470002088E88060882881183D607EC00612D5BB
:1044800085F8316085F8306013E006E09BF80000A5
:10449000C00702D007206076A676A9F8046089F8E4
:1044A0000060BDE8FF9F072085F83000CA2085F82E
:1044B00031004020A875B9F80400010A2974687415
:1044C00085F8356085F834606E86FFF74DF8C04397
:1044D00068864520A873EE736E752E754020A8750A
:1044E000B9F80800401CA9F80800010AA974E8748A
:1044F0002E83FFF70EF8C04328830D48C18B491C5B
:10450000C1830B488188491C818089F80060C8E715
:104510000346002909DD05488AB20E38C280006AC8
:10452000834202D019461DF09BB8704766020020F6
:104530008C71002010B5B94900220A70B84B087878
:1045400000EB400403EB84042260401CC0B20870FE
:104550000828F4D310BDF0B5B04A9078401CC5B21D
:10456000957000231370AE4E117801EB410006EBFD
:104570008000048847883C4304D0847A2C1B782C24
:1045800000DB0360491CC8B210700828ECD3F0BDF2
:104590002DE9F041A14F4FF0000C87F800C0A04E6C
:1045A0003B7803EB430206EB8202148884B1558802
:1045B00075B1B0F80080A0450AD14488AC4207D15B
:1045C0000868506088881081B8789072BDE8F081E2
:1045D0005B1CDAB23A70082AE2D387F800C03B7855
:1045E00003EB430206EB820214880CB9548824B111
:1045F0005B1CDBB23B70082BF1D33B78082B1DD141
:1046000087F803C087F801C087F800C0BC783A7803
:1046100002EB420306EB8303FD789B7AE31AAB427D
:1046200001DDFB707A70521CD2B23A70082AEED3C8
:104630007A783A7002EB420206EB82020068106060
:104640000868506088881081B8789072BEE72DE9BC
:10465000F047744D002029882A2902D22880BDE81D
:10466000F0872880704C714F224602F11601B4F891
:104670001490B2F826C0881DB7F80080128D7B8890
:104680004FF40076B9F5807F08D0B145E7D1C44535
:10469000E5D19A42E3D1BDE8F04779E7C445DED1E0
:1046A0009A42DCD1FFF774FFA682D4F8160020628C
:1046B000618BA1845E4B1A68C4F816209B886383C3
:1046C000C4F8062063812060A180A08BE084E08B89
:1046D00020853888A0837888E0834FF4C160A0816A
:1046E0002A202880BBE72DE9F05FDFF83CA1504B82
:1046F0005046BAF81E104FF6FF72008C9C881D6859
:10470000914209D1904207D14A480168CAF8001085
:104710008088AAF804003FE0444F474BB7F8009068
:104720001A88B7F802803D4F01EA020609EA020240
:104730003F1D964206D15A8800EA020308EA0202A7
:10474000934205D03D48018839804088788001E057
:1047500039807880314B4FF0000B83F800B03E88F1
:10476000DFF8BCC07F88197801EB41000CEB8000BA
:104770000288964202D14288974204D0491CC9B2AD
:1047800019700829EFD31978082912D04168CAF89E
:1047900000100089AAF80400CAF80650AAF80A40D6
:1047A0000820AAF80C001F4801880E310180BDE8DE
:1047B000F09FFF2206211C481CF064FFCAF820B0BD
:1047C000AAF824B0CAF80650AAF80A40CAF8165047
:1047D000AAF81A40AAF82660AAF82870AAF81C902D
:1047E000AAF81E804FF48070AAF81400AAF80E00F0
:1047F0000820AAF8100006208AF8120004208AF87F
:1048000013004FF4C160AAF80C0007480C49363079
:10481000086004482A210180C9E7000090020020B6
:10482000C07100205C020020C063002066020020EE
:1048300050020020F88804086A0200208C02002040
:1048400074020020014800687047000050000020FA
:104850002DE9FC5F53480546F8F739F90646002074
:10486000504C5149143C2218127D0A54401CC0B2CD
:104870000628F8D340F276411420F8F70BF9FEF73A
:1048800077FE94F82F0040B10621284600F05FFA29
:1048900000F076FA3046BDE8FC9F1A34657822783D
:1048A00045EA0220010241EA1027E178A37841EAB3
:1048B00003204FEA002C4CEA1020DFF8F0C0ACF8DF
:1048C0000070ACF80200A07A677A40EA072007027D
:1048D00047EA1027207B94F80BC040EA0C204FEAEF
:1048E000002C4CEA1020DFF8C8C0ACF80070ACF81F
:1048F0000200A079677940EA072C4FEA0C2848EAC1
:104900001C2AADF804A094F808C094F807804CEA7B
:1049100008294FEA092B4BEA1929ADF80690DFF870
:1049200094B0ABF800A0ABF80290C7F1FF073A4390
:104930008DF80020C0F1FF0005438DF80150C8F14B
:10494000FF0003438DF80230CCF1FF0001438DF8E6
:10495000031045EA0220020242EA1020164A1080A3
:1049600041EA0320010241EA102050800120FEF7B5
:104970003DFDE089010241EA102080B2FEF7EAFE27
:1049800000F078FC09F0DAF884E710B50B4940F242
:10499000EE50F8F785F980B210BD09480749008844
:1049A000F8F74DB91C7B0020500200206602002061
:1049B0008C0200206A0200206E020020C0630020EA
:1049C0005C0200200748008D010241EA10200649E0
:1049D00080B209688988884201D100F091BB704794
:1049E00070470000087B00207C0200203522027006
:1049F000012242708170C01C704736210170042171
:104A00004170E649C969C0F80210801D7047322123
:104A1000017004214170E149496AC0F80210801D0B
:104A20007047372101700321417001228270C170EB
:104A300006210171401D7047FF2100F8011B7047DE
:104A40002DE9F0410446012020706070D34D287E8E
:104A5000A0700020E070D24E31686160208180211A
:104A60006181D0490968E16020616061A061D5E998
:104A7000051204F11C0007461CF0F2FDA869C0F104
:104A8000100138441CF005FE402104F12C001CF0FC
:104A900000FE802104F16C001CF0FBFD7068C4F87E
:104AA000EC00BDE8F08170B5BF4D2C682046FFF7E3
:104AB000C7FF012104F1F000FFF798FFFFF7B1FFF6
:104AC000FFF7BAFF01462868BDE87040091AFFF7F2
:104AD0001FBD70B5B44D2C682046FFF7B1FF032110
:104AE00004F1F000FFF782FFFFF787FFFFF78FFF6A
:104AF000FFF7A2FF01462868BDE87040091AFFF7DA
:104B000007BD10B544180023A44A29E001783329D1
:104B100020D006DC01290BD003290DD006291CD199
:104B20000EE0352910D0362910D0FF2915D11BE011
:104B3000D0F80210916210E0D0F8021011630CE07E
:104B4000D0F80210D16208E0837806E0D0F80210B5
:104B5000D16102E0D0F8021011624178801C084453
:104B6000A042D3D3184610BD184610BD70B58E486C
:104B70000468207802280DD104228949201D1CF0E8
:104B8000D2FD38B9854D04F11C00D5E905121CF0A1
:104B9000CAFD08B1002070BD2069686283480188A1
:104BA00004F1F000BDE87040ABE77C4900204A68A2
:104BB00090807F480278437802EB03228A848278CF
:104BC000C37802EB0322CA844279837902EB032281
:104BD0000A85C279037A02EB03224A85427A837AF4
:104BE00002EB03228A85C37A007B03EB0020C88591
:104BF0000A86488670472DE9F0470122674C4FF43A
:104C0000BE77002521886B4E4FF4D77804F1080950
:104C1000B94245D007DC4FF47A7A59B1A1F58071D9
:104C200053397DD113E041457BD04FF4DA70814296
:104C300076D183E00120A070A4F810A0FFF733FF25
:104C4000218A4846FEF7ECFB40F253102080307872
:104C5000800703D44846FEF7F5FBE8B330788007B9
:104C600003D5FFF783FF02283DD0208A4EF660214E
:104C7000884204D24FF6FF7101EA40002082208A68
:104C8000B0F57A5F3AD2A0780228D7D1A4F810A064
:104C90003570FFF71EFF218A4846FEF7C1FB2780CB
:104CA0003078800703D44846FEF7CCFBF0B130786B
:104CB000800703D5FFF75AFF052819D0208A42F252
:104CC0001071884217D800F57A7080B22082B0F552
:104CD000FA5F13D2A07800E002E00328D9D10FE0F8
:104CE0000020BDE8F0870220A070CFE70020F8E7A1
:104CF0000320A07004E025800020F2E7FFF755FFB5
:104D0000264800F002FC608C0106090C41EA1021E3
:104D1000208C020242EA102001EB0041322001E027
:104D200012E005E041434846FEF77AFBA4F8008014
:104D30004846FEF787FB0028ABD1D2E712B100222C
:104D40002080FBE70320CCE725800220C9E738B5A7
:104D5000124C6061A1610025A5704FF6FF70ADF89F
:104D60000000ADF802004FF486416846FEF797FC5C
:104D7000606010B14FF488418180258038BD3AE7EA
:104D800008B506488078002806D1ADF80000ADF8D7
:104D9000020004490880488008BD000020720020FD
:104DA000FE88040866020020740200205C020020D5
:104DB000227B00205802002010F8011B02E0401C5A
:104DC000491EC9B20029FAD101780029F4D1401C4A
:104DD000704770472DE9F047A84D00262E70A84A6D
:104DE0004FF001082878C0EBC00000EB400002EB58
:104DF00040042078012801D0022837D1022820D091
:104E00000220207084F80180A6709E4FD7F8009091
:104E1000C9F80060C9F80460C9F808602878FEF78E
:104E20006AFBA9F8000089F802804FF48070A9F8A5
:104E3000040039680C31241D641C0A46491C6E703C
:104E400022E06078401E10F0FF0060700ED1A07864
:104E5000401CC0B2A070082802D0A0786070D4E7CF
:104E6000042020700021601DFFF7B3FF2878401C4C
:104E7000C0B228700428B5D3BDE8F08701F8010B53
:104E80006878401C6870641C20782E2801D00028A7
:104E9000F4D16878107020780028CDD12869086096
:104EA000287D08713868BDE8F047091A491DC9B264
:104EB000FFF72EBB2DE9F041724F3C682088FEF7CA
:104EC0001AFB6E4EC0B23071C0EBC0016C4A01EBF0
:104ED000410102EB410504283DD2287802283AD14D
:104EE00003202870E07800F00F00287130B1042012
:104EF00028700021681DBDE8F0416AE7A088FEF730
:104F0000FAFAB070E088FEF7F6FAF07038680C3004
:104F1000FFF752FF001D4FF4807719E001788909EF
:104F200001D0841C02E0FFF747FF04462088B84206
:104F300006D16088B84203D12089B0F5806F0CD0CB
:104F40002089FEF7D8FA20440A30F178491EF17022
:104F5000F1780029E2D1BDE8F0816089E884A08978
:104F6000288505F12601681DBDE8F04131E710B53F
:104F700045480068C088B0F5545F0BD1434C207899
:104F8000000701D5FFF726FF2078800702D5BDE88E
:104F900010408FE710BD70B50146384D0020E87114
:104FA000A8716871364B6879C0EBC00202EB42020F
:104FB00003EB4204227862B1E278AE7AB21AAE799B
:104FC000B24201DDAA71E871401CC0B268710428C8
:104FD000E9D36879042807D1E8796871C0EBC0008B
:104FE00000EB400003EB4004601D1CF0BDFB012002
:104FF0002070A87AE070401CA87270BD2DE9F041C5
:1050000007461E4D002028721D4E287AC0EBC000B6
:1050100000EB400006EB40042078032804D1611D1A
:1050200038461CF072FB38B1287A401CC0B2287296
:105030000428EAD300208EE704F126008BE70F480E
:10504000C0680028FFD170470C48C068002801D014
:1050500000218180704710B5084A00205072084B2B
:105060000324507AC0EBC00101EB410103F8114069
:10507000401CC0B250720428F3D310BD9802002027
:105080005472002074020020800200205802002088
:10509000524800681C308168002902DD4068FFF733
:1050A00037BA70474D480068002141624CA0FFF7B5
:1050B00097BC10B5494804684E48017841F080011A
:1050C00001704DA0FFF78CFC00202077606210BDBE
:1050D0004848017821F0800101704DA0FFF780BCA5
:1050E0004448017821F0800101704FA0FFF778BC9F
:1050F0004048017821F08001017051A0FFF770BC99
:1051000070B50024354805681C35534E307880064C
:1051100001D5FFF7EDFF3078000601D5FFF7E0FF7E
:105120003078C00601D5FFF7D3FF3078400601D5AF
:10513000FFF7BFFF3078C00701D0FFF7B3FF30782B
:10514000800732D5454802884548016845481CF02B
:1051500087FA44480178EE290ED1417810290BD105
:10516000817849B9C17839B9017929B9417919B931
:10517000817909B9C17941B13B498079097988427E
:1051800008D0FF2806D028B10FE0012437490120BC
:1051900008700AE001243349012003F0E5FA31499F
:1051A000012003F0A5F9F8F7E7FB307800F00401DF
:1051B00000F00202114351EAC07103D1410601D44B
:1051C000000709D5012C04D12948686009484088A6
:1051D000A860BDE870405BE770BD00007C02002065
:1051E0007463705F7365727665722061636B65646A
:1051F000210D0A00AE0200207463705F7365727641
:10520000657220636F6E6E6563746564210D0A00BC
:105210007463705F73657276657220636C6F73651B
:1052200064210D0A000000007463705F736572767C
:1052300065722074696D656F7574210D0A00000038
:105240007463705F7365727665722061626F7274E9
:105250006564210D0A000000580200205C02002055
:1052600074020020FC720020087B00200100002056
:105270002874002010B54DF204242046FEF76AFA87
:10528000ED48848010BD70B505463C21EB481CF00C
:1052900000FAEA4C15B1012D03D004E0652020701E
:1052A00001E0672020700025241D04F8035CE44819
:1052B000017821704178A17081782171C178A17144
:1052C000817B21720179A172817E2173C17EA173DC
:1052D000017F2174417FA174018D2175090A6175D7
:1052E0004421A175E575C07B20766576A576E576C7
:1052F00025776577D3480668300AA077E67784F883
:105300002050CE481422D04925301CF0A9F9300E87
:1053100084F83500300C84F8360084F837503C218E
:10532000C648FFF7F5F8C9490120087070BD2DE99E
:10533000F0470024C648007880077DD5C54890F81E
:1053400000A0C54852460168BC483C301CF088F9B2
:10535000BA4EBE4F3C36BA4D30784FF00109A046E8
:1053600064286AD066287FD17078A97E88427BD174
:10537000B078E97E884277D1F078297F884273D16E
:105380003079697F88426FD1707C297888420BD14F
:10539000B17C6A78914207D1F17CAA78914203D11D
:1053A000317DEA7891420AD000285DD1B07C002896
:1053B0005AD1F07C002857D1307D002854D10120EB
:1053C000FFF761FF1A3585F8048072792A70B07989
:1053D0006870F379AB70317AE9706A74A874EB7411
:1053E000297596F8098085F80580B37AAB71F47A4F
:1053F000EC7196F80CC085F808C085F81680EB753E
:105400002C7685F819C0747B6C7296F80EC085F8FE
:105410000AC0F37BEB72367C2E73AC7685F81BC02A
:105420002B776E771A3D87F80190002A1CD0002850
:105430001AD0002918D001E016E017E000242E1938
:1054400004F12F00B17EF7F7A0F8F17F04F13300EB
:10545000F7F79BF896F8231004F13700F7F795F863
:10546000641CE4B2042CEAD3BDE8F08787F800900E
:10547000A97E2A7FEB7E6D7F14E006EB840090F816
:1054800001C08C450CD190F802C09C4508D190F821
:1054900003C0944504D10079A84201D187F8008067
:1054A000641CE4B2B4EB9A0FE7D338780028DBD061
:1054B000BDE8F0470020E6E610B5684C206880881B
:1054C000A0F54040BA3806D0A0F588504A3804D13B
:1054D000FFF72DFF01E008F045FB2068C088B0F51C
:1054E000545F0DD0B0F5864F06D0B0F5884F0BD184
:1054F000BDE81040FFF743BCBDE81040FFF73FBCDC
:10550000BDE81040FFF733BD10BD2DE9F041544C0C
:10551000818C2180C18C6180524D018D2980418D0B
:105520006980514F018E3980418E79802C30FFF790
:105530008BFDFFF79FFE424E1A36F089010241EAC9
:10554000102080B2FEF706F92088FDF7D4FF000A8C
:1055500030702088FDF7CFFF70706088FDF7CBFFBB
:10556000000AB0706088FDF7C6FFF0702888FDF76C
:10557000C2FF000A70712888FDF7BDFFB07168880E
:10558000FDF7B9FF000AF0716888FDF7B4FF3072CB
:105590003888FDF7B0FF000A70723888FDF7ABFF5E
:1055A000B0727888FDF7A7FF000AF0727888FDF7DF
:1055B000A2FF30731A3E0025741914F81A1F617483
:1055C0006079A075607AA07605F12F00F6F7DDFF0F
:1055D000617905F13300F6F7D8FF617A05F13700FC
:1055E000F6F7D3FF6D1CEDB2042DE5D316F81A0FB4
:1055F0007378B178F2787479C4F1FF042043B479F8
:10560000C4F1FF042343F479C4F1FF042143347A45
:10561000C4F1FF04224343EA0020030243EA1020BE
:10562000124B188042EA0120010241EA1020588002
:10563000BDE8F04108F082BA0C6F002054750020DC
:10564000087B00200C000020747C0020B2020020A7
:10565000580200205C02002074020020800200201A
:10566000660200206A0200208C0200206E020020E8
:105670000020F8490860F84988824873C87270476A
:105680002DE9F047F2F79AFDDFF8D09340F2255567
:1056900029464846F6F734FB0224F14FEE4E4FF010
:1056A0000008012808D040F2277A51464846F6F70C
:1056B00027FB012872D0ABE0B470B87C032801D07E
:1056C00098B3A5E0B08AE74D502807D24846F6F7D0
:1056D000A3FAB18A4A1CB282685401E0FFF7C8FFFE
:1056E000B08A01281CD0032820D0042824D0072801
:1056F00030D0F18A884212D12878FF2802D0397937
:10570000884239D11420F0727473D349203108785B
:10571000401CC0B2087063287AD981F8008077E015
:105720005020F082307BF07272E028E0687819280F
:105730006ED10620F0826BE0E878A97800EB0120BA
:105740000A2865D16878062862D10C20F082307B67
:10575000F0725DE06878032804D0062802D0102893
:1057600003D055E00820F08252E0A87900F1090149
:10577000F1820830F0724BE0FFF77AFF48E02946EB
:105780004846F6F7BDFA012842D14846F6F744FAF2
:10579000C1B2B54816F0E1FF3AE0FFE7B87C032854
:1057A00000D0A8BBB08B411CB183B049095C48460E
:1057B000F6F72EFA17F06FF8B08B318B884227D3AB
:1057C000F47000244FF47A7502E00120FDF7EEFD3D
:1057D00040214846F6F789FA20B92046641CA4B255
:1057E000A842F2D3AC4203D3A148C18A491CC1826A
:1057F00040214846F6F780FA002251464846F6F71F
:10580000B2F9A6F81C80B87C032805D0FFF730FF5A
:10581000BDE8F047F2F7D9BCF07B30740028F7D12F
:10582000FFF726FFF4E78B48016800228A48012928
:1058300005D0C283C18B642905D9C28318E7C18B07
:10584000491CC183F6E77047824901200860704710
:1058500070B506460C46814D40212846F6F74CFAB5
:1058600031462846F6F7D4F9002C04D03046BDE87E
:10587000704006F010BF70BD77490883012240F2E6
:1058800027717648F6F76FB970B5FFF7F1FE724CE5
:1058900003202073E07240F28370F6F708FFA073D4
:1058A0000A25642800D9A57340F28470F6F7FFFE3C
:1058B000E073642800D9E57367490020203108703F
:1058C000487070BD70B5A0F51C53103B17241144EF
:1058D000442B14D8B3FBF4F004FB103000282AD179
:1058E000B3FBF4F0C0B2C0EB0010624ABDE87040F8
:1058F00000EB4000C91D10442D221BF0B1BEA0F5E5
:105900003052D03A0125A02A16D8B2FBF4F004FB9D
:10591000102000280FD1B2FBF4F0C0B2C0EBC002DF
:1059200002EB0010544AC91D02EB40002E221BF06E
:1059300097FE5248457070BDA0F54852903AB2F5B6
:10594000397F15D21420B2FBF0F300FB1323002B98
:10595000F1D1B2FBF0F0C0B2C0EBC00202EB4010DC
:10596000474ABDE87040C91D104427221BF078BE8D
:10597000A0F5FE40C8382928DDD80E22B0FBF2F38E
:1059800002FB1303002BD6D1B0FBF2F0C4B23D4AA8
:10599000C4EBC40002EB8000C91D1C221BF060FE9A
:1059A000394904EB440001EB4000457170BD30B54E
:1059B000A0F51C53103B1724442B0DD8B3FBF4F077
:1059C000C0B2C0EB00102B4900EB40004218B3FB03
:1059D000F4F004FB10313AE0A0F53053D03B264DF3
:1059E000A02B0DD8B3FBF4F0C1B2C1EBC10000EBAA
:1059F000011005EB4002B3FBF4F004FB103126E08C
:105A0000A0F54853903BB3F5397F0ED21420B3FB79
:105A1000F0F1C9B2C1EBC10202EB011105EB410289
:105A2000B3FBF0F100FB113111E0A0F5FE40C838E6
:105A300029280CD80E21B0FBF1F2D2B2114BC2EBE7
:105A4000C20203EB8202B0FBF1F301FB130132F857
:105A5000110030BDA0012142B402002000380140F5
:105A6000087B0020BC760020D8D70020B07800202A
:105A7000A28100200682002090820020EC020020FB
:105A800090860020228E0020108E00202DE9F04FFD
:105A900089B004468B46154605EB0B20079001277D
:105AA00080B245EA0B280890642C7DD2012C1ED8C8
:105AB00029460020F6F769FD59460120F6F765FDF5
:105AC000FE4C257084F801B0207C40F00101217467
:105AD0001120F6F75AFD207C002866D00020607364
:105AE00009B00021BDE8F04F1020F6F74EBD032CA1
:105AF0001ED829460220F6F748FD59460320F6F73E
:105B000044FDEE4CA57084F803B0207C40F0020107
:105B100021741120F6F739FD207C002872D0002076
:105B2000607309B00021BDE8F04F1020F6F72DBDDD
:105B3000062C23D0E24E072C2FD0082C71D00F2C2E
:105B400070D0102C6FD0152C6ED01D2C6DD0DD496F
:105B5000252C08686AD0262C69D0272C68D0A4F19F
:105B60002800052871D8C0B2D44901440D7509B088
:105B70002946BDE8F04F2830F6F707BDCF4C257118
:105B800029460620F6F701FDCF492079487109B072
:105B90000020BDE8F04F15F0E7BFC84CA07BA8423D
:105BA00030D02946072001E020E32BE0F6F7EDFC9A
:105BB000A573C64F3D70207C40F008012174112070
:105BC000F6F7E3FC3878D2281FD0D3281DD0D92887
:105BD0001BD0D6281FD0D7281DD0D42829D0D5280F
:105BE00027D034282BD0BAA2BBA1B5481DF018F895
:105BF000002404F26170315DF6F757FD641CE4B2D5
:105C0000142CF6D309B0BDE8F08FB4A2B2A1AC4811
:105C10001DF006F8ECE7B3A2AFA1A9481DF000F80B
:105C2000E6E713E022E078E043E255E260E270E26A
:105C30007EE2AFA2A8A1A2481CF0F2FFD8E7AEA274
:105C4000A5A19F481CF0ECFFD2E780E2294608207E
:105C5000F6F79BFC9948C573017C41F0040101747F
:105C600009B01120BDE8F04FF6F78FBC93490D73D2
:105C7000062D4ED2DFE805F003101D2A42364FF400
:105C800016508860FDF746FA29461520F6F77DFC88
:105C90008D49062008733CE04FF496408860FDF77C
:105CA00039FA29461520F6F770FC87490320087356
:105CB0002FE04FF416408860FDF72CFA2946152096
:105CC000F6F763FC80490220087322E04FF461403C
:105CD0008860FDF71FFA29461520F6F756FC7A482A
:105CE000077316E04FF496308860FDF713FA2946E3
:105CF0001520F6F74AFC744807730AE04FF4E130C8
:105D00008860FDF707FA29461520F6F73EFC6E4835
:105D1000077309B0BDE8F04FB6E5684845737F2DBD
:105D200009D0632D0AD08E2D02D08F2D7FF46AAF5B
:105D30008E2D0CD010E07248077063E7632140F2AB
:105D4000B970F6F7B2FC6E48022101705AE70021E3
:105D500001741120F6F719FC002140F2A760F6F754
:105D6000A4FC00214FF4D560F6F79FFC052140F21A
:105D7000AD60F6F79AFC05215020F6F796FC614CD1
:105D80004FF47A75A581E8214920F6F78EFCA089A9
:105D9000010A4A20F6F789FC4FF4487060812021FF
:105DA0004720F6F782FC6089010A4820F6F77DFC5F
:105DB00002214520F6F779FC02214620F6F775FC12
:105DC00005214D20F6F771FCFF215E20F6F76DFCF2
:105DD00000215220F6F769FC00215120F6F765FCFE
:105DE000494C6800608107215420F6F75EFCA17AD7
:105DF0005320F6F75AFC00216020F6F756FC0021EC
:105E00005F20F6F752FCE58003216220F6F74DFC97
:105E1000A1796120F6F749FC00216420F6F745FCE2
:105E200000216320F6F741FC658003216620F6F728
:105E30003CFCA1786520F6F738FC3448002101705D
:105E40005620F6F732FC324C31212170322060703E
:105E50003320A0703420E0705720F6F726FC6178DC
:105E60005820F6F722FCA1785920F6F71EFCE178BD
:105E70005A20F6F71AFCFF215E20F6F716FC0521E2
:105E800040F20470F6F711FC052140F20370F6F7BA
:105E90000CFC052140F20270F6F707FC0B4D287848
:105EA000D2287CD0D3287AD0D92878D0D62877D0D9
:105EB000D72875D0342874D00DA22BE0087B0020A1
:105EC000747C00200C000020B4020020040000209C
:105ED0006F7468657200000025730000434F325FE5
:105EE0004E45540050726573737572650000000072
:105EF00048756D6469747900504D322E350000008C
:105F000001000020348C00203E0300207704002094
:105F100078040020AFF24001FE481CF081FE00240E
:105F200004F26170315DF6F7C0FB641CE4B2142C1E
:105F3000F6D30A2140F28370F6F7B7FB0A2140F24C
:105F40008470F6F7B2FB002140F28570F6F7ADFBE6
:105F500072B6F6F7FFF9F04E3046F6F728FA4FF62C
:105F6000FF7421463046F6F73FFAEC4E3046F6F71E
:105F70001EFA21463046F6F737FAE94E3046F6F774
:105F800016FA21463046F6F72FFAF6F7E9F962B627
:105F900000212E20F6F7F9FAC0212F2002E049E077
:105FA00050E057E0F6F7F1FAA8213020F6F7EDFAC5
:105FB00000213120F6F7E9FA03213220F6F7E5FA5D
:105FC000FF213320F6F7E1FAFF213420F6F7DDFA5E
:105FD000FF213520F6F7D9FA00213620F6F7D5FA59
:105FE000C0213720F6F7D1FAA8213820F6F7CDFAEC
:105FF00000213920F6F7C9FA01213A20F6F7C5FA4F
:1060000000213B20F6F7C1FA01213C20F6F7BDFA4A
:10601000F6213D20F6F7B9FA002140F2A970F6F713
:1060200044FB002140F28270F6F73FFB28783428C9
:1060300017D018E0AFF25C12AFF26411B5481CF053
:10604000EFFD6CE7AFF26412AFF27411B1481CF0CF
:10605000E7FD64E7B3A2AFF28011AE481CF0E0FDAB
:106060005DE710F08FFF0024FF2104F12300F6F715
:106070001CFB641CE4B2042CF6D30C212720F6F799
:1060800014FBAA4C05202071052140F2B470F6F7EC
:106090000CFB0F21218140F2B570F6F706FB208939
:1060A000010A40F2B670F6F700FBA1480221017028
:1060B000A8E5032D01D0002DFAD129461420F6F7CA
:1060C00064FA9C488574032D03D09B490220087014
:1060D00098E59948077095E5012DE9D9974805702D
:1060E00009B02946BDE8F04F40F2CE70F6F74DBA40
:1060F0006FF30F0048EA0008C1F80080294623200A
:10610000F6F7D3FA09B05946BDE8F04F2420F6F768
:10611000CCBA80B240EA0840086029462520F6F74C
:10612000C4FA09B05946BDE8F04F2620F6F7BDBACB
:10613000804C257129460620F6F727FA80492079F8
:10614000487109B00020BDE8F04F15F00DBD3D2CA1
:1061500009D0A4F13E00032809D8C0B2754908440B
:1061600080F82B504EE5734880F82F504AE5A4F193
:106170004200032805D8C0B26E49084480F8305068
:1061800040E5A4F14600032805D8C0B26949084497
:1061900080F8345036E54A2C0BD04B2C0DD04C2CCB
:1061A0000FD0502C11D05D2C92D1624880F82A502B
:1061B00028E5604880F8385024E55E49089848870B
:1061C00020E55C4880F83C501CE55E48012D01D07C
:1061D00015B103E0077001E000210170017809B0FA
:1061E0004FF4F860BDE8F04FF6F75FBAA4F54062EF
:1061F00047F619604FF484713E3A7DD0521E7CD030
:10620000D01E7BD0B4F5446F79D0401C78D04E4876
:1062100012F5ED6175D0B4F59B6F73D0891E72D005
:10622000491E71D0491E70D0491E6FD0491E6ED0D4
:10623000B2F10F006CD0454805EB0B2109B2027892
:1062400045EA0B2006B2A6F5A0704FF47A7C00EB6D
:10625000800001FB0CFC0690CDF810C0A5F13000C9
:10626000DFF8F0C00590642339484B439CF800C028
:10627000DFF8E490DFF8E4A0B4F5357F05D8BCF191
:10628000D40F46D0BCF1D50F43D040F28F3E7445B9
:1062900005D2BCF1D60F7DD0BCF1D70FFBD0932C2B
:1062A00002D2BCF1340F76D0B92C75D0D22C74D078
:1062B000C82C73D0C92C72D0DFF8A4E0CA2CBEF968
:1062C00000C06DD0CB2C6CD0CC2C6BD0CD2C6AD038
:1062D000CE2C69D0CF2C68D0D02C3FF42EADD12C51
:1062E00071D0D32C70D0D42C6FD0D52C6ED0D62CAE
:1062F0006DD0A4F5806235E05AE094E0CCE0E3E0B4
:10630000DBE0EDE0FDE0F6E001E106E10BE110E1AC
:1063100015E12CE1747C002000E0070800D007089C
:1063200000F00708504D323500000000CE8C0020F0
:1063300001000020087B0020000000200600002053
:10634000B402002063000020860000202903002002
:10635000228E002004000020A0000020FC09002064
:1063600064030020CF3A74D0B4F59A6F72D0921EB5
:1063700071D0521E032A6FD8059809283FF6DDAC6C
:1063800090B2FE490D5409B02946BDE8F04F573090
:1063900080B20BE0FEE3FEE3FEE3FEE3FEE3FEE39A
:1063A000FEE3FEE3FEE3FEE3FEE3FEE3F6F77DB984
:1063B000062DBFF4C2ACF24C25704DB1012D13D0A7
:1063C000022D28D11CE0F1E3F1E3F1E3F1E3F2E384
:1063D0004FF6FF72CDE90012029037210A23E94AF5
:1063E0000846FAF745F916E04FF6FF72CDE90012BC
:1063F000029037210A23E44A0846FAF739F90AE0FD
:106400004FF6FF72CDE90012029037210A23DF4ACE
:106410000846FAF72DF9217840F2BC70F6F745F9F5
:10642000DB48C77189E4062DFCD2DA4C257025B112
:10643000012D12D0022D27D11BE04FF6FF72CDE9BE
:106440000012029037215A23CE4A0846FAF710F973
:106450001AE07EE0FDE3FDE3FDE34FF6FF72CDE9D8
:106460000012029037215A23C74A0846FAF700F96A
:106470000AE04FF6FF72CDE90012029037215A234D
:10648000C24A0846FAF7F4F8217840F2BD70F6F7F0
:106490000CF9BF48077250E4022DC3D20DB101219F
:1064A00000E00021BC48017040F2C170F6F7FDF831
:1064B00009B0BDE8F04FFAF73BB8012DB2D109B0F1
:1064C000BDE8F04FFAF734B8062DABD2B3480570EB
:1064D000294640F2BE70F6F7E8F8AD4847722CE462
:1064E000A8F2D17162299DD2A0F8038009B0BDE85D
:1064F000F04FF7F7D6BB857109B0BDE8F04FF7F75D
:10650000D0BB457109B0BDE8F04FF7F7CABBC57104
:1065100009B0BDE8F04FF7F7C4BB057009B0BDE89E
:10652000F04FF7F7BEBB457009B0BDE8F04FF7F785
:10653000B8BB857009B0BDE8F04FF7F7B2BB98481B
:10654000057009B02946BDE8F04F40F2CF70F6F76C
:10655000ACB89448A0F8008029464E20F6F7A5F87C
:1065600009B05946BDE8F04F4F20F6F79EB8B92C58
:106570002BD0792C71D0652C70D0642C6FD0B4F5F1
:10658000987F1BD0A4F5807CBCF1750C16D0B4F5B7
:10659000F27F79D0BCF19E0277D0521E032A75D8C3
:1065A000059809289BD890B274490D5409B0294622
:1065B000BDE8F04F573080B2F6F777B8A9F8006021
:1065C000900776D57848068072E578490D73062DD8
:1065D00051D2DFE805F003101D2A45364FF416505E
:1065E0008860FCF797FD29461520F5F7CEFF68492E
:1065F000062008733FE04FF496408860FCF78AFD60
:1066000029461520F5F7C1FF61490320087332E0E0
:106610004FF416408860FCF77DFD29461520F5F7FC
:10662000B4FF5B490220087325E04FF461408860A5
:10663000FCF770FD29461520F5F7A7FF54480773AE
:1066400019E04FF496308860FCF764FD2946152068
:10665000F5F79BFF4E4807730DE011E022E02CE0B8
:106660004FF4E1308860FCF755FD29461520F5F719
:106670008CFF4748077309B0BDE8F04FFFF704B936
:106680002DB14B48077005E032E02DE046E0484868
:10669000002101704648017809B03F20BDE8F04F65
:1066A000F6F703B8A9F80060D00703D04148068088
:1066B000FEE411E040480770FAE40698092190FBD7
:1066C000F1F000B2A9F80000D10702D039490880E2
:1066D000EEE439480770EBE440F2B6308642E7DA80
:1066E000354802210170E3E46DB1344807700DE0D4
:1066F00015B1A9F8007002E00020A9F800002E48AA
:1067000004210170D4E42D49002008702B48017841
:1067100009B05620BDE8F04FF5F7C7BFA4F50072E9
:106720001A3A73D0B4F5067F7ED0521E7DD0B4F5F0
:10673000B97F7BD0A8327AD0B4F5BA7F78D0563200
:1067400077D0B4F58F7F75D0921E74D0B4F5907F5A
:1067500072D04A3A71D0B4F5E27F6FD05C3A6ED015
:10676000B4F5E37F6CD0921E6BD0521E132A69D809
:1067700002F0010812480770002123E0780400208D
:10678000A4000020DA2004087C3804081EAB0308AB
:10679000B4020020A5000020A7000020A6000020D1
:1067A000050000201A0300204C030020087B002075
:1067B000540300202A0300209C00002077040020BE
:1067C00051030020FD48018440F25C70F5F76CFF36
:1067D000002140F25D70F5F767FFA4F5E470C0F3A7
:1067E000460040F2347101EB8007491C01EB80093F
:1067F000B8F1000F7ED038462946F5F755FF09B0AD
:1068000048465946BDE8F04FF5F74EBFEC4C60895D
:1068100057287FF6D9AE40F68C2108FB01F1B1FB79
:10682000F0F1A1F6D2710EE033E022E03EE03AE072
:106830004CE03EE05BE04DE074E067E089E07EE044
:106840009DE090E04AE15738B1FBF0F02081A4F8D8
:106850000280A4F80080C1B240F2B570F5F725FFC0
:10686000208909B0010ABDE8F04F40F2B670F5F793
:106870001CBFD348A0F80880294640F2B570F5F750
:1068800014FF09B05946BDE8F04F40F2B670F5F775
:106890000CBFCB48057109B02946BDE8F04F40F266
:1068A000B470F5F702BFC748068011E4C64805700A
:1068B0000EE4C648868029465F20F5F7F6FE09B04B
:1068C0005946BDE8F04F6020F5F7EFBEC048A0F88C
:1068D000008047E4BD48068029466320F5F7E5FEC1
:1068E00009B05946BDE8F04F6420F5F7DEBEB74861
:1068F000C68000E073E029466120F5F7D6FE09B0B6
:106900005946BDE8F04F6220F5F7CFBEB14C257077
:1069100029465E20F5F7C9FE207809B0BDE8F04FA2
:10692000F6F79FBFA948468029466520F5F7BDFECA
:1069300009B05946BDE8F04F6620F5F7B6BE8AF8B3
:106940001A5009B02946BDE8F04F40F20470F5F73F
:10695000ACBE8AF8195009B02946BDE8F04F40F2A4
:106960000370F5F7A2BE0A2DB3D29B4805702946E5
:1069700040F23170F5F798FE984807700AE498489D
:106980000078012807D00228F8D1032DF6D19549C7
:10699000082008700CE4012D01D0002DFAD1924896
:1069A000057029464FF4DB60F5F77EFE8B480770D3
:1069B0000024AAF82040002140F25D70F5F774FE33
:1069C000002140F25C70F5F76FFE8348047009B057
:1069D0000021BDE8F04F40F23170F5F765BEA4F537
:1069E000E470C0F3460040F2327202EB800840F2DD
:1069F0003372711C02EB800A1CD076B378480078A1
:106A000001283DD00228C5D1784C4046217AF5F7BF
:106A10004BFE2089010A5046F5F746FE38462946C6
:106A2000F5F742FE48465946F5F73EFE6D49092006
:106A30000870F7E44046FF21F5F736FE5046FF2187
:106A4000F5F732FE3846FF21F5F72EFE09B048462D
:106A5000BDE8F04FFF21F5F727BE40460021F5F7CE
:106A600023FE50460021F5F71FFE38460021F5F7BA
:106A70001BFE09B04846BDE8F04F0021F5F714BEF3
:106A80004E48817D3846F5F70FFE4C48C08A010A12
:106A90004846F5F709FE40462946F5F705FE5046FB
:106AA0005946F5F701FEB4F5E47FC2D14A480078B3
:106AB0000128BED14E48414C0088301A2084C1B212
:106AC00040F25C70F5F7F0FD208C09B0C0F30721AF
:106AD000BDE8F04F40F25D70F5F7E6BDA4F58072B9
:106AE000E13A38D0121F39D0B4F5E17F4FD02232CD
:106AF0003ED01C3A60D00C3A5FD0B4F5F67F7FD020
:106B0000121F7ED0B4F5F87F7CD0B4F5F37F7AD035
:106B1000B4F5FA7F78D0921F77D0B4F5FB7F75D0AB
:106B2000921E74D0B4F5FF7F72D0083A71D0B4F5DC
:106B3000007F6FD0921E6ED0B4F5027F6CD0083A01
:106B40006BD0511E6AD0491E69D0C81FADD18DB31C
:106B5000284807708EE12848857163E4274805704E
:106B600009B02946BDE8F04F40F28270F5F79DBDAF
:106B7000AAF82060294640F25C70F5F796FD09B04E
:106B80005946BDE8F04F40F25D70F5F78EBDAAF8AA
:106B90001E6045E076E1FDE3FDE3FDE3FDE3FDE39B
:106BA000FDE3FDE3FDE3FDE3FDE3FDE3FDE3FDE3E5
:106BB000FDE3FDE35BE1FCE33FE051E0FC09002085
:106BC000CE8C00202A030020290300203E03002051
:106BD0004C0300207C0400205703002051030020B8
:106BE000500300200000002056030020A281002056
:106BF00066030020B0040020B40200205A030020E5
:106C00004FE037E095E0A5E0B1E081E0C3E0B9E016
:106C1000DBE0C9E0EFE0E4E009E1F6E013E11CE1CC
:106C2000294640F25A70F5F740FD09B05946BDE8D3
:106C3000F04F40F25B70F5F738BDAAF822602946A4
:106C400040F25E70F5F731FD594640F25F7009B0D1
:106C500002E0FCE3FCE3FCE3BDE8F04FF5F725BD03
:106C6000FD48857309B02946BDE8F04F40F28370B6
:106C7000F5F71BBD25B1012D02D0022D7FF4D9AE51
:106C8000F54C657429464FF4F560F5F70EFDF349B0
:106C9000087B0628BFF4CDAEDFE800F00D151D25FA
:106CA000332CED48C57309B02946BDE8F04F40F2DA
:106CB0008470F5F7FABC4FF416508860FCF72AFA96
:106CC000062020730BE44FF496408860FCF722FA0C
:106CD0000320207303E44FF416408860FCF71AFA8F
:106CE0000220207370E44FF461408860FCF712FAD0
:106CF000277369E44FF496308860FCF70BFA27732A
:106D000062E44FF4E1308860FCF704FA27735BE437
:106D1000D34A1180C0F80E30294640F28970F5F749
:106D2000C4FC09B05946BDE8F04F40F28A70F5F74F
:106D3000BCBC0DB1012DD5D1CA480570294640F221
:106D4000A970F5F7B2FC0020A9F80000C64804219C
:106D5000017039E4C548068129465120F5F7A5FCA4
:106D600009B05946BDE8F04F5220F5F79EBC05B179
:106D70000125057509B02946BDE8F04F40F286703F
:106D8000F5F793BC457609B02946BDE8F04F4FF4BE
:106D9000F260F5F78ABC057609B02946BDE8F04FE8
:106DA00040F28F70F5F781BCAD4AD180C0F82A302F
:106DB000294640F29470F5F778FC09B05946BDE8D1
:106DC000F04F40F29570F5F770BC05B1012580F8E1
:106DD000305009B02946BDE8F04F40F29170F5F708
:106DE00064BC80F8355009B02946BDE8F04F40F248
:106DF0009B70F5F75ABC80F8345009B02946BDE8BD
:106E0000F04F40F29A70F5F750BC954A9181049981
:106E1000C0F84610294640F29F70F5F746FC09B0CD
:106E20005946BDE8F04F4FF4F460F5F73EBC05B1AC
:106E3000012580F84C5009B02946BDE8F04F40F2DA
:106E40009C70F5F732BC80F8505009B02946BDE877
:106E5000F04F40F2A570F5F728BC80F8515009B00A
:106E60002946BDE8F04F40F2A670F5F71EBC8048F9
:106E70000021017009B02946BDE8F04F40F2A7702B
:106E8000F5F713BCA4F5007CBCF1BF0C1AD0B4F527
:106E9000307F28D0BCF1800C21D0A4F5507CBCF10F
:106EA000030F38D8059809283FF61CAF1FFA8CF05D
:106EB00070490D5409B02946BDE8F04F573080B2F3
:106EC000F5F7F3BB6948068029466320F5F7EDFB2B
:106ED00009B05946BDE8F04F6420F5F7E6BB7DB137
:106EE000654807700FE06148468029466520F5F740
:106EF000DCFB09B05946BDE8F04F6620F5F7D5BB7D
:106F00005D49002008705C48017809B05620BDE852
:106F1000F04FF5F7CABBB4F5517F4BD0DFF85C9169
:106F2000B4F52F7F52D0A4F5007CBCF1BD0C35D058
:106F3000BCF1040C58D0B4F5317F63D0BCF1040C23
:106F40005CD0BCF1020C60D0B4F5327F7DD0B4F5DA
:106F5000337F7DD0A4F2CD22132A7AD81446C4F30D
:106F6000460640F2B36101EB860A491E01EB860139
:106F70000391D007494601EB460400286AD03FF44C
:106F8000B1AE50465946F5F790FB29460398F5F700
:106F90008CFBA4F8368089F8807086E489F8035069
:106FA00089F8827009B02946BDE8F04F40F2A6602A
:106FB000F5F77BBB324C257029465E20F5F775FB53
:106FC000207809B0BDE8F04FF6F74BBC89F80050C7
:106FD000294640F2A560F5F768FB99F800000FF02C
:106FE00069F989F8040060E489F8015009B029467C
:106FF000BDE8F04F40F2AD60F5F757BB2148A0F86F
:10700000008052E489F802504FE4500703D51D4830
:10701000A0F8008049E4B9F80810B9F81000711A16
:107020000844A9F81000A9F80860C1B240F2A760AE
:10703000F5F73BFBB9F8100009B0C0F30721BDE834
:10704000F04F4FF4D560F5F730BBA9F810601BE0A6
:107050002AE059E032E00000B4020020087B002062
:10706000108E00205B0300209C0000203E030020C7
:10707000B00400207804002077040020888D0020D0
:107080007C0400204A030020F1B240F2A760F5F72B
:107090000CFBB9F8100009B0C0F30721BDE8F04FB0
:1070A0004FF4D560F5F701BB89F8205009B02946A7
:1070B000BDE8F04F40F2AF60F5F7F7BAA4F82280D0
:1070C0004FF6FF70804501D1E08602E0B9F8060076
:1070D000E08640F2B16000EB86005946F5F7E5FA2C
:1070E0004FF4D66000EB86002946F5F7DEFAE08E15
:1070F000010A5046F5F7D9FA94F836100398F5F7D7
:10710000D4FA89F8807039E4A4F54072063A13D0B5
:10711000253230D0521E132A6DD8D0B2C107F2D119
:10712000440809EB4406A6F84A804FF6FF708045F4
:107130003CD1A6F85E003DE0012D01D0002DE2D14A
:1071400089F8815029464FF4DB60F5F7AEFA89F8EB
:1071500080700021A9F8101040F2A760F5F7A5FA99
:10716000B9F8100009B0C0F30721BDE8F04F4FF4A3
:10717000D560F5F79ABA89F82150294640F2D960CE
:10718000F5F793FA89F880700021A9F8101040F201
:10719000A760F5F78AFAB9F8100009B0C0F3072123
:1071A000BDE8F04F4FF4D560F5F77FBAB9F80600A7
:1071B000A6F85E0040F2DB6000EB84005946F5F76C
:1071C00074FA40F2DA6000EB84002946F5F76DFAB4
:1071D00036F85E0F010A40F2DD6000EB8400F5F73F
:1071E00064FA40F2DC60317800EB8400F5F75DFA78
:1071F00089F880701DE4A4F54072033A25D0B4F5F7
:10720000417F41D0921E2AD0B4F5487F77D01C3AF6
:1072100076D0521E75D0521E74D0D21F73D0521E1B
:1072200072D0B4F54B7F70D0921E6FD0B4F54D7F05
:107230006DD0083A6CD0511E6BD0491E6AD0C81F61
:10724000D8D19DB3FE4807700EE1FE48857309B0A2
:107250002946BDE8F04F40F28370F5F726BA1DB11C
:10726000012D01D0022DC5D1F64C657429464FF48D
:10727000F560F5F71AFAF449087B06283BD2DFE8F7
:1072800000F00D161E26342DEE48C57309B02946B0
:10729000BDE8F04F40F28470F5F707BA4FF416508E
:1072A0008860FBF737FF0620207324E0D9E04FF415
:1072B00096408860FBF72EFF032020731BE04FF4FD
:1072C00016408860FBF726FF0220207313E04FF47E
:1072D00061408860FBF71EFF27730CE04FF4963087
:1072E0008860FBF717FF277305E04FF4E1308860F3
:1072F000FBF710FF2773D548022101702DE41BE036
:1073000009E024E02CE034E03FE06AE05FE084E064
:1073100071E08EE097E0CE4A1180C0F80E30294629
:1073200040F28970F5F7C1F909B05946BDE8F04F50
:1073300040F28A70F5F7B9B905B10125057509B0B4
:107340002946BDE8F04F40F28670F5F7AEB90576F4
:1073500009B02946BDE8F04F40F28F70F5F7A5B9A6
:10736000457609B02946BDE8F04F4FF4F260F5F7D5
:107370009CB905B1012580F8305009B02946BDE817
:10738000F04F40F29170F5F790B9B14AD180C0F852
:107390002A300FE070E037E28EE2B0E2BFE2CDE2E9
:1073A000E1E2FAE203E311E320E32EE338E350E302
:1073B0005EE36BE3294640F29470F5F776F909B085
:1073C0005946BDE8F04F40F29570F5F76EB980F878
:1073D000355009B02946BDE8F04F40F29B70F5F7F3
:1073E00064B980F8345009B02946BDE8F04F40F246
:1073F0009A70F5F75AB9964A91810499C0F84610E7
:10740000294640F29F70F5F750F909B05946BDE89A
:10741000F04F4FF4F460F5F748B905B1012580F855
:107420004C5009B02946BDE8F04F40F29C70F5F78A
:107430003CB980F8505009B02946BDE8F04F40F201
:10744000A570F5F732B980F85150294602E02FE3D4
:107450002AE363E309B040F2A670BDE8F04FF5F708
:1074600024B977480021017009B02946BDE8F04FE2
:1074700040F2A770F5F719B9DFF8D8A1682C54D0FD
:10748000504640F2AE73807F40F2AF78642C58D003
:107490004FF4F66C652C7AD06D2C79D06E2C78D0A8
:1074A0006F2C77D0702C76D0712C75D0722C74D054
:1074B000732C73D0742C72D0762C71D0772C70D042
:1074C000782C6FD0792C6ED07B2C6DD0872C6CD023
:1074D000882C6BD08E2C6AD08F2C69D0902C68D0E1
:1074E000912C67D0922C7DD0893C042C3FF606AFBE
:1074F0000798B0F5FA7FBFF401AF07985649401DD1
:1075000021F8140040F2C47000EB440080B2294618
:10751000F5F7CBF840F2C57000EB440009B05946CE
:10752000BDE8F04F80B2F5F7C0B81E2D01D28AF841
:107530000E5009B02946BDE8F04F40F2AA70F5F7A9
:10754000B4B8C00702D0AAF8021026E500291AD064
:10755000FBDD42484FF064020088A1EB000101FB13
:1075600002F191FBF0F0AAF81800C1B21846F5F745
:107570009CF8BAF8180009B0C0F307214046BDE8EE
:10758000F04FF5F792B80020AAF8180005E512E0D0
:107590003BE044E04DE06FE07BE088E091E09AE082
:1075A0009CE0A8E0B4E0C0E0CCE0D5E0E0E0EBE0B7
:1075B000F6E001E10FE14008C00702D0AAF804108C
:1075C000EBE400291DD0C0DD25484FF0640200889F
:1075D000A1EB000101FB02F191FBF0F0AAF81A0007
:1075E000C1B200E001E16046F5F75FF8BAF81A00B1
:1075F00009B0C0F30721BDE8F04F40F2B170F5F7D4
:1076000054B80020AAF81A00C7E48AF8135009B049
:107610002946BDE8F04F40F2AB70F5F746B88AF85E
:10762000145009B02946BDE8F04F40F2AC70F5F7B0
:107630003CB83C2D00D33C2505B9012512E00000E3
:10764000B0040020B4020020087B002001000020CC
:10765000108E0020AE8E0020DA040020D40400201A
:10766000D60400208AF8155009B02946BDE8F04F2D
:1076700040F2AD70F5F719B8AAF818602946184617
:10768000F5F713F809B059464046BDE8F04FF5F755
:107690000CB8AAF81A6029466046F5F706F809B052
:1076A0005946BDE8F04F40F2B170F4F7FEBF8AF8DA
:1076B0001C5009B02946BDE8F04F40F2B270F4F713
:1076C000F4BF8AF81D5009B02946BDE8F04F40F2DA
:1076D000B370F4F7EABF8AF81E505EE4FE48868075
:1076E00029465F20F4F7E1FF09B05946BDE8F04FA5
:1076F0006020F4F7DABFF848C68029466120F4F725
:10770000D4FF09B05946BDE8F04F6220F4F7CDBF71
:10771000F148068029466320F4F7C7FF09B05946AF
:10772000BDE8F04F6420F4F7C0BFEB48468029461F
:107730006520F4F7BAFF09B05946BDE8F04F66205E
:10774000F4F7B3BFE548057009B02946BDE8F04F2E
:1077500040F2BB70F4F7A9BF012DBED88AF81F50C4
:1077600009B02946BDE8F04F40F2BF70F4F79DBF65
:10777000032DB2D88AF8205009B02946BDE8F04F51
:1077800040F2C370F4F791BF0A2DA6D8D44885748F
:1077900009B02946BDE8F04F4FF4FA60F4F785BF11
:1077A000012D9AD8CE48C57409B02946BDE8F04FDE
:1077B00040F2D170F4F779BF0698092190FBF1F0FF
:1077C00000B2A9F80000D10702D0C64908800AE437
:1077D000C548077007E4A9F80060D00702D0C14887
:1077E00006800EE4C04807700BE4A9F8006090071B
:1077F00002D5BE48068004E440F2B6308642F0DA94
:10780000B9480221017005E4B9490D73062D4ED225
:10781000DFE805F003101D2A42364FF41650886049
:10782000FBF778FC29461520F4F7AFFEAC4906209B
:1078300008733CE04FF496408860FBF76BFC2946E8
:107840001520F4F7A2FEA649032008732FE04FF499
:1078500016408860FBF75EFC29461520F4F795FE7C
:107860009F490220087322E04FF461408860FBF7D3
:1078700051FC29461520F4F788FE9948077316E055
:107880004FF496308860FBF745FC29461520F4F745
:107890007CFE934807730AE04FF4E1308860FBF701
:1078A00039FC29461520F4F770FE8D48077309B09E
:1078B000BDE8F04FFDF7E8BF072DA4D28D4C257031
:1078C00029463E20F4F761FE2078012810D00328D5
:1078D0000ED006280CD0022803D0042801D0052899
:1078E00091D109B04FF49640BDE8F04F07F017BCB6
:1078F00009B04FF41650BDE8F04F07F010BC7E48B9
:10790000B8F1000F01D0077001E00021017001788B
:1079100009B04FF4EC60BDE8F04FF4F7C6BE15B106
:107920007648077002E075480021017073480178BD
:1079300009B03F20BDE8F04FF4F7B7BE7048744679
:107940000088A8EB00006044AEF80000C1B25B20E4
:10795000F4F7ABFE208809B0C0F30721BDE8F04F73
:107960005C20F4F7A2BE67487446B0F90000301AF4
:1079700000EB8000092190FBF1F06044AEF80000BC
:10798000C1B25B20F4F791FE208809B0C0F3072153
:10799000BDE8F04F5C20F4F788BEA9F80060D0077E
:1079A00002D05048068025E44F48077022E406982C
:1079B000092190FBF1F000B2A9F80000D10702D034
:1079C0004849088016E44848077013E47446AEF846
:1079D0000060F1B25B20F4F768FE208809B0C0F3C4
:1079E0000721BDE8F04F5C20F4F75FBEA9F8006006
:1079F000900702D53D48068080E440F2B6308642CA
:107A0000FADA39480221017078E415B1A9F800705A
:107A100002E00020A9F800003348042101706DE461
:107A2000500703D53848A0F8008067E4374C208819
:107A30002189301A08442081C1B24B20F4F735FE69
:107A4000208909B0C0F30721BDE8F04F4C20F4F7BE
:107A50002CBE2E4C2681F1B24B20F4F726FE208955
:107A600009B0C0F30721BDE8F04F4C20F4F71DBE6C
:107A70002648A0F80A8029464720F4F716FE09B0E8
:107A80005946BDE8F04F4820F4F70FBE1F48A0F854
:107A90000C8029464920F4F708FE09B05946BDE894
:107AA000F04F4A20F4F701BE5DB1194807700BE0B2
:107AB0001848057009B02946BDE8F04F5020F4F78A
:107AC000F4BD1349002008701148017809B0562010
:107AD000BDE8F04F20E000003E030020C00400207D
:107AE000B40200202A0300209C0000204C03002048
:107AF000087B0020FC0200205303002054030020D8
:107B000060030020620300204A030020348C002020
:107B100077040020FB020020F4F7C7BDA4F58062C3
:107B2000DE3A3DD0521E45D0B4F59C6F59D0921E1E
:107B30004ED0521E63D0521E64D0521E65D0521ECB
:107B400067D0921E69D0B4F59D6F7DD0921E71D022
:107B5000521E7AD0521E79D0B2F5E06276D0A4F5EA
:107B60008062EC3A73D0B2F5E06270D0A4F5806226
:107B7000ED3A3FF441AF521E6AD0A2F69A62132A40
:107B800067D8FA49089821F81200101C7FF434AF26
:107B900009B02946BDE8F04F40F2BA70F4F785BD50
:107BA000F348290604D4017821F080010170CCE467
:107BB0000570CAE4002DFAD0142D00D31425ED4829
:107BC0002946057009B04520BDE8F04FF4F76DBDBA
:107BD000E948057009B02946BDE8F04F4D20F4F79B
:107BE00064BD002DE3D0142D00D31425E3482946AD
:107BF000057009B04620BDE8F04FF4F756BDE048E7
:107C00000570A2E4DF4806809FE4DF48A0F800800A
:107C10009BE4DE48A0F8008097E4DD488680294692
:107C20005F20F4F742FD09B05946BDE8F04F6020EF
:107C3000F4F73BBDD648068029466320F4F735FDAE
:107C40005946642009B005E008E014E020E02CE08B
:107C500038E043E0BDE8F04FF4F727BDCC48C680DC
:107C600029466120F4F721FD09B05946BDE8F04FDF
:107C70006220F4F71ABDC648468029466520F4F70D
:107C800014FD09B05946BDE8F04F6620F4F70DBD6C
:107C9000BF48068129465120F4F707FD09B059462F
:107CA000BDE8F04F5220F4F700BDB948468129469F
:107CB0005320F4F7FAFC09B05946BDE8F04F5420C0
:107CC000F4F7F3BCB34C257029465E20F4F7EDFCC5
:107CD000207809B0BDE8F04FF5F7C3BDA4F53062D8
:107CE000B83A33D0521E3BD0521E43D0121F4BD055
:107CF000153A6ED0521E132A78D802F00108A64811
:107D00000770A6480021018440F25C70F4F7CCFCB7
:107D1000002140F25D70F4F7C7FCA4F6D430C0F344
:107D2000460040F2347101EB8007491C01EB8009E9
:107D3000B8F1000F5BD038462946F4F7B5FC09B01E
:107D400048465946BDE8F04FF4F7AEBC944805707C
:107D500009B02946BDE8F04F40F20270F4F7A5BC27
:107D60008AF8195009B02946BDE8F04F40F2037077
:107D7000F4F79BBC8AF81A5009B02946BDE8F04FC9
:107D800040F20470F4F791BC012D02D0002D7FF475
:107D90000EAF8448057029464FF4DB60F4F784FC8D
:107DA0007D4807700024AAF82040002140F25D7051
:107DB000F4F77AFC002140F25C70F4F775FC7A4825
:107DC000047009B00021BDE8F04F40F23170F4F7C3
:107DD0006BBC0A2DBFF4EBAE73480570294640F228
:107DE0003170F4F761FC6C4807700DE465E0A4F6AF
:107DF000D430C0F3460040F2327202EB800840F209
:107E00003372711C02EB800A2FD0EEB36348817D80
:107E10003846F4F749FC6148C08A010A4846F4F73D
:107E200043FC40462946F4F73FFC50465946F4F7D8
:107E30003BFCA4F53060D438D7D15B4800780128EA
:107E4000D3D15A48554C0088301A2084C1B240F230
:107E50005C70F4F729FC208C09B0C0F30721BDE861
:107E6000F04F40F25D70F4F71FBC4046FF21F4F77D
:107E70001BFC5046FF21F4F717FC3846FF21F4F7AE
:107E800013FC4846FF2100E004E009B0BDE8F04FD4
:107E9000F4F70ABC40460021F4F706FC50460021E6
:107EA000F4F702FC38460021F4F7FEFB09B048461F
:107EB000BDE8F04F0021F4F7F7BBA4F53062E83AD3
:107EC00050D01C3A51D0B4F53F6F75D0133274D0F6
:107ED000521E73D0133A72D0521E71D0521E70D0FF
:107EE000521E6FD0143A6ED0521E6DD0521E6CD0FE
:107EF000521E6BD0D21F6AD0521E69D0521E68D05B
:107F0000521E67D0B4F5436F7DD0083A7CD0511E25
:107F10007BD0491E7AD0C81F79D0401E78D0401E31
:107F200077D0401E76D0083875D02148353173D0CF
:107F3000491E72D0B4F5406F70D0891E6FD0491EB3
:107F40006ED0491E7FF451AF468129464FF4F06050
:107F5000F4F7ABFB09B05946BDE8F04F40F2817031
:107F6000F4F7A3BB1348857131E434E0A28100200B
:107F7000F6020020F8020020FA020020F902002098
:107F8000290300202A0300204C0300204A0300207C
:107F90003E0300207C04002051030020FC09002047
:107FA00059030020560300205703002066030020D9
:107FB000988C0020B402002035E016E042E050E04A
:107FC00059E062E0A7E0B7E0C1E0D1E0D9E0E1E04C
:107FD000ECE0FCE005E1FE48057009B02946BDE88B
:107FE000F04F40F28270F4F760BBAAF82060294697
:107FF00040F25C70F4F759FB09B05946BDE8F04F08
:1080000040F25D700DE008E1F5E012E11BE124E1D2
:1080100032E13EE143E146E150E15DE178E169E1D1
:1080200084E1F4F742BBAAF81E60294640F25A7078
:10803000F4F73BFB09B05946BDE8F04F40F25B70E6
:10804000F4F733BBAAF82260294640F25E70F4F7D9
:108050002CFB09B05946BDE8F04F40F25F70F4F7D1
:1080600024BBDC48857309B02946BDE8F04F40F2D7
:108070008370F4F71ABBD748C57309B02946BDE829
:10808000F04F40F28470F4F710BB25B1012D02D0FF
:10809000022D7FF469AFCF4C657429464FF4F5602B
:1080A000F4F703FBCC49087B062830D2DFE800F068
:1080B000030B131B29224FF416508860FBF72AF894
:1080C0000620207323E04FF496408860FBF722F8E7
:1080D000032020731BE04FF416408860FBF71AF86A
:1080E0000220207313E04FF461408860FBF712F820
:1080F00027730CE04FF496308860FBF70BF827737A
:1081000005E04FF4E1308860FBF704F82773B348CB
:108110000221017047E40DB1012DFBD1B04805707B
:10812000294640F2A970F4F7C0FA0020A9F800002F
:10813000AC480421017036E405B10125057509B08C
:108140002946BDE8F04F40F28670F4F7AEBAA64A71
:108150001180C0F80E30294640F28970F4F7A5FA74
:1081600009B05946BDE8F04F40F28A70F4F79DBA65
:10817000057609B02946BDE8F04F40F28F70F4F75C
:1081800094BA457609B02946BDE8F04F4FF4F26045
:10819000F4F78BBA05B1012580F8305009B02946B3
:1081A000BDE8F04F40F29170F4F77FBA8E4AD1806B
:1081B000C0F82A30294640F29470F4F776FA09B0F4
:1081C0005946BDE8F04F40F29570F4F76EBA80F86A
:1081D000345009B02946BDE8F04F40F29A70F4F7E8
:1081E00064BA80F8355009B02946BDE8F04F40F236
:1081F0009B70F4F75ABA7C4A91810499C0F84610F2
:10820000294640F29F70F4F750FA09B05946BDE88C
:10821000F04F4FF4F460F4F748BA05B1012580F847
:108220004C5009B02946BDE8F04F40F29C70F4F77D
:108230003CBA80F8505009B02946BDE8F04F40F2F2
:10824000A570F4F732BA80F8515009B02946BDE85C
:10825000F04F40F2A670F4F728BA15B163480770E2
:1082600002E062480021017009B02946BDE8F04FE4
:1082700040F2A770F4F719BA012D06D0002D7FF453
:1082800049AF5B490420087091E459490320087004
:108290008DE4002DF8D156490520087087E4544933
:1082A0000620087083E4534880F804B045715249B1
:1082B000072008704748A0F81A8078E4068029460D
:1082C00040F27670F4F7F1F909B05946BDE8F04F85
:1082D00040F27770F4F7E9B9468029464FF4EF6031
:1082E000F4F7E3F909B05946BDE8F04F40F2797070
:1082F000F4F7DBB9C680294640F27C70F4F7D5F973
:1083000009B05946BDE8F04F40F27D70F4F7CDB9A1
:108310008680294640F27A70F4F7C7F909B05946C9
:10832000BDE8F04F40F27B70F4F7BFB906812946F3
:1083300040F27E70F4F7B9F909B05946BDE8F04F44
:1083400040F27F70F4F7B1B9012080F313882B4815
:1083500001682B4A01F4E06111430160BFF3408FD3
:10836000FEE77CB5274B0125274E5418B0F5FA6F70
:108370002AD0A0F5E061D33918D0891C4CD0091F50
:108380004DD0491C51D0891F1F2954D8C80645D14A
:1083900003F10A004021054619F07BF9E11D02B006
:1083A0002846BDE87040402219F05AB9607901288A
:1083B00034D10EF07BFF7C21124819F06AF9F57078
:1083C000BDE87C4006F039B860791870F5701DE0A2
:1083D0005A030020B4020020087B00200100002086
:1083E0005B0300209C000020108E0020B0040020C1
:1083F0000000002010030020FD0200200CED00E032
:108400000400FA05B89A0020EF02002006F015F8E3
:108410000EF04CFFFFF798FF607958707CBD6079D3
:10842000217900EB012098807CBD6079217900EBF7
:10843000012058807CBDA0F2FA710F290ED80807E0
:10844000F8D1FF482021054619F023F9E11D02B0BB
:108450002846BDE87040202219F002B9A0F500615D
:108460000A3922D00C39E5D1A0F61600062190FB7E
:10847000F1F201FB12000028DCD1207A8DF8000017
:10848000A07A8DF80100207B8DF80200A07B8DF88A
:108490000300207C8DF80400A07C8DF80500684660
:1084A0000FF0F5FEE74805707CBDA0F60A000C2130
:1084B00090FBF1F201FB12000028F5D1207A03F8BD
:1084C0006A0FA07A5870207B9870A07BD870207CAF
:1084D0001871A07C5871207D9871A07DD871207E84
:1084E0001872A07E5872207F9872A07FD8727CBDCF
:1084F0002DE9F05F8846002819D0042817D00627F8
:1085000008EB0704E078A17800EB012086B26078E0
:1085100010280ED006286ED1A6F5FA6064286BD814
:10852000424639463046BDE8F05F002319E7002790
:10853000E6E7282E0CD0A6F51C500F3845F6E301CF
:10854000884233D8424639463046FDF7BBF937E01A
:10855000DFF8F49299F82A00012831D1A0790C288B
:108560002ED1207A89F81400A07A89F81500207B92
:1085700089F81600A07B89F81700207C89F818007C
:10858000A07C89F81900002509EB0500017D05F1A3
:108590002800F3F7FAFF6D1CEDB2062DF4D3AB49BA
:1085A00001200870002089F82A0009E0A6F5FA6089
:1085B000642805D80023424639463046FFF7D1FEED
:1085C000DFF88CA2DFF88C929AF80000D42809D04A
:1085D000D52807D0342805D0D22803D0D32801D0FD
:1085E000D9281CD1A6F2CB20072818D8A0791428A6
:1085F00015D8002510E031E032E0781900EB080BC7
:1086000005F261709BF80710F4F74FF89BF807002C
:1086100009F805006D1CEDB2A079A842EDD89AF8D2
:108620000000D62801D0D72818D1A6F28536072E0B
:1086300014D8A079142811D800250CE0781900EB83
:10864000080605F26170F179F4F72FF8F07909F86E
:1086500005006D1CEDB2A079A842EFD8BDE8F09FEF
:10866000627921793046BDE8F05FFDF70FBA7449B1
:108670004A39B0F5FA6F1FD0A0F5E062D13A19D0AF
:10868000521E1BD0921E1BD0521E1BD0521E1BD03E
:10869000B0F5FB6F1AD0111F1F2919D86848403850
:1086A000CA1701EBD26222F01F02891AC9B230F850
:1086B000110070474878704708787047887970478C
:1086C0004888704788887047C8797047087A70472B
:1086D000A0F2FA710F290AD85948CA1701EB127291
:1086E00022F00F02891AC9B230F811007047A0F6C3
:1086F0000A0103290AD852482030CA1701EB9272A6
:1087000022F00302891AC9B2405C7047A0F60E013C
:1087100003290AD84A482430CA1701EB927222F082
:108720000302891AC9B2405C7047A0F612010329FE
:108730000AD843482830CA1701EB927222F003028C
:10874000891AC9B2405C7047A0F61600052809D8FE
:108750003B4A2C32062190FBF1F301FB1300C0B21F
:10876000105C7047002070472DE9F34FD3B0002212
:108770009046539804AD00280BD05398042808D095
:108780004FF00608002000212954401CC0B20628E2
:10879000FAD3549810F80800002869D0549901EBD6
:1087A00008067178F378B47803EB04239BB2029344
:1087B00073790393062406295FD010297ED0DFF851
:1087C000889003297BD0A9F24C414978192977D1A7
:1087D000A9F51674511C8DB2A05403F05CFF70789B
:1087E000691C8EB2605503F056FF99F80400711CA5
:1087F0008DB2A05503F04FFF99F80000691C8EB2AE
:10880000605503F048FF99F80100711C8DB2A05526
:1088100003F041FF99F80200691C8EB2605503F025
:108820003AFF99F80300711C8DB2A05503F033FF95
:1088300009480078691C89B26055084802780FE041
:10884000029B0020E7040020087B0020B3020020E8
:1088500004000020747C0020D7020020D6020020F3
:10886000481C80B2625455B0BDE8F04FFDF704B823
:1088700055B0BDE8F04FFCF7FBBE539888B3539852
:1088800004282FD0549800788DF810005498407820
:108890008DF8110000208DF812008DF813008DF86E
:1088A00014008DF81540549A08EB0001525C6A548C
:1088B000401CC0B20628F6D3539802E039E093E09A
:1088C0000CE0052829D008F1060204A9FD4818F09B
:1088D000C7FEFD4808F10608A0F8008055B0BDE8C5
:1088E000F08FFFE70020F949CA8A09E054990B5C30
:1088F000414608F101081FFA88F86B54401CC0B2C9
:108900009042F3D3424604A9F14818F0A9FE55B0AD
:108910004046BDE8F04FFCF7AFBF08F1060204A9DE
:10892000EC4818F09DFEEC4808F10608A0F800801D
:10893000D4E7539858B35398042828D05498007813
:108940008DF81000549840788DF8110000208DF8B3
:1089500012008DF813008DF814008DF81540549A0C
:1089600008EB0001525C6A54401CC0B20628F6D3E2
:10897000539805282CD008F1060204A9D14818F014
:108980006FFED14808F10608A0F80080A6E7002491
:10899000549808EB0401405C685403F07CFE641CAE
:1089A000E4B2062CF4D3CD48017808EB0400295436
:1089B000CB49284409784170C548DDE90412743870
:1089C000C0E91D1255B00820BDE8F04FFCF754BFB8
:1089D00008F1060204A9BF4818F042FEBE4808F19B
:1089E0000608A0F8008079E705F8080005EB080400
:1089F0006170039949005291A17003F04CFE6078B8
:108A000003F049FEA07803F046FE08F103040020BD
:108A10005190DFF8D0A2B44FDFF8D0B2B44E03F0DB
:108A2000AFBC51990298084480B264287BD20328D5
:108A300012D8002119F800204F92601C80B22955ED
:108A4000431C4F9A9CB22A54084603F024FE4F98C8
:108A500003F021FE03F090BC042833D0052841D058
:108A600006284FD007285FD0082876D00B286DD075
:108A700009286CD00E286BD00F286AD0102869D036
:108A8000632868D0152867D01D2877D0252876D090
:108A9000262875D0272874D0A0F12801052971D87F
:108AA00089B2002049440A7D4F92611C89B2285541
:108AB0004B1C4F9A9CB26A5403F0EDFD4F9803F0A3
:108AC000EAFDC7E7002044224F92611C89B2285575
:108AD0004B1C4F9A9CB26A5403F0DDFD4F9803F093
:108AE000DAFDB7E7002000224F92611C89B22855B9
:108AF0004B1C4F9A9CB26A5403F0CDFD4F9803F083
:108B0000CAFDA7E7002099F804204F92611C89B2A2
:108B100028554B1C4F9A9CB26A5403F0BCFD4F98E9
:108B200003F0B9FD96E76BE2002072490A784F9294
:108B3000611C89B228554B1C4F9A9CB26A5403F0B1
:108B4000AAFD4F9803F0A7FD84E706E01BE02FE0A5
:108B50003FE060E071E081E092E0002099F80F20B2
:108B60004F92611C89B228554B1C4F9A9CB26A5493
:108B700003F091FD4F9803F08EFD6BE791E0BFE0AD
:108B8000D1E0E3E0F3E0002050900F20F3F7CCFCBD
:108B90004F90611C509889B228554A1C4F9894B246
:108BA0006854509803F077FD4F9803F074FD51E737
:108BB000002051490A784F92611C89B228554B1CFC
:108BC0004F9A9CB26A5403F066FD4F9803F063FD20
:108BD00040E7002047490978D22916D0D32914D07C
:108BE000D92912D0D62913D0D72911D006214F91D7
:108BF000611C89B228554B1C4F9A9CB26A5403F0F1
:108C00004AFD4F9803F047FD24E707214F91EFE716
:108C100008214F91ECE7002199F80C204F92601C3D
:108C200080B22955431C4F9A9CB22A54084603F03F
:108C300032FD4F9803F02FFD0CE7002099F80D202E
:108C40004F92611C89B228554B1C4F9A9CB26A54B2
:108C500003F021FD4F9803F01EFDFBE6002199F87B
:108C600010204F92601C80B22955431C4F9A9CB231
:108C70002A54084603F00FFD4F9803F00CFDE9E677
:108C8000002099F812204F92611C89B228554B1C84
:108C90004F9A9CB26A5403F0FEFC4F9803F0FBFC21
:108CA000D8E6002015490A784F92611C89B22855F0
:108CB0004B1C4F9A9CB26A5403F0EDFC4F9803F0A2
:108CC000EAFCC7E628740020B0020020B4020020AD
:108CD000B0780020C4940020EC040020D7020020CB
:108CE000D6020020AE8E0020FC090020108E00204D
:108CF000228E0020040000209E000020060000209C
:108D0000FD480188C1F30720CAB24F92611C89B2A5
:108D100028554B1C4F9A9CB26A5403F0BCFC4F98E8
:108D200003F0B9FC96E6F4480168080EC1F3074366
:108D30004F93611C89B228554A1C4F9B94B26B54C7
:108D400003F0A9FC4F9803F0A6FC83E60020EB4952
:108D50004A794F92611C89B228554B1C4F9A9CB29C
:108D60006A5403F098FC4F9803F095FC72E62E28A5
:108D700015D0A0F12F01032922D889B2002049443F
:108D80008B7E4F93611C89B228554A1C4F9B94B22D
:108D90006B5403F080FC4F9803F07DFC5AE60020F2
:108DA00099F81E204F92611C89B228554B1C4F9A8E
:108DB0009CB26A5403F06FFC4F9803F06CFC49E6D8
:108DC000A0F13301032911D889B200204944CB7F97
:108DD0004F93611C89B228554A1C4F9B94B26B5427
:108DE00003F059FC4F9803F056FC33E6A0F137012D
:108DF000032912D889B20020494491F823204F92C8
:108E0000611C89B228554B1C4F9A9CB26A5403F0DE
:108E100042FC4F9803F03FFC1CE63B281BD03C284B
:108E20002AD03D283AD0A0F13E01032947D888B284
:108E30000021484490F82B204F92601C80B22955A5
:108E4000431C4F9A9CB22A54084603F024FC4F98C6
:108E500003F021FCFEE5002099F827204F92611CC9
:108E600089B228554B1C4F9A9CB26A5403F013FCEC
:108E70004F9803F010FCEDE5B9F82810080ACAB2C3
:108E80004F92611C89B228554B1C4F9A9CB26A5470
:108E900003F001FC4F9803F0FEFBDBE5002099F89E
:108EA0002F204F92611C89B228554B1C4F9A9CB2BF
:108EB0006A5403F0F0FB4F9803F0EDFBCAE5A0F114
:108EC0004201032913D888B20021484490F8302089
:108ED0004F92601C80B22955431C4F9A9CB22A5471
:108EE000084603F0D8FB4F9803F0D5FBB2E5A0F19C
:108EF0004601032913D888B20021484490F8342051
:108F00004F92601C80B22955431C4F9A9CB22A5440
:108F1000084603F0C0FB4F9803F0BDFB9AE54A28D2
:108F200017D04B2827D04C2837D0502846D05D2862
:108F300055D0002000224F92611C89B228554B1C4D
:108F40004F9A9CB26A5403F0A6FB4F9803F0A3FB20
:108F500080E5002199F838204F92601C80B2295595
:108F6000431C4F9A9CB22A54084603F094FB4F9836
:108F700003F091FB6EE5B9F83A10080ACBB24F93B3
:108F8000611C89B228554A1C4F9B94B26B5403F064
:108F900082FB4F9803F07FFB5CE5002099F83C20B2
:108FA0004F92611C89B228554B1C4F9A9CB26A544F
:108FB00003F071FB4F9803F06EFB4BE50020504926
:108FC0000A784F92611C89B228554B1C4F9A9CB26B
:108FD0006A5403F060FB4F9803F05DFB3AE5002014
:108FE00099F82A204F92611C89B228554B1C4F9A40
:108FF0009CB26A5403F04FFB4F9803F04CFB29E5F9
:10900000A0F540613E3932D0491E41D0B0F5446FE1
:1090100060D0C91E4DD0491E6DD0A0F58061D739F2
:109020007AD0B0F59B6F78D0891E77D0491E76D064
:10903000491E75D0491E74D0491E73D0A1F6AB618C
:10904000132970D82F4830F81100C0F30721C2B29D
:109050004F92601C80B22955431C4F9A9CB22A54EF
:10906000084603F018FB4F9803F015FBF2E40020CC
:1090700025490A784F92611C89B228554B1C4F9A9A
:109080009CB26A5403F007FB4F9803F004FBE1E441
:1090900000201E490A784F92611C89B228554B1C4A
:1090A0004F9A9CB26A5403F0F6FA4F9803F0F3FA21
:1090B000D0E4002016490A784F92611C89B22855E5
:1090C0004B1C4F9A9CB26A5403F0E5FA4F9803F098
:1090D000E2FABFE400200F490A784F92611C89B27E
:1090E00028554B1C4F9A9CB26A5403F0D4FA4F98FF
:1090F00003F0D1FAAEE417E00C000020B402002027
:1091000063000020A2810020A4000020A500002010
:10911000A7000020A600002017E03BE028E04BE07D
:109120005CE06DE07EE08FE00020FA490A784F9223
:10913000611C89B228554B1C4F9A9CB26A5403F0AB
:10914000AAFA4F9803F0A7FA84E4F3490888000AC2
:109150000988CAB24F92611C89B228554B1C4F9A9C
:109160009CB26A5403F097FA4F9803F094FA71E4B2
:109170000020E949C91E8A794F92611C89B228559D
:109180004B1C4F9A9CB26A5403F085FA4F9803F037
:1091900082FA5FE40020E049C91E4A794F92611CBF
:1091A00089B228554B1C4F9A9CB26A5403F073FA4B
:1091B0004F9803F070FA4DE40020D749C91ECA79D0
:1091C0004F92611C89B228554B1C4F9A9CB26A542D
:1091D00003F061FA4F9803F05EFA3BE40020CE49B9
:1091E000C91E0A784F92611C89B228554B1C4F9AB0
:1091F0009CB26A5403F04FFA4F9803F04CFA29E4FA
:109200000020C549C91E4A784F92611C89B2285571
:109210004B1C4F9A9CB26A5403F03DFA4F9803F0EE
:109220003AFA17E40020BC49C91E8A784F92611CA3
:1092300089B228554B1C4F9A9CB26A5403F02BFA02
:109240004F9803F028FA05E4A0F540614E391DD08F
:10925000A0F57D41F2392AD0A0F51C510F3945F611
:10926000E302914234D8FCF7A2FB010AC2B24F924A
:10927000601C80B22955431C4F9A9CB22A54084660
:1092800003F009FA4F9803F006FA1AE40020A34904
:109290000A784F92611C89B228554B1C4F9A9CB298
:1092A0006A5403F0F8F94F9803F0F5F909E4002047
:1092B0009B490A784F92611C89B228554B1C4F9AE2
:1092C0009CB26A5403F0E7F94F9803F0E4F908E41C
:1092D000A0F5FA61642912D8FFF7C9F90146080A16
:1092E000CBB24F93611C89B228554A1C4F9B94B254
:1092F0006B5403F0D0F94F9803F0CDF912E4B0F5B8
:10930000357F05D887490978D42979D0D52977D0F0
:1093100040F28F31884205D282490978D6296ED031
:10932000D729FCD0932804D27E490978342901F04A
:10933000CD83C82801F03287C92801F04087CA28A8
:1093400001F04F87CB2801F06087CC2801F07087AF
:10935000CD2801F0A187CE2801F0B187CF2801F0F8
:10936000C287D02801F0D087D12801F0DE87D2282B
:1093700001F0EC87D32801F0FA87D42802F00980A5
:10938000D52802F01A80D62802F02A80A0F5806144
:10939000CF3920D0B0F59A6F02F04580891E02F0D7
:1093A0003180491E032902F24F8000215E4B184490
:1093B000A0F5805090F82E3B4F93601C80B2295549
:1093C000421C4F9B94B22B54084603F064F94F980B
:1093D00003F061F918E455480088010AC2B24F92BF
:1093E000601C80B22955431C4F9A9CB22A540846EF
:1093F00003F051F94F9803F04EF905E400E0F4E36F
:1094000079283DD065284CD064285DD0B0F5987F90
:1094100024D0A0F58071753920D0B0F5BB7F76D00F
:10942000B0F5F27F74D09E3960D0491E032970D800
:1094300000213D4B1844A0F5805090F8EC3D4F932F
:10944000601C80B22955421C4F9B94B22B54084695
:1094500003F021F94F9803F01EF910E4B888010ACF
:10946000C2B24F92601C80B22955431C4F9A9CB2E5
:109470002A54084603F00FF94F9803F00CF90FE453
:1094800000202B490A784F92611C89B228554B1C49
:109490004F9A9CB26A5403F0FEF84F9803F0FBF821
:1094A0000FE4B889C0F30721C2B24F92601C80B2AA
:1094B0002955431C4F9A9CB22A54084603F0EBF8F6
:1094C0004F9803F0E8F82DE4B98AC1F30720CAB237
:1094D0004F92611C89B228554B1C4F9A9CB26A541A
:1094E00003F0D9F84F9803F0D6F81BE40020114997
:1094F0000A784F92611C89B228554B1C4F9A9CB236
:109500006A5403F0C8F84F9803F0C5F80AE413E072
:1095100024E034E0A10400208900002005000020A0
:109520000800002004000020780400201A03002016
:109530005403002077040020F88A010AC2B24F9237
:10954000601C80B22955431C4F9A9CB22A5408468D
:1095500003F0A1F84F9803F09EF807E40020FE49BD
:109560000A784F92611C89B228554B1C4F9A9CB2C5
:109570006A5403F090F84F9803F08DF80EE4B0F5BC
:10958000067F66D0A0F50071193950D0491E79D0F8
:10959000491E70D0B0F5B97F6ED0A8316DD0B0F54E
:1095A000BA7F6BD0BA286AD0563169D0B0F58F7FB8
:1095B00067D0891E79D0B0F5907F77D04A3976D0C0
:1095C000B0F5E27F74D05C3973D0B0F5EF7F71D025
:1095D000B0F5F07F6FD0B0F5E37F6DD0483113293F
:1095E0006BD8C8B24108019100F00100002877D083
:1095F000019840F20C7101EB8000F3F758F850909D
:10960000019840F20B7101EB8000F3F750F84F9096
:10961000601C509980B22955421C4F9994B229542C
:10962000509803F038F84F9803F035F812E4CB481F
:10963000C188080ACBB24F93611C89B228554A1CD5
:109640004F9B94B26B5403F026F84F9803F023F825
:1096500011E40020C1490A794F92611C89B2285552
:109660004B1C4F9A9CB26A5403F015F84F9803F0C4
:1096700012F812E406E021E047E032E069E07BE026
:1096800054E09EE0B5480088010AC2B24F92601CC7
:1096900080B22955431C4F9A9CB22A54084602F0C6
:1096A000FAFF4F9802F0F7FF08E477E0AEE09CE0A5
:1096B000CFE0BEE0DEE0EFE0FEE01FE1A748018979
:1096C000080ACBB24F93611C89B228554A1C4F9BA4
:1096D00094B26B5402F0DFFF4F9802F0DCFF05E418
:1096E000FBE09F480088C0F30721C2B24F92601C84
:1096F00080B22955431C4F9A9CB22A54084602F066
:10970000CAFF4F9802F0C7FF08E4002095490A7885
:109710004F92611C89B228554B1C4F9A9CB26A54D7
:1097200002F0B9FF4F9802F0B6FF11E48E4881882D
:10973000C1F30720CAB24F92611C89B228554B1C55
:109740004F9A9CB26A5402F0A6FF4F9802F0A3FF12
:1097500010E486480088010AC2B24F92601C80B2B1
:109760002955431C4F9A9CB22A54084602F093FF95
:109770004F9802F090FF0FE400217D4802784F924D
:10978000601C80B22955431C4F9A9CB22A5408464B
:1097900002F081FF4F9802F07EFF0EE472480188CC
:1097A000C1F30720CAB24F92611C89B228554B1CE5
:1097B0004F9A9CB26A5402F06EFF4F9802F06BFF12
:1097C0000CE46948C088C0F30721C2B24F92601C04
:1097D00080B22955431C4F9A9CB22A54084602F085
:1097E0005AFF4F9802F057FF09E4002061490A78B8
:1097F0004F92611C89B228554B1C4F9A9CB26A54F7
:1098000002F049FF4F9802F046FF2FE45648418886
:10981000C1F30720CAB24F92611C89B228554B1C74
:109820004F9A9CB26A5402F036FF4F9802F033FF11
:109830001CE40020BA7E4F92611C89B228554B1C53
:109840004F9A9CB26A5402F026FF4F9802F023FF11
:109850000CE400217A7E4F92601C80B22955431C93
:109860004F9A9CB22A54084602F015FF4F9802F016
:1098700012FF0CE4B88B010AC2B24F92601C80B296
:109880002955431C4F9A9CB22A54084602F003FF04
:109890004F9802F000FF0BE400203A7E4F92611CCB
:1098A00089B228554B1C4F9A9CB26A5402F0F3FEC1
:1098B0004F9802F0F0FE0CE400202F490A784F92F6
:1098C000611C89B228554B1C4F9A9CB26A5402F015
:1098D000E2FE4F9802F0DFFE0CE4019840F20A71BC
:1098E00001EB8000F2F7E3FE5090019840F209711D
:1098F00001EB8000F2F7DBFE4F9089E6A0F5807166
:10990000C73919D0491E13295CD8C8B24108019142
:1099100000F00100F8B1019840F2357101EB8000D0
:10992000F2F7C5FE5090019840F2347101EB8000CF
:10993000F2F7BDFE4F9036E0002010490A784F92B2
:10994000611C89B228554B1C4F9A9CB26A5402F094
:10995000A2FE4F9814E016E09B000020CE8C002061
:109960002A030020290300203E0300204C0300208E
:10997000280300207C040020560300205703002009
:1099800002F089FE05E4019840F2337101EB80009A
:10999000F2F78DFE5090019840F2327101EB800099
:1099A000F2F785FE4F90601C509980B22955421CF9
:1099B0004F9994B22954509802F06DFE4F9802F0DE
:1099C0006AFE0AE4B0F5F17F7CD0A0F58071E3393E
:1099D00079D0891C78D0091F77D0B0F5F47F75D085
:1099E000091F74D0B0F5F57F72D0B0F5E17F70D06B
:1099F00026316FD01C396ED0B0F5EE7F6CD0891C4B
:109A00006BD00E396AD0B0F5F67F68D0091F67D0E9
:109A1000B0F5F87F77D0891E76D0B0F5F37F74D09B
:109A2000B0F5FA7F72D0091F71D0B0F5FB7F6FD00F
:109A3000891E6ED0B0F5FC7F6CD0891E6BD0B0F55E
:109A4000FD7F69D0B0F5FF7F67D0891F79D0B0F571
:109A5000007F77D0891E76D0491E75D0491E74D0FC
:109A6000B0F5017F72D0B0F5027F70D0891F6FD042
:109A7000491E6ED0491E6DD0B0F5037F6BD0891E94
:109A80006AD0491E69D0091F68D0B83967D0B0F5CF
:109A9000617FFBD0491E092973D889B2F84A12F8B0
:109AA000110002EB41014A784F92611C89B228559E
:109AB0004B1C4F9A9CB26A5402F0EDFD4F9802F095
:109AC000EAFD04E42AE00CE04AE05BE07CE06AE0C6
:109AD0009EE0AFE08AE0BFE0E6E0CFE0FDE01EE11F
:109AE0000CE1F98CC1F30720CAB24F92611C89B214
:109AF00028554B1C4F9A9CB26A5402F0CCFD4F98EB
:109B000002F0C9FD66E42EE11AE151E163E13BE1B7
:109B100081E170E1A3E18EE1D6E1E9E1B88CC0F327
:109B20000721C2B24F92601C80B22955431C4F9A44
:109B30009CB22A54084602F0AEFD4F9802F0ABFDED
:109B400048E4ADE1F6E1E4E105E215E23BE24DE295
:109B500026E25CE26CE290E27BE29FE2B2E2C2E2E9
:109B60000020C8498A794F92611C89B228554B1C44
:109B70004F9A9CB26A5402F08EFD4F9802F08BFD12
:109B800028E4C1E20020C0490A784F92611C89B2E2
:109B900028554B1C4F9A9CB26A5402F07CFD4F989A
:109BA00002F079FD16E4798D080ACAB24F92611C61
:109BB00089B228554B1C4F9A9CB26A5402F06BFD37
:109BC0004F9802F068FD05E4398D080ACAB24F9239
:109BD000611C89B228554B1C4F9A9CB26A5402F002
:109BE0005AFD4F9802F057FD07E4B6E2398CC1F3F5
:109BF0000720CBB24F93611C89B228554A1C4F9B5A
